:100000000C9451130C941A8A0C94EF890C94C489A3
:100010000C9499890C946E890C9443890C941889DA
:100020000C94ED880C9482130C9482130C9482131C
:100030000C9482130C9482130C9482130C948213EC
:100040000C9482130C9482130C9482130C948213DC
:100050000C9482130C9482130C9482130C946CB342
:100060000C9482130C945F900C9435900C94821332
:100070000C9482130C9482130C9482130C948213AC
:100080000C9482130C9482130C9482130C9482139C
:100090000C9482130C9482130C9482130C942828D1
:1000A0000C9482130C9482130C9482130C9482137C
:1000B0000C9482130C9482130C9482130C9482136C
:1000C0000C9482130C9482130C9482130C9482135C
:1000D0000C9482130C9482130C9482130C9482134C
:1000E0000C94821307634236B79BD8A71A39685617
:1000F00018AEBAAB558C1D3CB7CC5763BD6DEDFD4A
:10010000753EF6177231BF000000803F0800000006
:10011000BE922449123EABAAAA2ABECDCCCC4C3EFC
:1001200000000080BEABAAAAAA3E00000000BF00EB
:100130000000803F0000000000084178D3BB4387E7
:10014000D1133D190E3CC3BD4282AD2B3E68EC82FB
:1001500076BED98FE1A93E4C80EFFFBE01C4FF7F80
:100160003F00000000000C9432930C942F8C0C94F0
:10017000D3810C942B810C948A9D0C9495390C940A
:10018000EC210C94511C0C94BF130C94093C0C945E
:10019000AD3B0C945AAA0C949A130C94FA350C9417
:1001A000D1480C94281B0C94C1680C94B0180C9482
:1001B0003E490C9403840C94D7230C941BAA0C94F2
:1001C000AD9D0C946C180C944A170C9420170C9449
:1001D000C9810C94D1580C94CF580C94993B0C9431
:1001E000C2180C94F51D0C94FE160C94423A0C9413
:1001F0009E370C94CB480C9438160C94C01E0C946B
:10020000CB380C94758C0C9409140C9453CB0C942F
:10021000AD510C949F150C9477A10C9496180C94E6
:10022000D0650C9428330C9460140C9483750C9452
:1002300042AA0C94613B0C943D1B0C94FC560C940C
:1002400062820C9490520C94323B0C94A0230C9438
:1002500091190C9423AA0C947E1C0C94DA150C941E
:10026000081E0C9494C20C94BC170C9480370C9408
:100270005A370C94C26A0C944A3E0C9466170C943C
:10028000C7150C94C2480C9448AA0C949AA10C94DB
:1002900015AA0C94D0810C94163B0C9467840C9492
:1002A000D1800C94AC390C9469830C941E190C9475
:1002B0002D830C9402170C94E7140C94993A0C9427
:1002C000D2170C94F9300C94C5150C9439340C9455
:1002D000003B0C944FC40C94C2450C947A3A0C9495
:1002E00093800C94671C0C9431160C947EA10C9492
:1002F0007F660C9415C40C9418210C94FA160C9477
:100300006D660C946B650C9474570C94F6160C94F3
:1003100086370C9422160C94EE3B0C94FE820C94BF
:1003200066220C9435390C94A6420C94BE560C945B
:1003300064C40C94BB6F0C946C430C9434AA0C945E
:100340009F660C94A9A30C94413B0C947E350C94AD
:100350002C140C94D6150C948F570C94CB3B0C9406
:10036000FB580C9420200C94CA1C0C94AA390C94B1
:10037000E7360C94D2150C94773A0C94EE140C9446
:1003800060690C948E9D0C9433370C9457830C94B5
:10039000B3150C941A4A0C9487350C940A140C94D7
:1003A00096C30C94EA6A0C948F3A0C9463170C94DD
:1003B000181A0C940D690C9484130C946D390C94D8
:1003C00056AA0C941A3C0C94DF2F0C9463680C947E
:1003D00095800C945D170C9432240C94B9180C94ED
:1003E000E1510C94D2820C9406A30C947C660C947C
:1003F00048390C9470660C941F830C9459850C94A6
:100400003AAA0C949F390C9417160C94E1820C9420
:10041000C2800C94D43B0C94F3800C948F370C94D2
:1004200097A30C9494800C94171C0C94A8A10C9482
:10043000B3BC0C94E4140C9433140C948A660C949E
:1004400062660C948CA10C94D9810C9453370C9453
:100450008B150C94E2A30C947F210C9475560C948C
:10046000C9C30C9470830C943C370C940C160C94F8
:100470008EBB0C9470570C94C79D0C946E440C94D6
:10048000BC6A0C94E4650C9435230C948B220C9478
:100490002D560C94B7690C94B4820C9487840C94F8
:1004A0004CAA0C94FC210C940A930C942A570C949B
:1004B00026A30C944B220C94863B0C94AB650C94B5
:1004C0002C390C949C150C94B4130C9499150C9421
:1004D0007E750C94283C0C948C170C94801C0C9406
:1004E00019140C94821C0C94DCC30C94DE2F0C9415
:1004F000E5800C9408140C944B370C9440690C94D0
:10050000ED360C9427AA0C942AAA0C9416820C940B
:10051000E7B70C94D6170C9400210C9430AA0C94D5
:10052000AA220C94F1C30C94A63C0C944D180C9484
:10053000FFC30C9424180C94EA150C9482220C949A
:100540002A210C94F6190C94591F0C94713B0C94AD
:1005500081390C94332F0C94709D0C9440170C949B
:1005600052520C944F3C0C948D660C940A170C94C8
:10057000B7150C941B840C9407240C943EAA0C947D
:1005800079170C94AD1E0C94EA360C94CA150C9491
:100590000FA30C94863C0C94A1A10C94779D0C9411
:1005A0002F410C94AA150C943F3B0C94E46A0C94D4
:1005B00079690C946FC00C9449820C94F3350C94B7
:1005C0004C570C94FB3B0C9461170C94B66A0C943A
:1005D000A07C0C94F0690C949DC30C9478810C94CD
:1005E000F0360C94841C0C9434760C94E4360C9401
:1005F00006170C94513C0C94F5A20C949E130C9489
:1006000000750C94D7690C9485A10C9485840C9486
:1006100086BE0C945D3A0C9433180C9479370C9484
:10062000153C0C94AF190C94E8B50C949D1F0C94D8
:100630007C150C9455AA0C943F390C948C320C9474
:1006400097680C9481350C94EF290C9426BF0C9478
:100650006F230C940E170C949D1A0C94E3830C9446
:10066000DC200C94BF520C9451450C94F1550C9421
:1006700081800C941FAA0C94CA190C94BB150C947D
:100680005A390C9417180C94B0C30C94F7650C9459
:10069000F5360C94F9750C9416780C9450AA0C94B9
:1006A0001B574E414E494E495459494E46CDCCCC2C
:1006B0003D0AD7233C17B7D13877CC2B329595E636
:1006C000241FB14F0A000020410000C84200401C16
:1006D0004620BCBE4CCA1B0E5AAEC59D74636469ED
:1006E0006E6F70737578585B00454F46003D00494A
:1006F0004E3A00000020002300260029002C002F85
:1007000000320000010000030106010901204E6FC4
:1007100020656D69742064617461210020436F75E8
:100720006E74657220747970652E2076616C3D0060
:10073000494E3A0020436F756E746572207479706B
:10074000652E20494E434F525245435420496E7402
:10075000657272757074206E756D626572212121EB
:10076000004952513A0041637469766174652069A9
:100770006E2000416374697661746520696E2000A3
:100780002D3E00200023002D3E00200050656E64A9
:1007900065643A2023002D3E00456D69743A002DB2
:1007A0003E00456D69743A002D3E00456D69743A0E
:1007B000002D3E00456D69743A003D004C454741AF
:1007C000435920494E3A0020666F7220286D7329E4
:1007D0003A004354524C3A205363686564756C6523
:1007E00020636D642000206D730020666F7220000E
:1007F0004354524C3A2041726D6564200020446994
:100800007361726D6564004354524C3A2000207449
:10081000696D653A004354524C3A205265733A0070
:100820004354524C3A206D6F6D656E74617279203D
:100830006576656E74002054533A0020543A005493
:100840004845524D3A00436C65616E696E672061A0
:100850006C61726D20003D0050696E3A0043545245
:100860004C3A20436F6D6D616E6420626C6F636BF8
:10087000656420627920647269766572004354521F
:100880004C3A204F4E3A416C726561647920416365
:10089000746976650A004354524C3A2048414C54DE
:1008A0003A416C726561647920496E61637469765E
:1008B000650A004354524C3A20584F4E3A2044693E
:1008C0007361626C65640A004354524C3A20584F7D
:1008D0004E3A416C72656164792041637469766552
:1008E0000A004354524C3A20584F464620736B69D5
:1008F000707065642E205072657620636D643A00D6
:100900004354524C3A205475726E6564206F66668B
:100910002066726F6D3A004354524C3A2052657310
:10092000746F7265642066726F6D3A004354524C66
:100930003A2049676E6F7265642C206368616E6E41
:10094000656C20636D643D0020457865633A004323
:1009500054524C3A204163746976653A00435452CC
:100960004C3A2048414C543A416C7265616479209C
:10097000496E6163746976650A004354524C3A20AB
:10098000584F4E3A2044697361626C65640A0043B3
:1009900054524C3A20584F4E3A416C72656164791A
:1009A000204163746976650A004354524C3A2058DA
:1009B0004F464620736B69707065642E20507265D7
:1009C0007620636D643A004354524C3A2054757259
:1009D0006E6564206F66662066726F6D3A004354E0
:1009E000524C3A20526573746F7265642066726F60
:1009F0006D3A0044697361726D696E67206E6F7441
:100A000020617574686F72697A6564004354524C52
:100A10003A20636F6D6D616E64206A757374206631
:100A20006F7220004354524C3A204E6F7420656E12
:100A30006F756768206D656D6F727920666F7220C3
:100A400067726F7570206F7065726174696F6E0088
:100A5000496E76616C69642061726700496E7661E7
:100A60006C69642061726700496E76616C6964200C
:100A7000617267004354524C3A20556E6B6E6F772B
:100A80006E2073756666697800536B697070696E65
:100A900067207363686564756C65642067726F7541
:100AA000702065786563004354524C3A2063686156
:100AB0006E6E656C2066726F7A656E004354524CA0
:100AC0003A206368616E6E656C2066726F7A656E3F
:100AD00000536B697070656420686F6D6965207381
:100AE00074756666002000205375623D00204974CD
:100AF000656D3D004354524C3A2052414D3D0043F8
:100B000054524C3A204F75744F664D656D6F727933
:100B10003A2000282D292000282B2920002076614A
:100B20006C7565206973200020756E6B6E6F776E33
:100B30000A005D3D005B0020696E76616C696400AF
:100B400020004143544956453A00206F6B003A005B
:100B5000206661696C6564003A0052657472796957
:100B60006E6720434D440A004354524C2F706F6C03
:100B70006C3A204F75744F664D656D6F72793A20EF
:100B800000207365632072656D61696E696E670030
:100B90005374617475732064656666657265640A72
:100BA000002D3E005075623A20002D3E00507562C7
:100BB0003A20002D3E005075623A200000000000EF
:100BC00000636D640000736574000076616C000062
:100BD00064656C00004853560000524742000066AE
:100BE000616E00006D6F6465006374726C006875FF
:100BF000650000736174000074656D700072617748
:100C000000002D3E005075623A20002D3E005075C8
:100C1000623A200053454E445354415455533A20B0
:100C2000556E6B6E6F776E20636D64200A00000056
:100C300000000000000000004F4E00000000000017
:100C400000004F464600000000000000524553548B
:100C5000000000000000544F47474C4500000000D2
:100C600048414C54000000000000584F4E00000066
:100C700000000000584F4646000000000000494EAA
:100C80004352454153450000444543524541534575
:100C90000000454E41424C4500000000444953418C
:100CA000424C45000000554E465245455A4500000D
:100CB000465245455A45000000004155544F00003A
:100CC0000000000046414E5F4F4E4C59000048491D
:100CD00047480000000000004D454449554D0000C4
:100CE00000004C4F570000000000000048454154F0
:100CF0005F434F4F4C004845415400000000000046
:100D0000434F4F4C000000000000445259000000C7
:100D1000000000005247420000000000000048535D
:100D20005600000000000000444D58000000000084
:100D300000444D58524742570000444D58524742D4
:100D400000000050574D0000000000004D42555378
:100D500044494D0000544845524D4F000000524553
:100D60004C41590000000047524F55500000000010
:100D7000564354454D500000004D425553564300D4
:100D800000004143484149455200005350494C45F9
:100D9000440000004D4F544F5200000000504944A1
:100DA0000000000000004D425553000000000055B7
:100DB000415254425244470052454C415950574DBC
:100DC00000444D5852474257570056454E54530021
:100DD000000000454C455641544F5200434F554E7C
:100DE000544552000048554D0000000000004D459C
:100DF0005243555259000020002D3E00436F6E763D
:100E0000657274696E6720002D3E0057726F6E67C1
:100E10002041737369676E6D656E7420005247429E
:100E2000783A20004853562064697361626C6564A7
:100E30000020764C6576656C3A0020436F6E7656DE
:100E40003A0020436F6E76533A0020486F743A00A0
:100E5000436F6C643A0020436F6E7665727465640C
:100E600020563A00436F6E76657274656420533A7B
:100E7000002D3E0057726F6E672041737369676E75
:100E80006D656E7420002D3E0057726F6E672041B5
:100E9000737369676E6D656E7420002053756666A6
:100EA0003A002041543A0053746F7070696E6720A5
:100EB000496E7075747300206973200044656C6519
:100EC00074696E6720636F6E662E2052414D2077E5
:100ED00061733A0053746F70706564006E6F74686C
:100EE000696E6720746F2073746F700053746F7035
:100EF00070696E67206368616E6E656C73202E2E5C
:100F00002E0043616E206E6F7420636C65616E20ED
:100F10002D206C6F636B656400436F6E666967209C
:100F20006368616E676564206C6F63616C6C792CBB
:100F300020706F7274616C2064697361626C6564A7
:100F4000002F636F6E6669672E6A736F6E0072653D
:100F5000626F6F742000436D643A20002F636F6DE1
:100F60006D616E642F002F72616D2F002F697465A3
:100F70006D2F002F6974656D2F0022687474703AAC
:100F80002F2F6C617A79686F6D652E72752F70776F
:100F90006122004C6F636174696F6E3A20687474EB
:100FA000703A2F2F003F6D61633D002669703D0050
:100FB00026706F72743D00266E616D653D002F00D6
:100FC00020004D5154543A20436F6D706C65746528
:100FD0002E2052656D6F766520746F7069632000F6
:100FE00024636F6D6D616E64004D5154543A20431B
:100FF0006C65616E55702072657461696E65642000
:10100000746F7069632000220022004F75744F6670
:101010004D656D6F727921005D20003A5B004D5186
:1010200054543A005D00456D7074793A205B000AB3
:10103000003A004D41433A00554450205379736CB7
:101040006F6720696E697469616C697A65642E0ADC
:10105000005379736C6F6720706172616D733A0031
:101060004D5154543A20736574206669727374202C
:1010700062726F6B65720043757272656E74204C9C
:10108000414E20636F6E6669672869702C646E73C9
:101090002C67772C7375626E6574293A000A557354
:1010A0006520746865736520636F6D6D616E647330
:1010B0003A202768656C7027202D2074686973209A
:1010C000746578740A276D61632064653A61643AD7
:1010D00062653A65663A66653A3030272073657412
:1010E00020616E642073746F7265204D41432D61E1
:1010F00064647265737320696E20454550524F4D8C
:101100000A276970205B69705B2C646E735B2C67C7
:10111000775B2C7375626E65745D5D5D5D27202D58
:1011200020736574207374617469632049500A27C1
:101130007361766527202D20736176652063757253
:1011400072656E7420636F6E66696720696E204EEB
:101150005652414D3B204F4E7C4F4646202D206538
:101160006E61626C652F64697361626C6520617584
:10117000746F736176650A2767657427205B636FF8
:101180006E66696720616464725D27202D20676543
:101190007420636F6E6669672066726F6D2070726F
:1011A000652D636F6E666967757265642055524C74
:1011B00020616E642073746F726520616464722CA8
:1011C000204F4E7C4F4646202D20656E61626C6537
:1011D0002F64697361626C6520646F776E6C6F61F8
:1011E00064206F6E20737461727475700A276C6F5F
:1011F000616427202D206C6F616420636F6E6669C7
:10120000672066726F6D204E5652414D0A277077E7
:101210006427202D20646566696E6520616E6420F8
:1012200073746F7265204D515454207061737377DD
:101230006F72640A276F746170776427202D2064B1
:101240006566696E6520616E642073746F726520D7
:1012500048545450204150492070617373776F7225
:10126000640A276C6F67205B73657269616C5F6CE1
:101270006F676C6576656C5D205B7564705F6C6F25
:10128000676C6576656C5D27202D20646566696EE8
:1012900065206C6F67206C6576656C2028302E2E7B
:1012A00037290A276B696C6C27202D2074657374AD
:1012B000207761746368646F670A27636C65617285
:1012C00027202D20636C65617220454550524F4D9B
:1012D0000A2773656172636827202D207365617228
:1012E000636820312D77697265206465760A2772FC
:1012F00065626F6F7427202D207265626F6F742096
:10130000636F6E74726F6C6C657200536F667420DD
:101310007265626F6F74696E672E2E2E00206E6587
:10132000770020697320003157543A003157543AFE
:1013300020536561726368696E6720646576005248
:10134000414D3D000A5379736C6F6720000A312DBF
:101350007769726520000A6D71747420000A696EE5
:101360007075747320000A6974656D7320000A43F8
:101370006F6E666967757265643A002F00496E3A50
:101380002000496E697469616C697A696E672049E9
:101390006E70757473003157543A207365747570AC
:1013A000207265736F6C7574696F6E2000315754CD
:1013B0003A204453323438322D313030206E6F743D
:1013C0002070726573656E74003157543A2044532F
:1013D000323438322D313030204932432072657337
:1013E000746F726564003157543A204275732072ED
:1013F00065736574206572726F72003157543A20BC
:1014000042757320526573657420646F6E65003198
:1014100057543A204453323438322D313030207012
:10142000726573656E742C20726573657400457205
:10143000726F7220312D7720696E697400315754B4
:101440003A204453323438325F3130305F493243CE
:101450005F544F5F31575F42524944474520696EA0
:101460006974003B003D0050696E3A003B003D4C02
:101470004F5700546865726D6F3A004F6E65207764
:101480006972652052656164790A0042726F6B650A
:10149000727320636F6E666967757265643A0041A6
:1014A00070706C79696E6720636F6E666967004C57
:1014B0006F6164656420455441473A004E6F207364
:1014C000746F72656420636F6E666967004C6F614C
:1014D0006465642066726F6D20454550524F4D0023
:1014E0006C6F6164206661696C6564004A534F4E9D
:1014F000206465746563746564004C6F6164696E33
:101500006720436F6E6669672066726F6D20454580
:1015100050524F4D00436F6E666967206175746F5E
:10152000736176653A000A5379736C6F672064655E
:10153000627567206C6576656C3A00536572696107
:101540006C206465627567206C6576656C3A005343
:10155000617665640A005365742064796E616D6913
:10156000632049500A004F54412050617373776FD4
:10157000726420757064617465640A004E6F20495E
:101580005020616472657373002053617665640056
:101590004C6F6164696E67204854545020636F6ECD
:1015A000666967206F6E20737461727475703A009B
:1015B000000000000000000000004F4E000000008E
:1015C000000000004F4646000000000000005245A9
:1015D0005354000000000000544F47474C450000A2
:1015E000000048414C54000000000000584F4E00DD
:1015F000000000000000584F4646000000000000B8
:10160000494E4352454153450000444543524541EC
:1016100053450000454E41424C45000000004449FE
:101620005341424C45000000554E465245455A45EF
:101630000000465245455A45000000004155544FB0
:1016400000000000000046414E5F4F4E4C59000024
:10165000484947480000000000004D454449554DA9
:10166000000000004C4F57000000000000004845FB
:1016700041545F434F4F4C00484541540000000027
:101680000000434F4F4C000000000000445259003E
:10169000000000000000524742000000000000006F
:1016A00048535600000000000000636F756C642012
:1016B0006E6F742070617273653A200055706461BA
:1016C0007465640A00454550524F4D20636C656156
:1016D0007265640A004D5154542050617373776FE2
:1016E000726420757064617465640A002B002D00BB
:1016F000455461673A200047657420455441473A94
:101700002000485454502F312E310025733A2025A3
:10171000730D0A0020485454502F312E310D0A48C1
:101720006F73743A2025730D0A4163636570743AD0
:10173000202A2F2A0D0A436F6E6E656374696F6EDF
:101740003A20636C6F73650D0A0025730020000D4D
:101750000A00474554006661696C656420746F2017
:10176000636F6E6E6563740A004552524F523A20A1
:101770005365727665722072657475726E65642049
:1017800000436F6E666967206E6F74206368616ED8
:101790006765640A00446F6E652E0A00436F6E66CB
:1017A00069672070617273696E67206661696C6534
:1017B000640A004765742061626F72746564006733
:1017C0006F7420436F6E6669670A006874747020D6
:1017D000726574636F6465200066726565200043FE
:1017E0006F6E666967205552493A20687474703A82
:1017F0002F2F002044656661756C7420636F6E66E0
:1018000069672073657276657220757365643A2026
:10181000006C617A79686F6D652E7275000A282DEB
:10182000294352595054000A282D2950554C5345EC
:10183000206F6E2050494E3132000A282D29434135
:101840004E000A282D294D455243555259000A2869
:101850002D294D554C544956454E54000A282B29E4
:1018600050574D5F52454C4159000A282D294D448F
:101870004E53000A282D295541525442524944479B
:1018800045000A282B295359534C4F47000A282D4D
:1018900029504944000A282D294D43503233303114
:1018A00037000A282D294152544E4554000A282B4E
:1018B000294F5441000A282D29535049204C4544B2
:1018C000000A282D294D4F544F5220435452000AEC
:1018D000282D294143204841494552000A282D29F5
:1018E0004343533831312026204844433130383087
:1018F000000A282B29524553544152545F4C414E03
:101900005F4F4E5F4D5154545F4552524F525300FA
:101910000A282D294841524452455345542C2075DC
:1019200073696E6720736F6674000A282B29434F12
:10193000554E544552000A282D29444854000A287F
:101940002B294453323438322D313030000A282BC1
:10195000294F57495245000A282D2949504D4F44D7
:10196000425553000A282D294D4F44425553000A31
:10197000282D29444D58000A282B2957697A6E656D
:101980007435783030000A282B294672656552611B
:101990006D207072696E74696E67000A282B295772
:1019A00041544348444F47006C617A79686F6D65D4
:1019B0002E7275000A436F6E6669672073657276D2
:1019C00065723A003230313130334C0020432B2BDA
:1019D0002076657273696F6E3A00303864656436DC
:1019E000325F323032362D30312D3039000A4C61C1
:1019F0007A79686F6D652E7275204C6967687448D6
:101A0000756220636F6E74726F6C6C65722000205B
:101A10004F464600204F4E0020425950415353003C
:101A2000536176656420746F20454550524F4D00D8
:101A3000536176696E6720636F6E66696720746FA5
:101A400020454550524F4D2E2E00556E6B6E6F77D0
:101A50006E207375666669782000556E6B6E6F77C1
:101A60006E20636D642000436F756E7465723A205A
:101A70000020696E69740070696E230072656C6184
:101A8000794374723A20002073746F700052656C51
:101A900061792D4F757420230072656C61794374F0
:101AA000723A200069646C65006F66660068656163
:101AB00074696E670066616E00647279696E6700B2
:101AC000636F6F6C696E6700616374696F6E00208D
:101AD000697320004F7574200072656C61794374DE
:101AE000723A2000556E6B6E6F776E207375666666
:101AF0006978200072656C61794374723A200055F0
:101B00006E6B6E6F776E20636D64200072656C6122
:101B1000794374723A2000616374696F6E00726574
:101B20006C61794374723A20005B305D3A2000208A
:101B30002D202D202D20EFBBBF003E003E31202D5B
:101B400020005B305D3A2000202D202D202D20EF3D
:101B5000BBBF003E003E31202D20005379736C6FD7
:101B60006720726573756D6564005379736C6F6778
:101B700020726573756D6564005379736C6F6720AF
:101B800073757370656E6465640000000000006327
:101B90006D640000736574000076616C000064651C
:101BA0006C00004853560000524742000066616EC8
:101BB00000006D6F6465006374726C006875650089
:101BC00000736174000074656D70007261770000CD
:101BD00020002E00696E00735F6F7574006D796868
:101BE0006F6D65004354524C2F657865633A204F02
:101BF00075744F664D656D6F72793A2000202D3EE9
:101C000020004D5154543A2000202D3E2000456DB7
:101C100069743A203C00202D3E20004974656D43D4
:101C20006D643A2000202D3E20004974656D3A20F5
:101C3000003157543A2042757320726573657420E1
:101C40006572726F72003157543A20427573205298
:101C50006573657420646F6E65003157543A204493
:101C600053323438322070726573656E742C207272
:101C700065736574004932432052657365740000D2
:101C80005EBCE2613FDD83C29C7E20A3FD1F419DBF
:101C9000C3217FFCA2401E5F01E3BD3E6082DC23C6
:101CA0007D9FC1421CFEA0E1BF5D0380DE3C62BEA1
:101CB000E0025CDF81633D7C22C09E1D43A1FF46A4
:101CC00018FAA427799BC584DA3866E5BB5907DB87
:101CD000856739BAE406581947A5FB7826C49A6582
:101CE0003BD987045AB8E6A7F91B45C6987A24F869
:101CF000A6441A99C7257B3A6486D85B05E7B98C58
:101D0000D2306EEDB3510F4E10F2AC2F7193CD1156
:101D10004FADF3702ECC92D38D6F31B2EC0E50AF2D
:101D2000F1134DCE90722C6D33D18F0C52B0EE3238
:101D30006C8ED0530DEFB1F0AE4C1291CF2D73CA13
:101D4000947628ABF517490856B4EA6937D58B570E
:101D500009EBB536688AD495CB2977F4AA4816E9F9
:101D6000B7550B88D6346A2B7597C94A14F6A874F0
:101D70002AC896154BA9F7B6E80A54D7896B353EA1
:101D80003E2000496E76616C696420636F6D6D6101
:101D90006E64003E3E3E004E6F204D414320636F17
:101DA0006E666967757265643A207365742066694A
:101DB000726D776172652773204D41430A00454576
:101DC00050524F4D207369676E6174757265206F54
:101DD0006B00496E697469616C697A696E67204548
:101DE0004550524F4D2E00476F742049502061647A
:101DF00064726573733A00276970205B69705B2CAD
:101E0000646E735B2C67775B2C7375626E65745DB3
:101E10005D5D5D27202D2073657420737461746986
:101E2000632049500A004661696C656420746F2024
:101E3000636F6E6669677572652045746865726E5A
:101E40006574207573696E6720444843502E20598D
:101E50006F752063616E20736574206970206D61F9
:101E60006E75616C6C792100204D41534B3A002016
:101E700047573A0020444E533A004C6F6164656402
:101E80002066726F6D20666C6173682049503A005D
:101E90000A7573657320444843500A005374617295
:101EA00074696E67206C616E004142434445464749
:101EB00048494A4B4C4D4E4F50515253545556572A
:101EC00058595A6162636465666768696A6B6C6DCC
:101ED0006E6F707172737475767778797A3031328B
:101EE000333435363738392B2F3D004261736963FF
:101EF00020003A004F544120696E697469616C6931
:101F00007A65640A0044454641554C54207061731B
:101F100073776F726420666F72204F544120415076
:101F2000492E20557365206F746170776420636F4C
:101F30006D6D616E6420746F2073657400706173E1
:101F400073776F7264004D5154543A2074727969FA
:101F5000796E67206E656E78742062726F6B657241
:101F6000004D5154543A20546F6F206D616E7920AA
:101F7000636F6E6E656374696F6E206572726F72E7
:101F8000732E2052657374617274204C414E002090
:101F900074727920616761696E20696E20352073E3
:101FA00065636F6E6473004D5154543A20666169E5
:101FB0006C65642C2072633D004D5154543A2041AD
:101FC00077616974696E6720666F722072657461EB
:101FD000696E656420746F7069637300636F6E6E01
:101FE00065637465642061732000202E2E2E00200E
:101FF000757365723A003A000A4D5154543A2041C3
:102000007474656D7074696E6720636F6E6E65635E
:1020100074696F6E20746F2000646973636F6E6EF5
:102020006563746564005573696E67204D5154543F
:102030002070617373776F72642066726F6D2063B6
:102040006F6E66696700446576696365204E616DF1
:10205000653A004D5154543A204174206C656173C7
:102060007420646576696365206E616D6520616EBC
:10207000642062726F6B6572204950206D757374B5
:1020800020626520636F6E666967757265640075AE
:102090007074696D652C6672656568656170003085
:1020A0003864656436325F323032362D30312D304F
:1020B00039004C696768744875622000246E616D50
:1020C0006500526562696E6420737563636573733E
:1020D0002E20495020616464726573733A00457222
:1020E000726F723A20726562696E64206661696C13
:1020F0000052656E657765642073756363657373FD
:102100002E20495020616464726573733A004572F1
:10211000726F723A2072656E6577656420666169D8
:102120006C000A4E6F206C696E6B00436F6E7469B1
:102130006E756520776974682070726576696F7551
:10214000736C79206C6F6164656420636F6E66697F
:10215000670033307320454550524F4D206973203E
:102160006E6F742072656C6F616465642E205265B9
:10217000626F6F74004D5154543A2041636365702F
:1021800074696E6720636F6D6D616E64732E2E2EA1
:102190000A004E6F204D51545420636F6E6669677C
:1021A00075726564004C6F6164696E6720636F6E61
:1021B0006669672066726F6D20706F7274616C2043
:1021C00064697361626C65642E2075736520676550
:1021D00074204F4E20746F20656E61626C65004301
:1021E0006F6E6669672069732076616C696400436D
:1021F0006F6E74696E75652077697468207072659A
:1022000076696F75736C79206C6F616465642063A7
:102210006F6E666967005365747570204F54410096
:102220002072656164206572726F7220666F722021
:10223000003E2000203C003157543A003157543AB8
:10224000206E6F7420696E6974003157543A2042D1
:102250005553592074696D656F7574003157543A40
:10226000204453323438325F4552524F525F434F0D
:102270004E464947003157543A20312D77697265EF
:102280002073686F727465640072656164790024FC
:10229000737461746500757074696D65006672654C
:1022A00065686561700024737461747300204578FB
:1022B00070697265640A00202D746172676574200C
:1022C0007A6F6E652D0020416C61726D20457870CB
:1022D000697265640A0020636D643A002043757278
:1022E0003A00205365743A002054696D65723A00D3
:1022F000204C6F636B733A0052414D3D000000214A
:1023000000240027002A002D0030003300010100C6
:1023100000040107010A0100002200250028002B0B
:10232000002E003100340002010000050108010BFD
:102330000105050505070508080808020202020A4A
:102340000A08080404040401010101010101010358
:1023500003030303030303040707070C0C0C0C0C13
:102360000C0C0C0202020206060606060606060B06
:102370000B0B0B0B0B0B0B0102102020080810207D
:102380004010204080020102010804020101020401
:1023900008102040808040201008040201800402C0
:1023A0000180402010080402010804020101020417
:1023B0000810204080010204081020408000000A1C
:1023C0000B02090C0D0E08070304010000000000B9
:1023D00000000000000000000000000000000000FD
:1023E00000000000000000000012111000000000BA
:1023F00000000000000000000000000000000000DD
:102400000000006F637465742F73747265616D00F2
:102410006170706C69636174696F6E2F6A736F6E3F
:1024200000746578742F706C61696E00436F6E7410
:10243000656E742D547970653A2000436F6E6E6539
:102440006374696F6E3A20636C6F736500416363F8
:102450006573732D436F6E74726F6C2D416C6C6F6E
:10246000772D4F726967696E3A202A00556E6B6E40
:102470006F776E004E6F74204D6F64696669656496
:10248000004F4B004D6F766564207065726D616E14
:10249000656E746C7900496E7465726E616C205360
:1024A0006572766572204572726F72005061796C48
:1024B0006F616420546F6F204C61726765004E6FCE
:1024C0007420666F756E64005757572D4175746898
:1024D000656E7469636174653A2042617369632053
:1024E0007265616C6D3D2241636365737320726533
:1024F00073747269637465642200556E61757468E3
:102500006F72697A6564005061796C6F61642073E1
:10251000697A652077726F6E670042616420726528
:10252000717565737400485454502F312E3120005A
:102530002000000000000000000000004F4E0000DE
:102540000000000000004F464600000000000000B0
:1025500052455354000000000000544F47474C457B
:102560000000000048414C54000000000000584F9B
:102570004E00000000000000584F464600000000DA
:102580000000494E435245415345000044454352E3
:10259000454153450000454E41424C450000000076
:1025A00044495341424C45000000554E4652454572
:1025B0005A450000465245455A4500000000415525
:1025C000544F00000000000046414E5F4F4E4C59F2
:1025D0000000484947480000000000004D454449BC
:1025E000554D000000004C4F570000000000000057
:1025F000484541545F434F4F4C004845415400000B
:1026000000000000434F4F4C000000000000445207
:102610005900000000000000524742000000000086
:1026200000004853560000000000000057726F6E13
:1026300067207061796C6164004D5154543A2043B5
:1026400054524C2F7478743A204F75744F664D6510
:102650006D6F72793A2000202D3E2041543A00439C
:1026600068616E20747970653A004E6F2073746FE4
:102670007265642076616C756573202D20646566D3
:1026800061756C743A20005361766564204554414D
:10269000473A0053657420455441473A200053CBD4
:1026A000E8B511241FBECFEFD1E2DEBFCDBF00E001
:1026B0000CBF16E0A0E0B2E0ECEBF0EC01E00BBFE9
:1026C00002C007900D92A639B107D9F72CE0A6E910
:1026D000B6E001C01D92A932B207E1F713E1C0E5EF
:1026E000D3E100E006C021970109802FFE010E947E
:1026F0002ED8CF34D10780E00807A9F70E94FAB599
:102700000C944CE00C940000CF93DF931F92CDB754
:10271000DEB76983DC01ED91FC910280F381E02D4D
:1027200041E050E0BE016F5F7F4F19950F90DF9140
:10273000CF910895FC01818D928D0895CF93DF9301
:102740001F92CDB7DEB76983DC01ED91FC91028069
:10275000F381E02D41E050E0BE016F5F7F4F19959E
:102760000F90DF91CF910895FC019485FB01848542
:10277000981303C081E0983008F080E00895CF936B
:10278000DF931F92CDB7DEB76983DC01ED91FC9139
:102790000280F381E02D41E050E0BE016F5F7F4F8A
:1027A00019950F90DF91CF910895FC01818191E0FF
:1027B000909340098093610910926709109266090D
:1027C000089520915E07260F3327331F21323105EC
:1027D000ECF420913A09FC0190E080E0243069F0AB
:1027E00082E00895A0915E072191AC01425C584FB0
:1027F000A40FB52FB11D2C930196861798F38091E5
:102800005E07680F60935E0780E0089581E0089599
:1028100008950895E091690980916809E81730F4F6
:10282000F0E0EF57F84F808190E008958FEF9FEF31
:10283000089590916909809168092FEF3FEF9817EB
:1028400048F4E92FF0E0EF57F84F208130E09F5F28
:1028500090936909C9010895809168099091690967
:10286000891B990B0895CF92DF92EF92FF920F93FD
:102870001F93CF93DF937C01CB018A012091400904
:10288000222389F0EB016B01C40ED51ECC15DD05AA
:1028900069F06991D701ED91FC910190F081E02DF3
:1028A000C7011995F3CF642F0E94E113C801DF918E
:1028B000CF911F910F91FF90EF90DF90CF900895EF
:1028C000CF93DF931F92CDB7DEB769832091400984
:1028D0002223F9F020916609203258F021E030E0FF
:1028E000FC013383228390E080E00F90DF91CF9151
:1028F000089580916709E82FF0E0EF5BF64F99812A
:1029000090838F5F809367098093660981E090E0F0
:10291000ECCF61E0CE0101960E94E113F7CF90E089
:10292000FC01EF5CFC4DE491F0E0EE0FFF1FE95E6F
:10293000FC4DA591B4912C9189589C4DFC0184913A
:10294000822391E009F490E0892F0895FC01DC01D5
:102950008D918111FDCF30E020E050E040E08AE031
:102960009191992301F1443051055CF59E3271F447
:102970002F3F310509F02CF5DB01A40FB51F12968E
:102980002C934F5F5F4F30E020E0EACF829FD00171
:10299000839FB00D1124292F990F330B2053310938
:1029A0002A0F3B1FDDCF2F3F310509F054F444308F
:1029B00051053CF4640F751FFB01228381E090E018
:1029C000089590E080E0089590E080E00895DC01B3
:1029D000ED91FC910284F385E02D1994DF92EF9242
:1029E000FF920F931F93CF93DF93EC010C891D8906
:1029F0000115110559F01D8A1C8AC801DF91CF917C
:102A00001F910F91FF90EF90DF900895EC85FD8569
:102A10008E859F85DF01A80FB91F2C91243209F004
:102A200055C011962C912B3709F050C00296E80F33
:102A3000F91FF12CE12CDF01D190DD2009F446C013
:102A40008DE7D816E9F08FEFE81AF80AF4CF198A63
:102A5000188A2C853D852115310579F08E859F8555
:102A6000280F391FF9012081222321F001969F8729
:102A70008E873EC01D861C86C0CF0FEF1FEFBDCFD7
:102A8000E114F10419F11C928E859F8502966C85E4
:102A90007D85680F791FE881F9810684F785E02D2F
:102AA000CE011995998B888B1B8A1A8AEC85FD8536
:102AB0008E859F85E80FF91FEE0DFF1DD2828E8552
:102AC0009F850396E80EF91EFF86EE8628893989D0
:102AD0002115310509F4BDCF8A899B89280F391F3B
:102AE000F9012081222309F4B2CF01969B8B8A8BB6
:102AF000022F220F110B81CFDC011C96ED91FC916E
:102B00001D971E968D919C91E80FF91F8081082ECC
:102B1000000C990B0895DC0115968D919C910097FE
:102B200039F0DC01ED91FC910680F781E02D1994DC
:102B3000089583E090E0089584E190E00895DC0139
:102B4000ED91FC910484F585E02D60E0199581E01C
:102B500090E008958FE090E09093B5078093B407DC
:102B600088EC90E00895FC01848195810895FC0132
:102B7000768765870895DC01ED91FC9102A0F3A1B1
:102B8000E02D199591E089270895862F089581E019
:102B90008627089521E0FC018485883008F020E034
:102BA000822F0895FC01848595850895FC01848910
:102BB000958908952CE234E0FC0131832083FB01E8
:102BC0004089518962897389FC01428353836483FC
:102BD00075830895DC01ED91FC91048CF58DE02D59
:102BE0001994DC011196EC911197EF70E150EB30E4
:102BF00008F03EC0F0E08827EF5FF94E8F4F0C944D
:102C00002ED81716171638160C160C163116221653
:102C1000221622160C160C1614962D913D914D91EC
:102C20005C911797A4E6B0E00E94E4D7089514964B
:102C30006C9184E6689FB0011124072E000C880B6C
:102C4000990B089520E030E048EC52E414966D9121
:102C50007D918D919C9117970E94BFD60E942BD990
:102C6000089514966D917D918D919C91179708957B
:102C700060E070E0CB010895FC01A7812A2F2E7F30
:102C8000C9F081818F7081508330A0F4A695A15046
:102C9000BB0B2BE531E00E9445D824E630E040E054
:102CA00050E00E94C5D7DA01C90187569F4FAF4F48
:102CB000BF4F08958FEF9FEF0895FC01A681B78164
:102CC000109721F118969C9118979F708EEF890F9D
:102CD000823010F091111AC019964D935D936D9347
:102CE0007C931C97A681B78118969C911897907F2A
:102CF000926018969C930680F781E02D8085982F2E
:102D0000907F903619F48F70806A80870895FC0157
:102D1000238130E090E080E0FC01EE0FFF1FE853DC
:102D2000F94FA081B181A217B30761F4880F991FF1
:102D3000880F991FFC01EC54F94F40835183628343
:102D400073830895A081B181AB2B19F42081318167
:102D5000EDCF019685309105F9F60895FC012381A8
:102D600030E090E080E0FC01EE0FFF1FE853F94FE8
:102D7000408151814217530761F4880F991F880FD2
:102D8000991FFC01EC54F94F60817181828193811C
:102D9000089540815181452B89F431832083880F28
:102DA000991F880F991FFC01EC54F94F1082118272
:102DB0001282138260E070E0CB01089501968530A5
:102DC000910589F6F7CF880F991F880F991FFC018D
:102DD000E456F94F80819181A281B3810196A11DB2
:102DE000B11D80839183A283B383089585E090E031
:102DF0000C94E31684E090E00C94E31683E090E0FA
:102E00000C94E31682E090E00C94E31681E090E0ED
:102E10000C94E31690E080E00C94E316CF93DF93DC
:102E2000EC01E881F9810484F585E02D1995298963
:102E30003A892F5F3F4F3A8B298BDF91CF910895CD
:102E4000CF93DF93EC018E8581110DC081E090E07E
:102E500049895A892C853D854217530708F080E03F
:102E6000DF91CF910895E881F9810484F585E02D03
:102E7000CE0119958F3F910549F780E090E0F0CFA2
:102E8000FC01848595856817790708F4CB01928B3E
:102E9000818B0895CF93DF93FC012685222351F087
:102EA000EC010190F081E02D0190F081E02D6FEFB9
:102EB00019951E86DF91CF910895FC018785908931
:102EC000089581E0089590E080E00895DC01129675
:102ED000ED91FC91309761F00280F381E02D309705
:102EE00039F0862F8295807F60856F70682B6087B0
:102EF0000895DC011296ED91FC91309751F002801B
:102F0000F381E02D309729F0808582958F7090E0D5
:102F1000089590E080E00895CF93DF93CDB7DEB7BA
:102F200060970FB6F894DEBF0FBECDBF19821A822C
:102F30001B821C821D821E821F8218868A81807FCE
:102F400081608A836FEF3E819F81888529817A81A4
:102F50005B814C814C873E87888B372F452F5C8562
:102F60007E85892F988960960FB6F894DEBF0FBED4
:102F7000CDBFDF91CF9108950F931F93CF93DF9330
:102F800000D000D01F921F92CDB7DEB781E0289607
:102F90000FB6F894DEBF0FBECDBFDF91CF911F916A
:102FA0000F910895FC01738362830895CF92DF929D
:102FB000EF92FF920F931F93CF93DF9300D000D037
:102FC000CDB7DEB78C016B017A01FC01808D8830B2
:102FD00010F40E94BE988CE294E09A838983F601F3
:102FE00082819381A481B5818B839C83AD83BE83D1
:102FF000B701CE0101960E9411A9F801808F883097
:10300000A0F4F586E486128E118E81E026960FB626
:10301000F894DEBF0FBECDBFDF91CF911F910F910E
:10302000FF90EF90DF90CF90089580E0EFCFCF93A7
:10303000DF93EC01888D883020F40E94BE9888E0F0
:10304000888FDF91CF910895FC01808D883040F406
:10305000218D328D232B21F00E94909790E00895CE
:103060008FEF9FEF0895CF93DF93FC0124852830E5
:1030700028F08FEF9FEFDF91CF910895EC01019041
:10308000F081E02D0084F185E02D1995892B89F3DD
:103090008C850E94909790E0EECFCF93DF93FC0158
:1030A000218D328D2115310529F48FEF9FEFDF91AE
:1030B000CF910895EC01808D4217530708F0A901C4
:1030C0000E94DF971816190684F7298D3A8D281B60
:1030D000390B3A8F298FEBCF0F931F93CF93DF9349
:1030E0001F92CDB7DEB7FC01218D328D232B41F429
:1030F0008FEF9FEF0F90DF91CF911F910F91089568
:103100008C0141E050E0BE016F5F7F4FFC01808D7C
:103110000E94DF97181619065CF7F801818D928DD1
:103120000197928F818F898190E0E4CFCF93DF93D5
:103130001F92CDB7DEB741E050E0BE016F5F7F4F19
:10314000FC0184850E94DF971816190634F48981E2
:1031500090E00F90DF91CF9108958FEF9FEFF9CF1F
:10316000FC018485883010F40C94DF9790E080E0B7
:103170000895FC018485883010F40C94B89790E091
:1031800080E008950F931F93CF93DF9300D000D07A
:103190001F921F92CDB7DEB78C01D80159964D9181
:1031A0005C915A974115510551F0ED91FC91048CB9
:1031B000F58DE02D70E060E0C8011995EECFF801C3
:1031C000808D0E94B897892BB1F148E050E0BE0194
:1031D0006F5F7F4FD80158968C910E94DF97181629
:1031E0001906F4F4D801509684E0FE01319601905E
:1031F0000D928A95E1F78D8190E0982F88272E8196
:10320000820F911DF801958B848B8F81282F30E0E0
:10321000322F22278885820F932F911D928F818FC5
:1032200028960FB6F894DEBF0FBECDBFDF91CF91C9
:103230001F910F91089590E080E0F2CFCF92DF923E
:10324000EF92FF920F931F93CF93DF93CDB7DEB72B
:10325000AF970FB6F894DEBF0FBECDBF7C016A01F9
:103260000CE214E01A8309831C861B8688EE93E027
:10327000A0E0B0E08D879E87AF87B88B82E094E0B6
:103280009A878987188F0F8B198E1A8E1B8E1C8E2A
:1032900088E089A31BA70AA71CA61DA61EA61FA619
:1032A0008091A3099091A409A091A509B091A609C4
:1032B0008EA39FA3A8A7B9A78B839C83AD83BE834E
:1032C00018861F82AE01465D5F4FCE0101960E94B7
:1032D00007B181309105B1F4D701ED91FC910488DB
:1032E000F589E02D1DA30CA38CA59DA5AEA5BFA5BA
:1032F0008EA39FA3A8A7B9A7A601BE016C5D7F4FAF
:10330000C7011995AF960FB6F894DEBF0FBECDBFBB
:10331000DF91CF911F910F91FF90EF90DF90CF90B1
:1033200008950F931F93CF93DF93EC018B01888D4A
:10333000883010F40E94BE98B80182E00E9407997C
:10334000888F883050F41D870C871A8E198E81E083
:10335000DF91CF911F910F91089580E0F9CF0F93E6
:103360001F93CF93DF938C01EA01FC0184858830A1
:1033700048F40E942E97892B39F481E090E0F801FF
:1033800093838283D0E0C0E0CE01DF91CF911F9183
:103390000F910895EF92FF920F931F93CF93DF93B6
:1033A0007C0180911309D4E0833309F0D8E003E075
:1033B00019E0C0E0F801219131918F01F70184817A
:1033C00095812817390729F0CF5FDC13F3CF80E010
:1033D00006C08C2F0E94CC988431B1F781E0DF9138
:1033E000CF911F910F91FF90EF900895CF93DF93AE
:1033F000EC018C858830D0F40E94CC98843189F01F
:10340000882379F0883169F021E08C3159F4E88122
:10341000F9810084F185E02DCE01199521E0892BF9
:1034200009F420E0822FDF91CF91089580E0FBCF57
:103430006F927F928F929F92AF92BF92CF92DF92C4
:10344000EF92FF920F931F93CF93DF938C015B0159
:103450007A0180911309882309F46CC024E0622E5C
:10346000833311F098E0692E83E0C82E89E0D82ECE
:103470004601712CC0E0D4012D913D914D01F80120
:10348000848195812817390799F48C2F0E94CC9854
:10349000D82F873119F08C3109F040C08C2F0E9451
:1034A000B897892B29F4DC3119F48C2F0E94B0983D
:1034B000CF5F6C12E0CF711008C0D801ED91FC9184
:1034C0000084F185E02DC8011995D0E0F601219125
:1034D00031916F01D80114968D919C91281739076D
:1034E00051F48D2F0E94CC98873129F4A701B501A2
:1034F0008D2F0E942E97DF5FDC13E8CFC701DF918D
:10350000CF911F910F91FF90EF90DF90CF90BF90E0
:10351000AF909F908F907F906F900895843139F095
:103520008111C6CFF401329711821082C1CF772466
:103530007394BECFF12CE12CE1CFCF92DF92EF92CA
:10354000FF920F931F93CF93DF93CDB7DEB7AF9763
:103550000FB6F894DEBF0FBECDBF8C016B017A01B0
:103560008CE294E09A8389831B821C821D821E82D6
:103570001C861B8648EE53E060E070E04D875E8756
:103580006F87788B22E034E03A872987988F8F8B7A
:10359000198E1A8E1B8E1C8E28E029A39BA78AA742
:1035A0001CA61DA61EA61FA6D8011C968C918830AD
:1035B00060F40E94CC98882321F0F80184850E9451
:1035C000B09888E0D8011C968C938091A3099091C3
:1035D000A409A091A509B091A6098EA39FA3A8A7AD
:1035E000B9A78B839C83AD83BE8318861F82AE01EF
:1035F000465D5F4FB601CE0101960E9407B100976C
:10360000C1F0D801ED91FC910684F785E02D8CE2A4
:1036100094E09DA38CA38CA59DA5AEA5BFA58EA36C
:103620009FA3A8A7B9A7A701BE016C5D7F4FC801E2
:103630001995AF960FB6F894DEBF0FBECDBFDF91E0
:10364000CF911F910F91FF90EF90DF90CF90089551
:10365000CF93DF93EC018C85883060F40E94CC9886
:10366000873111F08C3131F48C850E9411978115CE
:10367000984088F3DF91CF910895FC0184858830CC
:1036800010F40C94119790E080E00895CF93C62F2A
:103690000E94D51361EE87EA99E00E9460146C2FB6
:1036A00087EA99E00E946014CF910C94FAAB0E94D3
:1036B000D51381E00E940AAB91E0811190E0892F3F
:1036C0000895ECEBF0E080818A7B808360E084E108
:1036D0000E945EAA60E085E10C945EAA65E0FC01B0
:1036E000828193810E94439D009749F0FC0180856F
:1036F000982F907F21F082958F7090E0089590E050
:1037000080E00895CF92DF92EF92FF926A017B01F1
:1037100063E0FC01828193810E94439DFC01892B1F
:10372000A9F080858D7091F4C094D094E094F094C9
:10373000CC24CA9481859285A385B4858C219D2152
:10374000AE21BF2181879287A387B487FF90EF9036
:10375000DF90CF900895CF92DF92EF92FF926A01AF
:103760007B0163E0FC01828193810E94439DFC0107
:10377000892BA9F09085892F8D7089F4907F9260B4
:103780009087CC24FF2441855285638574854C291C
:103790005D296E297F294187528763877487FF904F
:1037A000EF90DF90CF900895CF92DF92EF92FF924B
:1037B0006A017B0163E0FC01828193810E94439D49
:1037C000009791F0FC0120852F70223069F461850B
:1037D0007285838594856C217D218E219F21FF90A8
:1037E000EF90DF90CF90089560E070E0CB01F7CFCD
:1037F000CF93C62F63E0FC01828193810E94439D99
:10380000FC01892B91F09085892F8D7071F4907F48
:103810009260908781859285A385B4858827BB2790
:103820008C2B81879287A387B487CF910895CF93FC
:10383000DF93EC0169E97AE187EE9AE00E94C48C9B
:103840006DE87AE187EE9AE00E94C48C6C817D81FC
:1038500087EE9AE00E9452A167E87AE187EE9AE04B
:103860000E94C48C87EE9AE00E94F68A60E08C8108
:103870000E948CAAE881F9810484F585E02D60E03E
:10388000CE01199581E090E0DF91CF9108956CEE23
:1038900076E1811102C06EEE76E186E39AE00C9447
:1038A000C48C6BE073E186E39AE00E94C48CF0E084
:1038B000E0E0199584EF91E0089568E17BE08111E3
:1038C00002C063E17BE087EE9AE00C94C48CDC01DB
:1038D00055962C915597273781F4ED91FC91008CEA
:1038E000F18DE02D199569EE76E087EE9AE00E9461
:1038F000C48C87EE9AE00C94F68A08950C94C7CE97
:103900000C94C7CE0C94C7CEEF92FF920F931F93E7
:10391000CF93DF93EC018B0180913B0790913C07A3
:103920000097A9F0FC0120852F70263081F40E94B9
:10393000CB9CFC0190859F70943049F481859285E1
:10394000DF91CF911F910F91FF90EF900895EE8836
:10395000FF88C70101970D97D0F46EE274E0C801AB
:103960000E948FDC892B99F48FE2888F85E08E9DF1
:10397000B0018F9D700D11246657744E46E050E0E3
:10398000CE0149960E949BD0CE014896D9CF90E0B7
:1039900080E0D6CFCF93C1E068EE73E080E090E0A6
:1039A0000E94FDAB6C2F86E39AE00E944BA1CF5F93
:1039B000C43191F784EF91E0CF910895EF92FF9297
:1039C0000F931F93CF93DF936115710511F480E07E
:1039D0008CC0EB018C0188858F70823009F440C067
:1039E0008430A9F763E777E087EE9AE00E94C48C01
:1039F000F801638187EE9AE00E944BA162E374E0D4
:103A000087EE9AE00E946D8C69857A8587EE9AE050
:103A10000E946D8C87EE9AE00E94F68AF801E080A1
:103A2000F180E114F10499F267E374E0C7010E94A8
:103A3000CB9C8C01009759F2FC0180858F708630F9
:103A400031F669857A856115710509F44AC0FB0173
:103A50008081882309F445C0C8010E94CB9C40C0E6
:103A600066E677E087EE9AE00E94C48CF8016381F5
:103A700087EE9AE00E944BA162E374E087EE9AE041
:103A80000E946D8C49855A856B857C852AE030E0E3
:103A900087EE9AE00E94E78B87EE9AE00E94F68A12
:103AA000F801E080F180E114F10409F490CF67E3BC
:103AB00074E0C7010E94CB9C8C01009709F487CF6A
:103AC000FC0180858F708550823008F080CF698539
:103AD000862F9A85892B29F06150C8010E94439D49
:103AE0007C01F801F286E18681E0DF91CF911F91A0
:103AF0000F91FF90EF900895EF92FF920F931F9315
:103B0000CF93DF930097C1F0FC0120812223A1F025
:103B10008C0181ECE82E8BE0F82EC1E0D0E0B701FB
:103B2000C8010E9464D0892B49F02196F5E0EF0E80
:103B3000F11CCE30D10599F7D0E0C0E0CE01DF9185
:103B4000CF911F910F91FF90EF900895CF93DF9346
:103B500000D000D01F921F92CDB7DEB7E0E2FAE0AE
:103B6000128A118A80E090E19587848784E890E04A
:103B7000948B838B81E0868780E090E2908B8787AF
:103B800087E7858B1C821B8287E892E09A83898372
:103B9000FE83ED838FEF9FEF98878F8360E37AE159
:103BA00086E39AE00E94C48C6091DD067091DE0687
:103BB000CE0101960E94CCA280E29AE00E94671C8E
:103BC00060E27AE186E39AE00E94C48C86E39AE0A0
:103BD0000E94F68A0E9437B428960FB6F894DEBF8A
:103BE0000FBECDBFDF91CF910895892B71F0FB01FE
:103BF000828193810E949B9E65ED76E186E39AE047
:103C00000E94C48C88EC90E0089590E080E0F2CFB0
:103C10000F931F93CF93DF93EB0102970CF483C0B4
:103C20000A811B816AEB75E1C8010E9446D0892B8D
:103C300051F481E00E9429A188EC90E0DF91CF91BE
:103C40001F910F91089564EC75E1C8010E9446D060
:103C5000892B11F480E0EECF60E975E186E39AE00C
:103C60000E94C48C0E948BA0672F6095617070E0E9
:103C700086E39AE00E9452A186E39AE00E94F68AC7
:103C80008091120A9091130A892BE9F10A811B8114
:103C90000E942C9E8823B9F1F80101900020E9F7D9
:103CA0003197E01BF10BB09770F582E70E94179EE9
:103CB0008091120A9091130ADC01ED91FC91008829
:103CC000F189E02D60E270E01995B8018091120A47
:103CD0009091130A0E946D8C8091120A9091130AA0
:103CE000DC01ED91FC910190F081E02D60E01995EF
:103CF0008091120A9091130ADC01ED91FC910488E5
:103D0000F589E02D19956A817B8186E39AE00E940E
:103D10006D8C69E875E186E39AE00E94C48C86E3C5
:103D20009AE00E94F68A8091B4079091B5070297B5
:103D30003CF080EF9FEF9093B5078093B4077CCF62
:103D40006CE775E180E49AE00E94C48C80E49AE01C
:103D50000E94F68A84EF91E071CF892B71F0FB010C
:103D6000828193810E94E99E66E675E186E39AE08E
:103D70000E94C48C88EC90E0089590E080E0F2CF3F
:103D8000EF92FF920F931F93CF93DF93CDB7DEB7E0
:103D90002C970FB6F894DEBF0FBECDBF8C017B0110
:103DA0008CE294E09A8389831B821C821D821E828E
:103DB00098878F8319861A861B861C860530110505
:103DC000ECF0BE01695F7F4FF701808591850E940D
:103DD000A614892B99F0CE0107960E948C9FBE01F4
:103DE000695F7F4FF701868197810E94A614892B16
:103DF00061F0CE0107960E9436A00EC0CE0101965A
:103E00000E948C9F0430110554F7CE0101960E9448
:103E100036A003301105A4F1BE01695F7F4FF701A1
:103E2000848195810E94A614892B51F1CE010796B9
:103E30000E94E19FBE01695F7F4FF70182819381FC
:103E40000E94A614892B19F1CE0107960E94379F74
:103E50006FE475E186E39AE00E94C48C80E00E94E2
:103E600020A188EC90E02C960FB6F894DEBF0FBE30
:103E7000CDBFDF91CF911F910F91FF90EF900895EB
:103E8000CE0101960E94E19F023011059CF6CE0101
:103E900001960E94379F01301105D1F6CE0101969F
:103EA0000E94379F66E575E186E39AE00E94C48C24
:103EB000CFCF0F931F93CF93DF938C01EB0102972A
:103EC000C4F08A819B810E94F8CF809301029927D8
:103ED0000E9433A10230110549F08C819D810E941E
:103EE000F8CF8093000299270E943DA1C8ECD0E052
:103EF00002C0C0E9D1E06BE375E186E39AE00E947D
:103F0000C48C6091010286E39AE00E944BA166E2B4
:103F100075E186E39AE00E94C48C6091000286E31A
:103F20009AE00E944BA186E39AE00E94F68ACE01B5
:103F3000DF91CF911F910F910895CF93DF93EB0104
:103F40000297ACF16AEB75E18A819B810E9446D0B1
:103F5000892B29F40E948BA07D7F0E94D0A064EC65
:103F600075E18A819B810E9446D0892B29F40E94A9
:103F70008BA072600E94D0A065E175E186E39AE0B3
:103F80000E94C48C0E948BA071FB662760F971E0CF
:103F9000672770E086E39AE00E9452A186E39AE0E8
:103FA0000E94F68A88EC90E0DF91CF9108950E94FC
:103FB000A61DF8CF0F931F93CF93DF93FC01C4810D
:103FC000D5812097C9F18B0188858F70853021F5C7
:103FD000CE010E94EBA18017110671F16CF1602FE8
:103FE000CE010E94439DFC01892B31F180858F70A9
:103FF000823039F461857285838594850E9460D60C
:1040000006C08330C9F46185728583859485DF910C
:10401000CF911F910F910895672B71F4823029F48D
:1040200069857A858B859C85E9CF833029F46985FC
:104030007A858B859C85EBCF60E070E0CB01E7CF84
:104040000F931F93CF93DF93FC01738362836115FA
:10405000710559F18B01EC011682CB010E94FBA185
:1040600097FD28C09D838C838C819D81009719F0DA
:104070008634910524F080E290E09D838C8361E09A
:1040800070E0C8010E94DA1F20E030E04AE754E403
:104090000E94BFD60E9432D9611571058105910534
:1040A00089F06F83788789879A87DF91CF911F91F5
:1040B0000F9108959195819591099D838C8381E05D
:1040C0008E83D2CF88E893E1A0E0B0E08F83988719
:1040D000A987BA87EACF2F923F924F925F926F9251
:1040E0007F928F929F92AF92BF92CF92DF92EF9288
:1040F000FF920F93CF93DF9300D01F92CDB7DEB71F
:104100007C017A8369835C834B83DB011C92FC0115
:1041100060818FEF860F883108F04BC034FF49C0B3
:10412000FAE06F9FB00111246E5C7A4DCD010E94C0
:104130009BD0D70111968C918F7041F04B815C819F
:1041400067EB74E089819A810E949FDCE981FA81A2
:1041500001900020E9F7319729813A81E21BF30BA6
:1041600019012E0E3F1E4B815C814E1B5F0B41508F
:1041700051095C834B83D7011196EC911197EF7035
:1041800009F4F5C0E150EC3008F0F1C0F0E0882708
:10419000E353FF4D8F4F0C942ED8DC207F21EC2170
:1041A0004B2266222A21FC21FC21FC21182100211E
:1041B000822229803A80DFCFF7018481282F30E0E6
:1041C00050E040E0002359F030E0A4E6B0E00E9467
:1041D000F7D72FEF30E040E050E00E94C5D75F9363
:1041E0004F933F932F938BE394E09F938F93FC81A6
:1041F000FF932B812F933F922F920E94D7DCB2C066
:1042000017968C9117978F9316968C9116978F937C
:1042100015968C9115978F9314968C918F938EE3AE
:1042200094E09F938F93BC81BF93EB81EF93E3CF97
:1042300017968C9117978F9316968C9116978F934C
:1042400015968C9115978F9314968C918F9382E489
:1042500094E0E7CF1496CD90DD90ED90FC90179709
:10426000F7FE34C084E6882E912CA12CB12CC70116
:10427000B601A50194010E94C5D79B01AC01882716
:104280009927DC01821B930BA40BB50BBF93AF9353
:104290009F938F9366277727CB016C197D098E0931
:1042A0009F09A50194010E94C5D75F934F933F9347
:1042B0002F9386E494E09F938F933C813F934B81AF
:1042C0004F933F922F920E94D7DC4CC0C701B6019A
:1042D00024E630E040E050E00E94C5D79F938F93E2
:1042E0007F936F935F934F933F932F9387E494E073
:1042F0009F938F939C819F93AB81AF93E2CFC70134
:104300000E943C16BC01D7011696CC9016971796C2
:10431000DC901797D0FADD24D0F814969C9114976E
:104320001596FC90EB80BC80292F30E050E040E0F7
:1043300077FD35C0011135C07F936F931F921F9297
:104340001F929F931F92FF92DF92CF9280E594E09D
:104350009F938F93FC81FF932B812F933F922F92FA
:104360000E94D7DC0FB6F894DEBF0FBECDBF8981A7
:104370009A810F900F900F900F90DF91CF910F9136
:10438000FF90EF90DF90CF90BF90AF909F908F9075
:104390007F906F905F904F903F902F9008950023F3
:1043A00061F0292F30E0A4E6B0E00E94F7D72FEFAC
:1043B00030E040E050E00E94C5D75F934F933F93B9
:1043C0002F931F92FF92DF92CF9283E594E09F9309
:1043D0008F93BF92EF9275CF15968C9115971F9280
:1043E0008F9316969C91169717968C9181708F9348
:1043F0009F9386E594E015CF14968D909D90AD9097
:10440000BC90179720E030E0A901C501B4010E94DB
:1044100059D62401350187FF04C077FA709477F8E4
:104420007094C301B2010E942BD96B01072E000CBE
:10443000880B990B0E9460D69B01AC01C301B201AD
:104440000E944CD820E030E04AE754E40E94BFD6F6
:104450000E94B6D90E942BD9062F772E20E030E09B
:10446000A901C501B4010E9459D687FF07C07F92F8
:104470000F93DF92CF928CE594E0D3CE7F920F938F
:10448000DF92CF928DE594E09F938F933C813F9391
:104490004B814F93B0CE14968C9114971F928F93AB
:1044A00015968C9115971F928F9316968C911F924B
:1044B0008F9383E594E09F938F93BC81BF93EB81AF
:1044C000EF933F922F920E94D7DC4CCF17968C919E
:1044D00017971F928F9314968C9114971F928F9316
:1044E00015968C9115971F928F9316968C911F920B
:1044F0008F9380E594E09F938F93BC81BF93EB8172
:10450000EF93DFCE14966D917C914B815C81C1015C
:104510000E94BDDC2CCF1F93CF93DF93FC01162F9D
:10452000C389D489818992899C012F5F3F4F328B47
:10453000218BC80FD91FCE010E947DD7181721F0FB
:10454000612FCE010E9485D781E090E0DF91CF916D
:104550001F910895FC0181899289248535858217F0
:10456000930740F423893489820F931F0E947DD7DB
:1045700090E008958FEF9FEF0895DA01E091A10791
:10458000F0E0FE2FEE27E60FF71F90E0982F882728
:10459000A901BD018E0F9F1F0C948394CF93DF93CD
:1045A0001F92CDB7DEB72091A10730E0322F22272E
:1045B000260F371F90E0982F8827498341E050E06D
:1045C000BE016F5F7F4F820F931F0E9483940F90F5
:1045D000DF91CF910895CF93DF931F92CDB7DEB7D0
:1045E00041E050E0BE016F5F7F4F0E94F8938981E8
:1045F0000F90DF91CF9108952091A10730E0322FE5
:104600002227620F731F90E0982F8827860F971F2D
:104610000C94EB2263E070E00C94FC22DA01E09150
:10462000A107F0E0FE2FEE27E60FF71F90E0982F8E
:104630008827A901BD018E0F9F1F0C94F89344E0B9
:1046400050E0BC018FE090E00C94839444E050E093
:10465000BC0185E090E00C94839444E050E0BC0100
:1046600081E090E00C94839408959F92AF92BF9262
:10467000CF92DF92EF92FF920F931F93CF93DF932E
:104680008C015B01942EE52EFC01C688D788F08C46
:1046900080E591E00E94DEA68F2D0E94D496C92D60
:1046A000DE2D8C179D0708F4EC019E01A501B601D3
:1046B0008F2D0E945196F801868997898C0F9D1F36
:1046C000978B868BCE01DF91CF911F910F91FF9039
:1046D000EF90DF90CF90BF90AF909F900895CF93D1
:1046E000FC01C08D80E591E00E94DEA660E270E0F2
:1046F0008C2F0E94E89362E070E08C2F0E94FC22D5
:1047000084FD16C062E070E08C2F0E94FC2283FFC3
:104710000AC048E162E070E08C2F0E94CE2280E067
:1047200090E0CF91089580E591E00E94DEA6E3CF6E
:1047300040E162E070E08C2F0E94CE2281E0F0CF59
:10474000FF920F931F93CF93DF93EB01FC01178A26
:10475000168A2A81211109C02B81211106C02C81C2
:10476000211103C02D81222301F141155105E9F0EA
:104770008A01FC01F08C80E591E00E94DEA6AE018A
:104780004E5F5F4F24E030E06CE070E08F2D0E94C0
:10479000BD22B8018F2D0E94DB9881E090E0DF916F
:1047A000CF911F910F91FF90089580E0F7CF0F9365
:1047B0001F93CF938C01FC016481758181E20E947B
:1047C0000799C82F8830F8F480E591E00E94DEA6B2
:1047D0008C2F0E940A23833131F08C2FCF911F91AF
:1047E0000F910C94B09862E070E08C2F0E94E893D7
:1047F000F80184819581EC2FF0E0EE0FFF1FED5F53
:10480000F64F91838083CF911F910F9108950F935D
:104810001F93CF93DF931F921F92CDB7DEB7FC019A
:1048200024852830E0F48C0180E591E00E94DEA62A
:1048300022E030E0AE014F5F5F4F60E170E0F801D1
:1048400084850E940E2389819A8198278927982739
:104850000F900F90DF91CF911F910F91089590E0ED
:1048600080E0F6CF0F931F93CF93DF931F921F9299
:10487000CDB7DEB7FC0124852830E0F48C0180E55B
:1048800091E00E94DEA622E030E0AE014F5F5F4F74
:1048900064E070E0F80184850E940E2389819A818A
:1048A0009827892798270F900F90DF91CF911F911C
:1048B0000F91089590E080E0F6CFCF93DF93EC0165
:1048C0008CE294E0998388831A821B821C821D8269
:1048D00080E591E00E94DEA6BE016E5F7F4F44E05E
:1048E00050E08FE090E00E94F893CE01DF91CF91ED
:1048F00008950E944495882331F0809113098433F0
:1049000029F0873381F090E080E0089580E591E020
:104910000E94DEA685E390E00E94EB2285FD0DC09B
:1049200082E090E0089580E591E00E94DEA68EE2AC
:1049300090E00E94EB2280FFF3CF81E090E00895A9
:1049400010923A0981E0809339091092140961E0CC
:1049500084E10E945EAA61E085E10E945EAAE9EB23
:10496000F0E080818E7F808380818D7F808388E4EA
:104970008093B80085E48093BC000895CF93DF93C3
:1049800091E090933D07882361F0C091B800D091E9
:10499000BA000E94611B0E94A024D093BA00C09369
:1049A000B800DF91CF910895CF92DF92EF92FF92FE
:1049B0000F931F93CF93FC01C1810E94E5AA6B0165
:1049C0007C0180913A09811164C081E080933A09A9
:1049D000809339099FEF909338091092370910920C
:1049E00036098093150980911509CC0FC82BC09307
:1049F000150980911409813009F081C010921409C1
:104A00000E94E5AA6B017C01809115098093BB008F
:104A100080913C0990913D09A0913E09B0913F09D8
:104A2000892B8A2B8B2BA1F00E94E5AA00913C09CF
:104A300010913D0920913E0930913F096C197D0983
:104A40008E099F09061717072807390708F442C07F
:104A50008091BC0083FDD8CF85EC8093BC000E9480
:104A6000E5AA6B017C0180913A09813009F449C0C3
:104A700080913709811167C080913709E6E1F9E03B
:104A8000A1E8B7E090E0981751F121912D939F5F35
:104A9000FACF80913C0990913D09A0913E09B091D7
:104AA0003F09892B8A2B8B2B09F48BCF0E94E5AA17
:104AB00000913C0910913D0920913E0930913F0938
:104AC0006C197D098E099F090617170728073907F2
:104AD00008F077CF80913B090E94BE2480E01092BD
:104AE00069098093680987EA99E00E941914CF91B7
:104AF0001F910F91FF90EF90DF90CF90089585EE7A
:104B0000ACCF80913C0990913D09A0913E09B091B4
:104B10003F09892B8A2B8B2B09F4A5CF0E94E5AA8C
:104B200000913C0910913D0920913E0930913F09C7
:104B30006C197D098E099F09061717072807390781
:104B400008F091CFC7CF81E099CF8F929F92AF921B
:104B5000BF92EF92FF921F93CF93DF93EC010E94DD
:104B600030AC4B015C0110E08BE4E82EF12C0E948C
:104B700030AC681979098A099B09683E7340810540
:104B8000910510F5ED85FE85309709F0199560EFD8
:104B9000CE010E94461BCE010E94D424182F80FD16
:104BA0000FC08A81813009F41A82812FDF91CF9161
:104BB0001F91FF90EF90BF90AF909F908F900895BE
:104BC000C7010197F1F7D3CF81E08A83EECF1F931E
:104BD000CF93DF93EC01162F0E94A525CE010E94F2
:104BE000D51362ED87EA99E00E946014612F70E0AE
:104BF0006095709584E0660F771F8A95E1F7612BC9
:104C000087EA99E00E9460140E94FAABCE010E94EC
:104C1000D424811731F084E08A83DF91CF911F91F2
:104C200008958A818430C9F71A82F7CFCF93DF9332
:104C3000EC0163EC0E94461BCE01DF91CF910C94F6
:104C4000D4240F931F93CF93DF93EC01162F042FDF
:104C50000E94A525002341F0CE010E941626682F50
:104C60006460CE010E94E725CE010E94D51365EA5B
:104C700087EA99E00E946014612F87EA99E00E9418
:104C80006014DF91CF911F910F910C94FAABEF92CA
:104C9000FF920F931F93CF93DF938C017B0140E032
:104CA00065E50E942126E70188E0E80EF11C699184
:104CB00040E0C8010E942126CE15DF05C1F7DF9133
:104CC000CF911F910F91FF90EF900895CF93DF93B5
:104CD000EC010E94D51340E060EFCE010E94212636
:104CE000DF91CF910C94FAAB0F931F93CF93DF9387
:104CF000EC010E94A52580FD36C0CE010E9416263B
:104D000060E0CE010E94E725CE010E94A525CE01DC
:104D10000E94D51364EB87EA99E00E9460140E9418
:104D2000FAABCE010E94A525082F10E082FF16C025
:104D300082E08A838881882341F0CE010E94162672
:104D4000682F6160CE010E94E72515950795802F99
:104D50008170DF91CF911F910F9108958A818230E8
:104D600049F71A82E7CF80E0F4CFCF92DF92EF923B
:104D7000FF920F931F93CF93DF938C01EB017A0186
:104D8000FC01858196810E9474268823C1F1BE01B1
:104D9000F801858196810E94472640E06EEBF8017C
:104DA000858196810E942126E7016701F9E0CF0EF7
:104DB000D11CF801E580F680C7010E94A525C70136
:104DC0000E94D51366E987EA99E00E9460140E9468
:104DD000FAABC7010E94A52561EEC7010E94461BE0
:104DE000C7010E94D4248993CC16DD0611F7F8017F
:104DF000858196810E94742691E0813009F090E0CF
:104E0000892FDF91CF911F910F91FF90EF90DF904D
:104E1000CF900895CF93DF93EA010E94B5268823AF
:104E200081F0DE0189E090E0815039F0ED91E927D1
:104E3000F0E0E158F34E9491F7CF81E028852913F3
:104E400080E0DF91CF910895CF93DF9300D000D021
:104E500000D0CDB7DEB7AE014F5F5F4F0E940A278B
:104E6000882331F08D818F33A9F020F48F31A1F0A8
:104E700080E007C08F3521F08F37D1F78CE001C07B
:104E80008BE029960FB6F894DEBF0FBECDBFDF9141
:104E9000CF9108958AE0F5CF89E0F3CF6F927F92AA
:104EA0008F929F92AF92BF92CF92DF92EF92FF923A
:104EB0000F931F93CF93DF93FC01248521118CC0A6
:104EC000872E762EEC010E947426882309F486C072
:104ED000CE010E94A52540E060EFCE010E94212670
:104EE00010E000E066246A94AA24A394B12CE02E7A
:104EF000E694E694E694F12C802F8770650101C05A
:104F0000CC0C8A95EAF78B85082E000C990B0817B4
:104F1000190734F5FE01EE0DFF1D93809C20CE0194
:104F20000E94A525CE010E94D51368E787EA99E083
:104F30000E946014992011F080E8982E692D87EA6C
:104F400099E00E9460140E94FAABCE010E94A52550
:104F5000982F907485FF0BC0992369F08EEF2AC0BB
:104F60009924939408171907D1F2912CD8CF911155
:104F700002C087FF602EFE01EE0DFF1D938187FFAB
:104F800028C0C92AC3820F5F1F4F0034110509F0E2
:104F9000AECF6B86FFEF6F1202C081E08C87239645
:104FA000E72DF82DCF01089629912193E817F907ED
:104FB000D9F781E0DF91CF911F910F91FF90EF9092
:104FC000DF90CF90BF90AF909F908F907F906F9029
:104FD0000895C094C922D6CF80E0ECCF8FEFEACFFE
:104FE00085ED8093BC0080913C0990913D09A09192
:104FF0003E09B0913F090796A11DB11D23E0B6956A
:10500000A795979587952A95D1F72091BC0024FD07
:1050100003C010923A09089540913C0950913D090E
:1050200060913E0970913F09452B462B472B69F350
:105030000097A105B10541F02AE22A95F1F700C0D9
:105040000197A109B109E1CF80913B090C94BE24DD
:105050001F920F920FB60F9211240BB60F922F933F
:105060003F934F935F936F937F938F939F93AF93F0
:10507000BF93EF93FF938091B900887F803609F446
:105080004DC008F040C0883209F4A9C028F580312D
:1050900009F49DC0C8F4882309F4FBC0883009F4E2
:1050A00096C0FF91EF91BF91AF919F918F917F91AA
:1050B0006F915F914F913F912F910F900BBE0F9089
:1050C0000FBE0F901F901895883109F488C0803268
:1050D00041F78093380914C0803409F49DC040F42E
:1050E0008033B9F38833E9F68093380985ECB0C092
:1050F000803509F485C0883509F496C0883489F66E
:105100000E94F027CECF883909F48CC038F5883753
:1051100029F050F4883611F0803719F683E0809337
:105120003A091092800757C0883809F47BC080394B
:1051300019F0803809F0B5CF80918007803208F0EF
:1051400071C0E091800781E08E0F8093800780918D
:10515000BB00F0E0E05AF84F80833DC0803B39F05F
:10516000E0F4803A09F479C0883A09F09ACF84E0F3
:1051700080933A0910925F0710925E07E0916409EC
:10518000F0916509199580915E0781110FC081E04A
:1051900080935E0710923E0709C0803C09F4A6CFB9
:1051A000883C09F4A3CF883B09F07BCFE0915F07EF
:1051B00081E08E0F80935F07F0E0E25CF84F808122
:1051C0008093BB0090915F0780915E0729C080911A
:1051D00015098093BB0085EC8093BC0062CF909151
:1051E000370980913609981758F5E091370981E021
:1051F0008E0F80933709F0E0EA5EF64F8081E9CFA9
:10520000E091370981E08E0F809337098091BB00D0
:10521000F0E0EA5EF64F808390913709809136097D
:105220009817C8F285E8D8CFE091370981E08E0F52
:10523000809337098091BB00F0E0EA5EF64F8083EF
:105240008091390981115CCF81E08093140984EA4F
:105250008093BC0010923A0924CF85EC8093BC0067
:1052600010923A0980918007803230F4E0918007F3
:10527000F0E0E05AF84F10826091800770E0E09112
:105280006209F091630980E697E019951092800712
:1052900008CF1092380934CF009789F0FC0120859F
:1052A0002F70253061F40E94439D009741F0FC016E
:1052B00020852F70243019F481859285089590E01F
:1052C00080E008950F931F93CF93DF9365E77CE110
:1052D00087EE9AE00E94E88C81E00E940AAB0E946F
:1052E000611B61E085E10E948CAA60E084E10E947C
:1052F0008CAAC4E1D0E010E001E0612F85E10E94BA
:105300005EAA10276AE070E080E090E00E94FDABAA
:10531000219799F764E170E080E090E00E94FDAB96
:105320000E941FA78091AB079091AC07009729F1CD
:105330000E94571B882309F18091AB079091AC071D
:105340000E9466266AE57CE187EE9AE00E94E88C7E
:10535000E091AB07F091AC0700838091AB0790918F
:10536000AC070E94742666E47CE1811102C061E30F
:105370007CE187EE9AE00E94E88C81E0DF91CF919A
:105380001F910F910895CF92DF92EF92FF920F93AA
:105390001F93182F6A017B010E9430AC04C09695C0
:1053A0008795779567951A95D2F76C217D218E2187
:1053B0009F218B019C0101501109210931090E3FE8
:1053C0001F4F2F4F3F4F20F061E070E080E090E0F2
:1053D0001F910F91FF90EF90DF90CF9008953F9233
:1053E0004F925F926F927F928F929F92AF92BF92F5
:1053F000CF92DF92EF92FF920F931F93CF93DF93A1
:1054000000D000D0CDB7DEB77C01362E80913A07B0
:10541000882309F40DC1D70114969C918091000254
:10542000891708F405C18091380790913907BAE0CF
:105430006B1318C28D51994FFC011082D701189639
:105440008D919C91892B09F4EFC08091DF0690919A
:10545000E006A091E106B091E206892B8A2B8B2B06
:1054600009F0CEC00E9430AC2B013C01F701008551
:105470001185D80119966D917C916115710599F48A
:10548000F80185809680A780B08480919D099091D5
:105490009E09A0919F09B091A00988169906AA06B5
:1054A000BB0609F487C0D8011B964D915C911C97EF
:1054B0004115510509F47EC0F701248153968C9162
:1054C000539790E0322F377002C0959587953A95A3
:1054D000E2F780FF6FC0C22ED12CC601887F937087
:1054E000892B39F451968D919C91887F9370C82AAD
:1054F000D92AD8018D919C91DC01ED91FC91611527
:10550000710509F4C4C00688F789E02D1995019743
:1055100009F050C06CE3F801808191810E94FA8A01
:10552000A60170E060E02AE0D8018D919C910E9474
:10553000AA8AF8012281808191816CE37BE1222398
:1055400011F06AE37BE10E94C48CD8011D966D9135
:105550007C911E978D919C910E946D8C60E2F80168
:10556000808191810E94FA8AD8011F966D917C9169
:1055700050978D919C910E946D8CF80122818081C1
:1055800091816FE27BE1222311F069E27BE10E94CD
:10559000C48C63EE76E0D8018D919C910E946D8C55
:1055A000F80180819181DC01ED91FC91008CF18DFD
:1055B000E02D19950E9430ACAB01BC01441955098E
:1055C00066097709F70185819681453651056105A0
:1055D000710508F472C0009721F069E77BE10E9431
:1055E000E88C4FEF5FEFBA0180E00E94C32960931F
:1055F000DF067093E0068093E1069093E20614C004
:105600000E9430AC0091DF061091E0062091E10687
:105610003091E206601B710B820B930B6033754770
:105620008105910508F01ECF1092390710923807B6
:10563000D70115968D919C911697009771F014964D
:105640003C9120910102231740F0DC01ED91FC9187
:105650000190F081E02D632D199581E090E0269670
:105660000FB6F894DEBF0FBECDBFDF91CF911F9173
:105670000F91FF90EF90DF90CF90BF90AF909F90F1
:105680008F907F906F905F904F903F900895048827
:10569000F589E02D2CE234E03A832983D801159670
:1056A0008D909D90AD90BC9018978B829C82AD821E
:1056B000BE82BE016F5F7F4F29CF4091DF065091C0
:1056C000E0066091E1067091E206452B462B472BE0
:1056D00009F4AACF009721F06AE67BE10E94E88CEA
:1056E0001092DF061092E0061092E1061092E20698
:1056F000D70118960D911C91F8016185728561158D
:10570000710591F4458056806780708480919D0971
:1057100090919E09A0919F09B091A0094816590641
:105720006A067B0609F480CFD8011B964D915C91E7
:105730001C974115510509F477CFF7012481539641
:105740008C91539790E0322F377002C095958795D2
:105750003A95E2F780FF68CFC22ED12CC601887F30
:105760009370892B39F451968D919C91887F937019
:10577000C82AD92AD8018D919C91DC01ED91FC9128
:105780006115710509F458C00688F789E02D19954F
:10579000019709F049CF6CE3F801808191810E9463
:1057A000FA8AA60170E060E02AE0D8018D919C9110
:1057B0000E94AA8AF80122818081918165E57BE1BE
:1057C000222311F063E57BE10E94C48CD8011D9671
:1057D0006D917C911E978D919C910E946D8C60E2E1
:1057E000F801808191810E94FA8AD8011F966D91FB
:1057F0007C9150978D919C910E946D8CF801228133
:105800008081918168E47BE1222311F062E47BE1F5
:105810000E94C48C6BE57BE1D8018D919C910E9424
:10582000C48CF80180819181DC01ED91FC91008CA8
:10583000F18DE02D1995F8CE0488F589E02D2CE244
:1058400034E03A832983D80115964D905D906D9090
:105850007C9018974B825C826D827E82BE016F5F66
:105860007F4F95CF843591050CF0E2CEBDE06B17EC
:1058700009F4DECE9C012F5F3F4F30933907209310
:1058800038078D51994FFC016083D2CE8F929F9241
:10589000AF92BF92CF92DF92EF92FF920F931F933E
:1058A000CF93DF937C014A015901C0913B07D0910E
:1058B0003C07062F660F110B209709F45CC0888502
:1058C0008F70863009F055C065E674E0CE010E9405
:1058D000CB9C6C0182E08816910449F06AE674E082
:1058E000E3E08E16910429F0D0E0C0E006C06EE639
:1058F00074E0CE010E94CB9CEC01C114D104D9F11B
:10590000F60180858F708430B1F561857285A801BC
:10591000C7010E94BDDCA80163E774E0C7010E94D3
:105920009FDC209779F188858F70843059F56985DF
:105930007A85A801C7010E949FDCA80163E774E093
:10594000C7010E949FDCA114B10429F0A801B50190
:10595000C7010E949FDCC701DF91CF911F910F917A
:10596000FF90EF90DF90CF90BF90AF909F908F907F
:105970000895D0E0C0E0A8016DED7BE1C7010E9471
:105980009BD0C9CFF2E08F16910481F083E0881696
:10599000910429F06091A3077091A407CACFA801D0
:1059A00067ED7BE1C7010E947DD0C7CFA80164ED00
:1059B0007BE1F8CFCF92DF92EF92FF920F931F938C
:1059C000CF93DF93CDB7DEB7C154D1090FB6F894AA
:1059D000DEBF0FBECDBF6C01AB0130E020E060E464
:1059E000CE0101967C010E94462CF7010190002017
:1059F000E9F731978F010E191F09A801B701C601F8
:105A00000E94AFDC892B11F010E000E0C801CF5BF1
:105A1000DF4F0FB6F894DEBF0FBECDBFDF91CF9141
:105A20001F910F91FF90EF90DF90CF900895EF922C
:105A3000FF920F931F93CF937C018C01C0E0C33082
:105A4000E1F0F801428150E070E060E02AE030E0EF
:105A500086E39AE00E94E78B62ED7BE186E39AE0C1
:105A60000E94C48CCF5F0F5F1F4FC43041F7CF91AE
:105A70001F910F91FF90EF900895F701458150E03D
:105A800070E060E02AE030E086E39AE00E94E78B75
:105A900060ED7BE1E3CFCF93DF931F921F92CDB7F1
:105AA000DEB780911D0C90911E0C009711F489E2D5
:105AB0009CE0BE016F5F7F4F681B790B072E000CC7
:105AC000880B990B0F900F90DF91CF9108954F9213
:105AD0005F926F927F928F929F92AF92BF92DF926E
:105AE000EF92FF920F931F93CF93DF93CDB7DEB763
:105AF00060970FB6F894DEBF0FBECDBFFC011986CC
:105B00001A861B861C868A85807F8A87A081B18140
:105B1000109709F4ECC08C91882309F4E8C0008147
:105B20001181D8019C91992309F443C09D3209F455
:105B3000E2C090539A3028F00F5F1F4F118300830B
:105B4000EECFC801D12CDC017D01E81AF90A2D91B4
:105B5000022E000C330B205331092A303105A0F3FB
:105B60005F016EE270E0C8010E9484DCFC010097D6
:105B700009F448C0DC014D018E1A9F0A11968C91E0
:105B80001197082E000C990BC09711960A9798F35D
:105B90008181282F082E000C330B205331092A3025
:105BA000310518F480330CF05BC020E030E0A9012F
:105BB00008C0D12CF12CE12CD3CF29E030E040E01B
:105BC00050E0AAE0B0E00E94E4D72B013C01228122
:105BD000822F022E000C990BC0978A30910570F429
:105BE00020330CF445C02A330CF046C0092E000CBB
:105BF000AA0BBB0B480E591E6A1E7B1E8114910412
:105C000009F088C0EF2809F07BC01D861E861F861C
:105C1000188A88E0FE013996DE01119601900D92F6
:105C20008A95E1F729813A814B815C816D817E8182
:105C30008F81988560960FB6F894DEBF0FBECDBFFA
:105C4000DF91CF911F910F91FF90EF90DF90BF9068
:105C5000AF909F908F907F906F905F904F9008953E
:105C60008A330CF0AACF032E000C440B550BA9CF9E
:105C700080E090E0DC01BECF89E090E0A0E0B0E001
:105C8000B9CFB8E0EB16F1040CF049C0C8010E948E
:105C900016D09B01AC01A4E6B0E00E94E4D7DD2061
:105CA00041F07094609450944094411C511C611CCC
:105CB000711C2A85207F26602A87460E571E681E83
:105CC000791E6CE270E0F501808191810E9484DC94
:105CD000009741F4D5011D921C924D865E866F8619
:105CE000788A97CF0196F50191838083F6CF412C76
:105CF000512C3201F2CFC8010196DD24D39423CF79
:105D0000C8010E9416D02A85207F2A602A872B018D
:105D10003C01D7CFF3E08F1691040CF4B2CFC80149
:105D20000E94F4CF2B013C018A85807F87608A879F
:105D3000C8CFCF92DF92EF92FF920F931F93CF9332
:105D4000DF93EC01A881B981109781F18C918823B0
:105D500069F108811981F8019081992351F09D32F0
:105D600041F090539A3028F00F5F1F4F198308833A
:105D7000F0CFC8010E9416D06B017C016CE270E08C
:105D8000C8010E9484DC009769F419821882C70157
:105D9000B601DF91CF911F910F91FF90EF90DF90AF
:105DA000CF900895019699838883F1CFC12CD12C8F
:105DB0007601EDCF0097B1F1FC01DB01AC01405F52
:105DC0005F4F80E090812FE9290F263098F4975596
:105DD0009295907F9C9321813FE9320F3630B0F449
:105DE0002755922B9D933296E417F50759F791E0CA
:105DF000892708952FEB290F263010F49753E8CF09
:105E000090539A3028F381E090E0E2CF3FEB320FDD
:105E1000363010F42753E5CF20532A3010F381E0B9
:105E200020E0DFCF80E008950097D1F0DC011696E6
:105E3000ED91FC913097A1F080858F70843021F432
:105E400081859285009771F40680F781E02D309767
:105E500039F080858F70843019F48185928508959A
:105E600090E080E00895CF92DF92EF92FF920F933F
:105E70001F93CF93DF93CDB7DEB769970FB6F89432
:105E8000DEBF0FBECDBFE091AB07F091AC073097FE
:105E900009F483C08091B8079091B907892B09F460
:105EA0007CC08FEF8387148613821482158216823A
:105EB00017821086118612866CE273E186E39AE0FF
:105EC0000E94C48C86E39AE00E94F68A8E010F5EDF
:105ED0001F4FBE016E5E7F4F8091AB079091AC0764
:105EE0000E944E2718160CF058C0A895DE01119696
:105EF0009E012E5E3F4F7D01F90141919F01842F4C
:105F000090E054E0959587955A95E1F7865D9D4F11
:105F1000FC0180818C93E42FEF70F0E0E65DFD4F93
:105F2000808111968C9311971296A017B10721F7D3
:105F3000198AB7018091B8079091B9070E94CB9C4C
:105F40006C0167E273E186E39AE00E94C48CB701BA
:105F500086E39AE00E946D8CC114D104B9F0C601A9
:105F60000E94142F7C01892B09F4B3CF62E273E104
:105F700086E39AE00E94C48CB70186E39AE00E940F
:105F80006D8C86E39AE00E94F68AA3CF6DE173E1FF
:105F900086E39AE00E94C48CF4CF88EC90E0699686
:105FA0000FB6F894DEBF0FBECDBFDF91CF911F912A
:105FB0000F91FF90EF90DF90CF900895089508958E
:105FC000EF92FF921F93CF93DF93192F7B01C82F7E
:105FD000D92FD7FF03C0D195C195D10961E08C2F8E
:105FE0000E948CAA82E0E816F10499F460E08C2FFC
:105FF0000E945EAA68E17AE187EE9AE00E94C48C72
:1060000087EE9AE0DF91CF911F91FF90EF900C9473
:10601000F68A612FEF2851F46095661F6627661F88
:106020008C2F0E945EAA64E17AE1E6CF661F6627A4
:10603000661F8C2F0E945EAA6FE07AE1DDCF6DEEC5
:1060400079E186E39AE00E94C48C6AED79E186E307
:106050009AE00E94C48C6CEC79E186E39AE00E949D
:10606000C48C64EC79E186E39AE00E94C48C86E3F8
:106070009AE00E94F68A64EB79E186E39AE00E9456
:10608000C48C68EA79E186E39AE00E94C48C6BE9EB
:1060900079E186E39AE00E94C48C66E879E186E3C0
:1060A0009AE00E94C48C67E779E186E39AE00E9457
:1060B000C48C6FE679E186E39AE00E94C48C64E6C2
:1060C00079E186E39AE00E94C48C67E579E186E392
:1060D0009AE00E94C48C6DE479E186E39AE00E9424
:1060E000C48C6EE379E186E39AE00E94C48C66E397
:1060F00079E186E39AE00E94C48C6AE279E186E362
:106100009AE00E94C48C60E179E186E39AE00E9403
:10611000C48C61EF78E186E39AE00E94C48C6CED58
:1061200078E186E39AE00E94C48C6FEC78E186E324
:106130009AE00E94C48C61EC78E186E39AE00E94C8
:10614000C48C65EB78E186E39AE00E94C48C6DEA2A
:1061500078E186E39AE00E94C48C62EA78E186E303
:106160009AE00E94C48C65E978E186E39AE00E9497
:10617000C48C6DE878E186E39AE00E94C48C62E802
:1061800078E186E39AE00E94C48C63E778E186E3D5
:106190009AE00E94C48C6AE678E186E39AE00E9465
:1061A000C48C6CE578E186E39AE00E94C48C6EE4CE
:1061B00078E186E39AE00E94C48C62E478E186E3A9
:1061C0009AE00E94C48C6AE378E186E39AE00E9438
:1061D000C48C67E278E186E39AE00E94C48C6DE1AA
:1061E00078E186E39AE00E94C48C86E39AE00C94FE
:1061F000F68A0F931F93CF93DF9300D000D0CDB7D3
:10620000DEB70E941F3067E770E186E39AE00E94E4
:10621000C48CCE0101960E945D24CE0101960E949D
:10622000172D0CE214E01A8309838091A309909141
:10623000A409A091A509B091A6098B839C83AD8385
:10624000BE83CE0101960E94172D1A8309831B82FB
:106250001C821D821E8280E591E00E94DEA644E041
:1062600050E0BE016D5F7F4F81E090E00E94F893A7
:10627000CE0101960E94172D1A8309831B821C826E
:106280001D821E8280E591E00E94DEA644E050E07F
:10629000BE016D5F7F4F85E090E00E94F893CE01D4
:1062A00001960E94172D6DE970E186E39AE00E9445
:1062B000C48C88EC90E026960FB6F894DEBF0FBE33
:1062C000CDBFDF91CF911F910F9108958091A207CB
:1062D0008823B1F0E091D306F091D406309731F0E5
:1062E000868197819093A6078093A50760E670E169
:1062F00086E39AE00E94C48C86E39AE00C94F68AC6
:106300000895CF92DF92EF92FF920F931F93CF9356
:10631000DF9300D000D0CDB7DEB780913A0781116E
:106320009AC08091B4079091B50702970CF493C07E
:106330008091DD069091DE06009709F48CC067E736
:1063400074E00E94CB9C8C01009709F484C00E94E9
:10635000EBA1E82EF12CE114F10409F47CC070E00B
:1063600060E0C8010E944C296C01EA94EF2809F40E
:1063700081C061E0C8010E94439DFC010185128536
:10638000CE0101960E945D24CE0101960E94E1A6F5
:1063900061E570E186E39AE00E94C48CB60186E371
:1063A0009AE00E946D8C63EF74E086E39AE00E94AD
:1063B0006D8CB80186E39AE00E9452A163EF74E00D
:1063C00086E39AE00E946D8C6AE679E086E39AE0C3
:1063D0000E946D8C86E39AE00E94F68A62E072E089
:1063E00085E09BE00E949119D092FB0AC092FA0AC4
:1063F0001093FD0A0093FC0A8AE699E0892BE9F5DF
:1064000085E794E09093FF0A8093FE0A8091A507A8
:106410009091A607009741F070E060E00E944C293F
:106420009093A4078093A3078091A3079091A4075A
:10643000009731F19093010B8093000B1092030BA6
:106440001092020B81E080933A0768E370E186E3E3
:106450009AE00E94C48C26960FB6F894DEBF0FBE59
:10646000CDBFDF91CF911F910F91FF90EF90DF9003
:10647000CF90089502E012E083CF8AE699E0C2CF80
:106480008AEC92E0892B19F485E794E0D3CF8AEC6B
:1064900092E0D0CF0F931F93CF9363E370E186E335
:1064A0009AE00E94C48C0AE11AE0C0E0F8018191F0
:1064B0008F01803130F46EE774E086E39AE00E9449
:1064C0006D8CC530C9F0F8013197408150E070E023
:1064D00060E020E130E086E39AE00E94E78B61E330
:1064E00070E186E39AE00E94C48CCF5FC630F1F67B
:1064F000CF911F910F91089540911F0A50E070E0D5
:1065000060E020E130E086E39AE00E94E78B86E3DA
:106510009AE00E94F68AE9CFEF92FF920F931F93C1
:10652000CF93DF9300D000D01F92CDB7DEB77B01B1
:10653000CE0107969F938F9301979F938F93019717
:106540009F938F9301979F938F9301979F938F931F
:1065500001979F938F938E010F5F1F4F1F930F9390
:1065600080E894E09F938F93DB0113968C911397AF
:106570008F9312968C918F930E9444DD0FB6F894FE
:10658000DEBF0FBECDBF0697ECF46AEA76E180E489
:106590009AE00E94C48CD70112966D917C9180E4A0
:1065A0009AE00E946D8C80E991E027960FB6F894EE
:1065B000DEBF0FBECDBFDF91CF911F910F91FF9036
:1065C000EF9008958091120A9091130A892BA9F1F6
:1065D0000E942C9E882389F182E70E94179E809159
:1065E000120A9091130ADC01ED91FC910088F18967
:1065F000E02D64E070E019958091120A9091130AE1
:10660000DC01ED91FC910280F381E02D46E050E049
:10661000B801199586E0F801AAE1BAE001900D925F
:106620008A95E1F78091120A9091130ADC01ED91AD
:10663000FC910488F589E02D19950E944A326CEB93
:1066400076E186E39AE00E94C48C88EC90E0ADCFBE
:106650000895EF92FF920F93CF93DF93CDB7DEB7FC
:10666000A0970FB6F894DEBF0FBECDBF7C0100E04F
:1066700020E030E340E250E0BE016F5F7F4F0E94B8
:106680006B20BE016F5F7F4F87EE9AE00E946D8C9A
:1066900062EA7EE087EE9AE00E94C48CF701618195
:1066A0006F7087EE9AE00E944BA16BE97EE087EE67
:1066B0009AE00E94C48CF701628187EE9AE00E9402
:1066C0004BA187EE9AE00E94F68AA0960FB6F89446
:1066D000DEBF0FBECDBFDF91CF910F91FF90EF9046
:1066E0000895CF93DF9300D000D01F921F92CDB7B3
:1066F000DEB7FC01628398E0DE01119601900D92F5
:106700009A95E1F729813A814B815C816D817E8187
:106710008F81988528960FB6F894DEBF0FBECDBF47
:10672000DF91CF910895CF93DF9300D000D01F92D7
:106730001F92CDB7DEB7FC01608398E0DE011196B1
:1067400001900D929A95E1F729813A814B815C8104
:106750006D817E818F81988528960FB6F894DEBF73
:106760000FBECDBFDF91CF9108952F923F924F92F0
:106770005F926F927F928F92AF92BF92CF92DF9291
:10678000EF92FF920F931F93CF93DF93CDB7DEB7B6
:10679000C457D1090FB6F894DEBF0FBECDBF3C0180
:1067A000AE960FAFAE97AF961FAFAF97E0962FAFF5
:1067B000E097E1963FAFE197E2964FAFE297E3961D
:1067C0005FAFE397E4966FAFE497E5967FAFE59709
:1067D00023961FAE1EAE2397FE01ED5BFF4F82E1B5
:1067E000DF011D928A95E9F77296119211928EE05F
:1067F000DF011D928A95E9F764E974E087EE9AE07B
:106800000E946D8CB50187EE9AE00E946D8C67EB5B
:1068100074E087EE9AE00E946D8CCE0183599F4F01
:106820000E942933D4FE2CC0AE96EFADAE97E8316E
:1068300008F067C1F0E08827EF5DFB4C8F4F0C94A8
:106840002ED8873539347E35813581357E353934DA
:1068500081358135813581358135813581353934D1
:1068600039348135813581353934393439343934E5
:10687000873568E37CE0CE018B5A9F4F0E946DD034
:106880000E94E99C882309F419C18091AF07811106
:1068900015C1A114B10409F05FC030E020E043E06D
:1068A00050E060E4CE0101960E94462CD30112967E
:1068B000ED91FC91608171814FE350E0CE01019632
:1068C0000E949FDCD5FE26C1AE968FADAE9782307A
:1068D00009F420C1853009F41DC1AF968FADAF9783
:1068E0008F709FE0980F9F70923018F0883009F0F9
:1068F00011C101E020E030E244E150E0BE016F5BF5
:106900007F4FCE0183599F4F0E946B20482DBE01BF
:106910006F5B7F4FCE0101960E94FEAC6EE07CE083
:1069200087EE9AE00E94C48CBE016F5F7F4F87EEB6
:106930009AE00E946D8C6BE07CE087EE9AE00E940A
:10694000C48CBE016F5B7F4F87EE9AE00E946D8C16
:1069500087EE9AE00E94F68AAF968FADAF978F7060
:106960001601270122243324B0E14B225524882329
:1069700011F0D5FC06C0211431044104510409F47E
:1069800009C130E020E043E050E060E4CE01019630
:106990000E94462CD3011296ED91FC916081718189
:1069A0004FE350E0CE0101960E949FDCA114B10498
:1069B00069F063E774E0CE0101960E9479DC4FE351
:1069C00050E0B501CE0101960E949FDC63E774E0C0
:1069D000CE0101960E9479DC4FE350E060ED7BE050
:1069E000211431044104510459F4E0968FADE0972D
:1069F0004FE350E06FED7BE0873011F066EC7BE019
:106A0000CE0101960E947DD0AF968FADAF978F706B
:106A10008450823008F0A5C067E1CE0183599F4FB2
:106A20000E949333A6962FAFA697A7963FAFA7973E
:106A3000A8964FAFA897A9965FAFA997AA966FAFF0
:106A4000AA97AB967FAFAB97AC968FAFAC97AD964E
:106A50009FAFAD9700E020E030E344E150E0BE019D
:106A60006F5B7F4FCE0183599F4F0E946B2066EB77
:106A70007BE087EE9AE00E94C48CBE016F5F7F4F7F
:106A800087EE9AE00E946D8C63EB7BE087EE9AE0E4
:106A90000E94C48CBE016F5B7F4F87EE9AE00E941C
:106AA0006D8C87EE9AE00E94F68A0E94E99C88230A
:106AB00029F08091AF07882309F45DC0B701A601D2
:106AC000C3010E94AB1B90E080E0CC58DF4F0FB6B3
:106AD000F894DEBF0FBECDBFDF91CF911F910F9114
:106AE000FF90EF90DF90CF90BF90AF908F907F900E
:106AF0006F905F904F903F902F90089562E47CE0FC
:106B0000BACE64E17CE087EE9AE00E94C48CE894FF
:106B1000D4F8B6CED4FE20CF66968FAD6697882384
:106B200009F41ACF482DBE016B5A7F4FCE01019652
:106B30000E94FEAC65E07CE087EE9AE00E94C48C87
:106B4000BE016F5F7F4F87EE9AE00E946D8C62E01E
:106B50007CE087EE9AE00E94C48CBE016B5A7F4FA6
:106B6000F3CE20E030E323282428252811F420E068
:106B700030E200E072CF482DBE016F5B7F4FCE0147
:106B800001960E94FEAC40E050E260E070E0C3017C
:106B90000E94821BD4FE97C0A114B10409F028C141
:106BA000AE96EFADAE97E150E63120F5F0E08827E4
:106BB000E352FA4C8F4F0C942ED8F036FA35FA3552
:106BC000FA35FA35F036FA35FA35FA35FA35FA3556
:106BD000FA35FA35F536ED36FA35FA35FA35F33554
:106BE000E436E736EA366CEE7CE0CE018B5A9F4FF6
:106BF0000E946DD030E020E043E050E060E4CE0140
:106C000001960E94462CD3011296ED91FC91608171
:106C100071814FE350E0CE0101960E949FDCA114E8
:106C2000B10469F063E774E0CE0101960E9479DC5B
:106C30004FE350E0B501CE0101960E949FDC63E76F
:106C400074E0CE0101960E9479DC4FE350E061ECE4
:106C50007BE0CE0101960E947DD06DEA7BE087EE5D
:106C60009AE00E94C48CBE016F5F7F4F87EE9AE06E
:106C70000E946D8C6AEA7BE087EE9AE00E94C48CE9
:106C8000BE016B5A7F4F87EE9AE00E946D8C87EEB3
:106C90009AE00E94F68A0E94E99C882309F40ECFAC
:106CA0008091AF0781110ACF482DBE016B5A7F4FEB
:106CB000CE0101960E94FEAC40E050E160E070E041
:106CC000C3010E94821BD6FE7CC040E051E060E020
:106CD00070E0C3010E94D41B672B682B692B09F459
:106CE00095C06CE97CE0CE018B5A9F4F0E946DD01D
:106CF00030E020E043E050E060E4CE0101960E94E5
:106D0000462CD3011296ED91FC91608171814FE385
:106D100050E0CE0101960E949FDCA114B10469F0FD
:106D200063E774E0CE0101960E9479DC4FE350E006
:106D3000B501CE0101960E949FDC63E774E0CE01AD
:106D400001960E9479DC4FE350E069EE7BE0CE01D2
:106D500001960E947DD064EA7BE087EE9AE00E9473
:106D6000C48CBE016F5F7F4F87EE9AE00E946D8CEE
:106D700061EA7BE087EE9AE00E94C48CBE016B5A08
:106D80007F4F87EE9AE00E946D8C87EE9AE00E941A
:106D9000F68A0E94E99C882309F490CE8091AF077F
:106DA00081118CCE482DBE016B5A7F4FCE010196CA
:106DB0000E94FEAC40E050E460E070E0C3010E943D
:106DC000821B81E090E081CE66EF7CE00ECF60E038
:106DD0007DE00BCF6AE07DE008CF64EC7CE005CF7E
:106DE000F3018285853009F005CF6AEB7CE0FDCEAA
:106DF00000E020E030E340E150E0BE016B5A7F4FFD
:106E0000CE0183599F4F0E946B20F4CE40E056E0A4
:106E100060E070E0C3010E94D41B611576408105DB
:106E2000910519F460EB7CE05ECF62E97CE05BCF1A
:106E3000DC011196EC911197EF70E150EB3008F006
:106E400039C0F0E08827E85DF84C8F4F0C942ED8BD
:106E50004B374B375A37333733373C375337533742
:106E600053373337333714966D917D918D919C91C3
:106E700017970E9460D6089514966D917D918D911B
:106E80009C91179724E630E040E050E00E94C5D77F
:106E9000CA01B901EECF14966C9170E090E080E0E9
:106EA0000E945ED6089514966D917D918D919C916E
:106EB0001797089560E070E0CB010895DC0111960A
:106EC000EC911197EF70E150EB3008F037C0F0E033
:106ED0008827E259F84C8F4F0C942ED88037803792
:106EE0009E37793779378F378637863786377937C0
:106EF000793714966D917D918D919C911797089596
:106F000014966C9170E090E080E0089514966D9175
:106F10007D918D919C9117970E942BD9089514967D
:106F20006D917D918D919C91179724E630E040E022
:106F300050E00E94C5D7CA01B901089560E070E031
:106F4000CB0108958F929F92AF92BF92CF92DF9222
:106F5000EF920F931F93CF93DF9300D000D01F9237
:106F60001F92CDB7DEB709831A832B833C834D83F1
:106F70005E836F837887DC0112962D913C912115F9
:106F80003105A1F490E080E028960FB6F894DEBFBA
:106F90000FBECDBFDF91CF911F910F91EF90DF908A
:106FA000CF90BF90AF909F908F9008958C01C901B2
:106FB0000E94EBA1C82ED12CB6E0CB16D104ACF4C4
:106FC0000E94FE92FC01892B19F08085807F8087CA
:106FD00080858F708087BF01F801828193810E9434
:106FE000CDA1FFEFCF1ADF0AE7CF65E0D8011296F7
:106FF0008D919C910E94439D6C01892B19F289818E
:10700000803108F0BFCFCE0101960E945E37161680
:1070100017061806190644F4F6018085982F9D700E
:1070200039F18F70873021F1D60118968C9118971D
:107030008F7018968C9367E078E087EE9AE00E9454
:10704000C48CD8011296ED91FC916081718187EE1C
:107050009AE00E946D8C6DEF77E087EE9AE00E94D7
:10706000C48C87EE9AE00E94F68A81E090E08CCF93
:107070000E9430AC4B015C01CE0101960E945E374C
:10708000860E971EA81EB91EF60181869286A386DB
:10709000B48682E0E11087E099819295907F892BF8
:1070A000D60118968C9360EF77E087EE9AE00E9405
:1070B000C48CD8011296ED91FC916081718187EEAC
:1070C0009AE00E946D8C6AEE77E087EE9AE00E946B
:1070D000C48CCE0101960E945E37AB01BC012AE050
:1070E00030E087EE9AE00E94E78B66EE77E0B5CF5E
:1070F000AF92BF92CF92EF92FF920F931F93CF93D5
:10710000DF93CDB7DEB7C856D1090FB6F894DEBF0E
:107110000FBECDBFA2960FAFA297A3961FAFA397A6
:10712000A4962FAFA497A5963FAFA597A6964FAF6D
:10713000A697A7965FAFA797A8966FAFA897A996AF
:107140007FAFA997970148E0FE01EF59FF4FDE019D
:10715000A75ABF4F01900D924A95E1F7A296EFAD65
:10716000A297E150ED3008F0F7C0EC2C5C01F0E0A4
:107170008827E254F74C8F4F0C942ED835393F397D
:107180009F39AA399539CB382C39AC39AC394839C3
:107190005A3981396D392130310531F4C5010E94E8
:1071A0006E1B009709F447C067E0CE01875A9F4FD6
:1071B0000E94933362ED77E087EE9AE00E94C48CE0
:1071C0006A966FAD6A9787EE9AE00E944BA167ECD2
:1071D00077E087EE9AE00E94C48CCE01875A9F4FD9
:1071E0000E945E37AB01BC012AE030E087EE9AE0F6
:1071F0000E94E78B87EE9AE00E94F68A6A960FADAE
:107200006A976B961FAD6B976C962FAD6C976D96CA
:107210003FAD6D976E964FAD6E976F965FAD6F9762
:10722000A0966FADA097A1967FADA197C5010E94D2
:10723000A23781E090E0C859DF4F0FB6F894DEBF67
:107240000FBECDBFDF91CF911F910F91FF90EF90B7
:10725000CF90BF90AF900895232B29F4C5010E94D1
:107260006E1B009741F366E0A0CF2130310529F471
:10727000C5010E946E1B0097F1F262E096CF232BAE
:1072800029F4C5010E946E1B0097A9F261E08DCF21
:1072900040E051E060E070E0C5010E94D41B672B24
:1072A000682B692B29F4C5010E946E1B009719F207
:1072B0006BE07BCF40E051E060E070E0C5010E94F0
:1072C000D41B672B682B692B31F0C5010E946E1B04
:1072D000009709F4B0CF6AE068CF40E056E060E084
:1072E00070E0C5010E94D41B6115764081059105AF
:1072F00031F4C5010E946E1B009709F49CCF6CE02D
:1073000054CF40E056E060E070E0C5010E94D41B1D
:10731000611576408105910531F0C5010E946E1B13
:10732000009709F488CF6DE040CF232B31F4C501DD
:107330000E946E1B009709F47ECF63E036CF2130A8
:10734000310531F4C5010E946E1B009709F473CF1B
:1073500065E02BCF64E029CF90E080E06CCFCF9345
:10736000DF93EC016115710539F48F8181708F8392
:1073700081E0DF91CF9108958981982F9F7029F145
:1073800080E09430B0F79B01770F440B550B2959DF
:10739000310941095109A4E6B0E00E94E4D72BE588
:1073A00031E040E050E00E94C5D737FF02C030E036
:1073B00020E02536310514F024E630E02F5F220F5F
:1073C0008F818170282B2F83D3CF807F8260898328
:1073D000DACF2F923F924F925F926F927F928F926D
:1073E0009F92AF92BF92CF92DF92EF92FF920F9354
:1073F0001F93CF93DF93CDB7DEB766970FB6F894A0
:10740000DEBF0FBECDBF6C0109871A872B873C8773
:107410004D875E876F87788B22E1E216F10480F555
:10742000F701ED5DFC4F8081898BCE0109960E94AA
:107430003C1697FD04C0BC01C6010E94AF398B8584
:10744000D60112968C93129789858C931196EC91A4
:107450001197EF70EC3008F06CC0F0E08827EC5C1E
:10746000F54C8F4F0C942ED8863B5D3A5D3ACB3B62
:10747000423A4F3C993BD43BD43BD43B993B993B5C
:10748000198AD3CF10E09A859F709D3008F002C40E
:10749000E92FF0E08827E05BF54C8F4F0C942ED855
:1074A000993A863CA63C863C513C513C863C863C05
:1074B0004A3E4A3E863C863C613B9A859F709D30A1
:1074C00008F00FC1E92FF0E08827E659F54C8F4FFF
:1074D0000C942ED8993A3F3B323B8F3A7A3A773A1E
:1074E000163B413B713B713B003B003B613B888954
:1074F000F60187838F85D60116968C9316978E8515
:1075000015968C9315978D8514968C9314971196D8
:107510008C911197807F892B11968C930AC08F854F
:107520009889F6018683878190FB80F987838E8511
:107530008583F989FF2309F460C0D60111968C91E7
:107540008F702F2F30E08217130609F456C06CEFAE
:107550007DE087EE9AE00E94C48CF60161816F7035
:1075600087EE9AE00E944BA169EF7DE087EE9AE0FA
:107570000E94C48C698987EE9AE00E944BA167EF54
:107580007DE087EE9AE00E94C48CD6010C911982AE
:107590001A821B821C821D821E821F821886898984
:1075A0008F709A81907F892B8A830983EE24EA94D5
:1075B000FE2C11961C91119712962C9112971396EE
:1075C0003C91139714964C91149715965C911597CE
:1075D00016966C91169717967C91CE0101960E9493
:1075E000E939F601208331834283538364837583B1
:1075F00086839783C6010E94293388E0F6015FC124
:107600008D859E85AF85B889B7FD0EC08F3F9105EA
:10761000A105B10529F024F08FEF90E0A0E0B0E0E3
:10762000D60114968C9385CF80E0FACF6D857E8548
:107630008F85988920E06D39BFEF7B078B079B070B
:107640006CF02FEF6115E4E67E078105910534F4B7
:1076500024E630E040E050E00E94C5D7D601149601
:107660002C9367CF8F859889F6018683878190FB5D
:1076700080F987838E8585838D8584835ACF8D8518
:10768000CFCF8D849E84AF84B88820E030E0A901FC
:10769000C501B4010E9459D660E087FD0FC020E00B
:1076A00030E04FE753E4C501B4010E9461D96FEFA8
:1076B000181624F0C501B4010E9432D9F601648382
:1076C00038CFD60111968C911197807F8C601196DE
:1076D0008C9311978D859E8515969C938E93149708
:1076E00028CF69E87EE087EE9AE00E94C48C6A8524
:1076F0006F7087EE9AE00E944BA166E87EE087EE0D
:107700009AE00E94C48CF6016181BFC09A859F7087
:1077100011968C911197807F892B11968C938D8572
:107720009E85AF85B889F60184839583A683B78348
:1077300000CF9A859F70933081F09C3011F24D8577
:107740005E856F857889F6014483558366837783E8
:107750008181807F892B8183ECCEC6010E94529D5E
:10776000D60114968C9314978F85988916968C93CE
:10777000169717968C91179790FB80F917968C9314
:1077800017978E8515968C93159711968C91119756
:10779000807F8260C1CECE0109960E94529DD601A3
:1077A00014968C931497F1CF9A859F709D3008F0B2
:1077B00057C0E92FF0E08827EF51F44C8F4F0C941D
:1077C0002ED8993AFB3B283CAD3B283C283CEE3B6D
:1077D0001A3C1A3C1A3C093C153C613B8D859E8540
:1077E000AF85B889F60184839583A683B7838181A9
:1077F000807F8660B0CF6D8570E090E080E00E9471
:107800005ED6D60114966D937D938D939C931797B6
:1078100090CE6D857E858F8598890E9460D6F60111
:10782000648375838683978384CE6D857E858F85FB
:107830009889E5CFF6018181807F982B91838D8592
:107840009E85AF85B88984839583A683B78371CEDF
:1078500011968C911197807F982B11969C935FCFF6
:1078600064E77EE087EE9AE00E94C48C6A856F70C0
:1078700087EE9AE00E944BA161E77EE087EE9AE0F6
:107880000E94C48CD60111966C916F7087EE9AE0BD
:107890000E944BA187EE9AE00E94F68A4ACE11E040
:1078A000F2CD4D855E856F857889F60144835583D9
:1078B000668377838181807F982B918388E0DE01C6
:1078C000119601900D928A95E1F729813A814B81B9
:1078D0005C816D817E818F81988566960FB6F89464
:1078E000DEBF0FBECDBFDF91CF911F910F91FF90F3
:1078F000EF90DF90CF90BF90AF909F908F907F9050
:107900006F905F904F903F902F900895963009F4BC
:10791000BFC048F46D85913071F06FEF70E0933027
:1079200051F060E008C0973009F4BEC09A506D85F0
:107930007E859230B0F784E68F8788898E7F888B2A
:107940001E868A85807F82608A876D872E8530E0DB
:10795000AFEFB0E00E94F7D7812C912C54018A94AC
:107960006115F4E67F078105910544F424E630E0D3
:1079700040E050E00E94C5D749015A01112309F4A3
:1079800073C02D852A8B022F10E028882694822D23
:107990008150990B1C019FEF2916390609F0A4C0EC
:1079A000A0E88A1691040CF086C08FE790E0881951
:1079B0009909809FD001819FB00D909FB00D112437
:1079C0002FEF30E00E9445D821E83EE740E050E04C
:1079D0000E94C5D7F6012783ABE9B0E0A501940169
:1079E0000E94E4D72FE7422E512C612C712CA30169
:1079F00092010E94C5D72C593F4F4F4F5F4F7901DD
:107A0000AEEFB1E0A50194010E94E4D7A301920179
:107A10000E94C5D7D8010E94E4D72FEF30E040E0A4
:107A200050E00E94C5D789012F3F310519F014F0AD
:107A30000FEF10E064E67EE087EE9AE00E94C48CCF
:107A4000B70187EE9AE00E9452A166E57EE087EEDC
:107A50009AE00E94C48CB80187EE9AE00E9452A17D
:107A600087EE9AE00E94F68A64E27EE087EE9AE072
:107A70000E94C48C87EE9AE00E94F68A6DE17EE057
:107A800087EE9AE00E94C48CC6010E94293351CD32
:107A90006D857E858F85988924E630E040E050E052
:107AA0000E94C5D7B90147CF6D857E858F8598899E
:107AB0000E942BD940CFA5019401205831094109DA
:107AC0005109ABE9B0E00E94E4D72FE730E040E095
:107AD00050E00E94C5D72C593F4F4F4F5F4F79015F
:107AE000D60117961C92A6CF9101AAEBBFEF0E9478
:107AF0003DD824E630E040E050E00E94C5D729019F
:107B00003A01B4E64B0E511C611C711C26E430E0B6
:107B1000D1010E9445D824E630E040E050E00E94C8
:107B2000C5D7DA01C9014E96A11DB11D8B8B9C8B67
:107B3000AD8BBE8B90E8891691040CF090C08FE756
:107B400090E088199909809FD001819FB00D909F86
:107B5000B00D11242B893C894D895E890E94EFD795
:107B60009B01AC01AFEFB0E00E94E4D724E63AE617
:107B700040E050E00E94C5D7D60117962C93A5018E
:107B80009401240D351D461D571DAEEFB1E00E9436
:107B9000E4D723EE30E040E050E00E94C5D7790101
:107BA0008A011901AFEFB0E0A50194010E94E4D76A
:107BB0002FE730E040E050E00E94C5D75901EA8944
:107BC000AE2FB0E0A80197010E94E4D72FEF30E07C
:107BD00040E050E00E94C5D789012F3F310519F0E0
:107BE00014F00FEF10E060E57EE087EE9AE00E946F
:107BF000C48C2AE030E0B301A20187EE9AE00E9433
:107C0000E78B6AE47EE087EE9AE00E94C48C2AE06B
:107C100030E04B895C896D897E8987EE9AE00E940D
:107C2000E78B62E47EE087EE9AE00E94C48CB501A7
:107C300087EE9AE00E9452A16AE37EE087EE9AE026
:107C40000E94C48CB80187EE9AE00E9452A161E3C1
:107C50007EE087EE9AE00E94C48CB101FDCEA501C2
:107C600094012058310941095109ABE9B0E00E9463
:107C7000E4D72FE730E040E050E00E94C5D72C5910
:107C80003F4F4F4F5F4F5901D60117961C92312C31
:107C9000212CA9CF6BE07EE087EE9AE00E94C48C95
:107CA0006A856F7087EE9AE00E944BA168E07EE0E3
:107CB00026CDFC019181892F8F7021F0823029F02F
:107CC00080E00895907F926091839B0177FF02C0CE
:107CD00030E020E02E3681E0380714F02DE631E068
:107CE0002683878130FB80F9878381E008950F9395
:107CF0001F93CF93DF93EC01088119816FE270E04D
:107D0000C8010E94CCDC009749F0FC011192CF0120
:107D1000DF91CF911F910F910C947C1DC8010E949F
:107D20007C1D009711F019821882DF91CF911F916D
:107D30000F910895DC011296ED91FC91309729F096
:107D400090859F7081E0953009F080E00895CF9292
:107D5000DF92FF920F931F93CF93DF93F12C611566
:107D6000710509F48DC06A01EB018C01CB010E9401
:107D70009A3EF82E882309F483C0D6FE0EC0D8019F
:107D80008C918B3009F450C008F041C040E051E0C4
:107D900060E070E08A3009F450C0D4FE09C0F801F8
:107DA000608186EF860F843018F0CE010E94F81BA8
:107DB000D5FE66C0D80114964D915D916D917C9170
:107DC000179711968C918F70873030F08930C8F1F9
:107DD0008A50823008F45DC0CE010E945D16EE81AB
:107DE000FF81309709F44CC080858F709EEF980F0B
:107DF000923010F0811144C0D80111968C91982FC7
:107E00009295907F80858F70892B808739C08C30C8
:107E100081F040E056E060E070E08D3009F0BDCFC9
:107E2000CE010E94AB1BB9CF40E051E060E070E0B2
:107E3000F7CF40E056E060E070E0CE010E94821B88
:107E4000ACCFEE81FF813097D9F080858F709EEFA7
:107E5000980F923010F0811113C0418752876387C9
:107E60007487EE81FF818085807F83608087EE81CB
:107E7000FF818085982F907F8F708067903629F2E0
:107E80008F2DDF91CF911F910F91FF90DF90CF90B9
:107E90000895CE010E945D16F3CF8F929F92AF920C
:107EA000BF92CF92DF92FF920F931F93CF93DF93F6
:107EB000EC018A819B810E94EBA1082F10E0043025
:107EC00011059CF40E94FE92FC01892B19F080851B
:107ED000807F808780858F708087BF018A819B81AA
:107EE0000E94CDA10F5F1F4FEACFEA81FB8106817F
:107EF00017810115110531F0D80112968D919C91D1
:107F00009D838C83EC81FD81309721F08281938168
:107F10009F838E83EE81FF81309749F00280F38149
:107F2000E02D309721F08281938199878887011510
:107F3000110541F0F80180858F70843059F128F4E3
:107F4000823071F0FF24FA940CC0853001F1863044
:107F5000C9F761EA74E0C8010E94CB9C8C01E7CFAD
:107F6000F184FA86CE010E949A3E811138C010E059
:107F700000E01C870B87DF91CF911F910F91FF903D
:107F8000DF90CF90BF90AF909F908F900895068123
:107F90001781CDCFC184D284C114D10499F2F601E6
:107FA0008081882379F298E2892E9DE0992EB12C68
:107FB000A12CFA2CC4010E9474D0AC01B401C601FA
:107FC0000E948DD0892BB9F1FFEFAF1ABF0A89E06B
:107FD000880E911CA7E1AA16B10459F7B3CFCE01C0
:107FE0000E94AFA18C010097B1F0FC0182819381C6
:107FF000892B39F08F2D0E94AFA28C01892B09F4B7
:10800000B6CFD801ED91FC910684F785E02DBE0135
:10801000C8011995AECF8F2D0E94AFA28C01892B7C
:1080200009F4A5CFEA85F0E0EE0FFF1FEA5DF44FFB
:1080300011830083E6CFC6010E944C918A2D90E007
:10804000B0E0A0E0F80181879287A387B48780859C
:10805000807F8260808785CFAF92BF92CF92DF9280
:10806000EF92FF920F931F93CF93DF93CDB7DEB7BD
:1080700065970FB6F894DEBF0FBECDBF8C017B01B4
:108080005A01FC0151834083148613861586168E8F
:10809000158E672B09F479C0452B09F476C06FE281
:1080A00070E0C7010E9484DC6C01892B09F465C073
:1080B000F701DE01119690E080E0BD0121912223BD
:1080C00041F02F3231F08431910519F02D93019652
:1080D000F5CF860F971FFC011082C5010E94CB9C33
:1080E000F80193838283FFEFCF1ADF0AD601F801EC
:1080F0003D9630E020E0CF01BD014D91442349F091
:108100004F3239F02F30310521F041932F5F3F4F2F
:10811000F3CFF801E20FF31F1586FB0140814F32C8
:1081200019F52F5F3F4FC601820F931F0E947C1DE0
:10813000F801968F858FC8010E949A3E882319F016
:10814000C8010E944D3F65960FB6F894DEBF0FBE82
:10815000CDBFDF91CF911F910F91FF90EF90DF90F6
:10816000CF90BF90AF9008950E947C1DF801968F2C
:10817000858F892B01F31586DECFB701C5010E94DB
:10818000CB9CF80193838283D6CFF80113821282AD
:10819000D2CFCF92DF92EF92FF920F931F93CF93A4
:1081A000DF93EC016A017B0188859985892BF1F4C5
:1081B0008A819B810E94EBA1082F10E005301105F8
:1081C000ACF40E94FE92FC01892B19F08085807F1F
:1081D000808780858F708087F987E887BF018A81D3
:1081E0009B810E94CDA10F5F1F4FE8CFE885F985E5
:1081F000309781F08085982F9F7051F4807F826046
:108200008087E885F985C186D286E386F48602C038
:108210009230B9F3DF91CF911F910F91FF90EF90C2
:10822000DF90CF900895FC0180859185009799F0AB
:10823000FC0120852F70223029F4618572858385A9
:1082400094850895253039F460E00E94439D00979D
:1082500011F0FC01F2CF60E070E0CB010895CF9205
:10826000EF92FF920F931F93CF93DF9300D000D034
:108270001F921F92CDB7DEB77C0109831A832B832F
:108280003C834D835E836F83788767E67AE187EE70
:108290009AE00E94C48CCE0101960E942933898104
:1082A00081112BC00B81013081F128F010E00230E8
:1082B000E9F5CC20F9F0CE0101960E94529DF7011C
:1082C00002811381892B81F0C8010E941341672B21
:1082D000682B692B79F44FEF5FEFBA0180E00E94C1
:1082E000C329AB01BC0103C040E050E0BA01C801A2
:1082F0000E94C94081E090E02AC08031B0F58E3004
:10830000B8F58130A9F18230B9F16AE57AE187EEFA
:108310009AE00E94C48C698187EE9AE00E944BA18A
:1083200087EE9AE00E94F68A01E010E06AE47AE1C2
:1083300087EE9AE00E94C48CB80187EE9AE00E9412
:1083400052A187EE9AE00E94F68A90E080E028969B
:108350000FB6F894DEBF0FBECDBFDF91CF911F9156
:108360000F91FF90EF90CF9008958351843068F67D
:10837000F70102811381A8CF40E050E0BA01F70174
:1083800082819381B5CF63E0FC01828193810E9459
:10839000439D009719F0FC01818508958FEF0895A2
:1083A000FF920F931F93CF93DF93CDB7DEB7C455E2
:1083B000D1090FB6F894DEBF0FBECDBF8C01F62EEB
:1083C000DC0116966C91FF2011F081E06827F8011E
:1083D00084810E945EAAF80187819085A185B2857B
:1083E000883E9340A105B10508F49BC069ED7AE190
:1083F00087EE9AE00E94C48C64ED7AE187EE9AE001
:108400000E94C48CD80114966D917C9187EE9AE0FD
:108410000E9452A16FEC7AE187EE9AE00E94C48C30
:108420006F2D70E087EE9AE00E9452A187EE9AE0ED
:108430000E94F68AFE01E55BFF4F8FE290E0819398
:10844000919388E0DF011D928A95E9F768EC7AE163
:10845000CE01855B9F4F0E9459D0F80182819381A4
:108460000E94C341FF2009F469C060EC7AE18531C4
:1084700051F069EB7AE1863131F06DEA7AE18F30C3
:1084800011F465EB7AE1CE018F5B9F4F0E946DD0B6
:108490008091B4079091B507059709F442C0D801BF
:1084A0001296ED91FC910280F381E02D0081118103
:1084B00001151105B1F140E450E0B801CE0101967B
:1084C0000E94BDDC6FE270E0CE0101960E9484DC68
:1084D000892B41F4980143E050E060E4CE0101961D
:1084E0000E94462C4FE350E0BE01655B7F4FCE01FA
:1084F00001960E949FDC0E94E99C882391F0809164
:10850000B4079091B507069761F48091AF07811188
:1085100008C041E0BE016F5B7F4FCE0101960E9413
:10852000FEACCC5ADF4F0FB6F894DEBF0FBECDBF06
:10853000DF91CF911F910F91FF90089569EA7AE141
:10854000823009F4A0CF64EA7AE19DCFAF92BF9266
:10855000CF92EF92FF920F931F93CF93DF9300D0B0
:1085600000D01F921F92CDB7DEB75C0109831A833A
:108570002B833C834D835E836F8378876EE17BE141
:1085800087EE9AE00E94C48CCE0101960E942933A6
:10859000E114F10439F067E17BE1C7010E9464D086
:1085A000009749F1F501028113810115110509F1C7
:1085B0008981811161C08B81813009F465C068F1C6
:1085C000823049F1082F10E064EF7AE187EE9AE0FB
:1085D0000E94C48C64EE7AE187EE9AE00E94C48C1B
:1085E000B80187EE9AE00E9452A187EE9AE00E94BD
:1085F000F68A90E080E028960FB6F894DEBF0FBEB2
:10860000CDBFDF91CF911F910F91FF90EF90CF9051
:10861000BF90AF900895CC20D1F0CE0101960E947A
:10862000529D892B09F44DC0C8010E941341672B4C
:10863000682B692BF1F44FEF5FEFBA0180E00E94E5
:10864000C329AB01BC01C8010E94C94012C0C801C6
:108650000E94C3418E3019F048F4813051F4CE01AC
:1086600001960E94529D892B21F0DECF83518430E8
:10867000B0F381E090E0BFCF8031F0F48E30A0F60F
:10868000813091F28230E9F06CE07BE187EE9AE094
:108690000E94C48C6FEF7AE187EE9AE00E94C48C4E
:1086A000698187EE9AE00E944BA187EE9AE00E94D2
:1086B000F68A01E010E088CF8351843008F4B4CF0B
:1086C000E3CF40E050E0BA01C8010E94C94060E039
:1086D000C5010E94D041CDCFDC01ED91FC91048415
:1086E000F585E02D62E0199581E090E00895CF9244
:1086F000DF92EF92FF920F931F93CF93DF93611559
:10870000710509F454C06A017B01EC01CB010E94A0
:108710009A3E082F882351F1D70116968D919C918E
:108720000097C9F1FC011085212F2F703EEF320F09
:10873000323010F0211124C012951F70D4FE04C0F5
:10874000C7010E94C3418883112339F18981807F49
:10875000182B1983D7011696ED91FC91818592858E
:10876000A385B4858C839D83AE83BF83802FDF91E7
:10877000CF911F910F91FF90EF90DF90CF900895D0
:10878000253049F460E00E94439D009721F0DC0110
:1087900018961C91D1CF10E0D1CFD7011696ED914C
:1087A000FC9180858F70823021F0833079F000E079
:1087B000DDCF41855285638574858981807F8A609C
:1087C00089834C835D836E837F83D0CF41855285BF
:1087D000638574858981807F876089834C835D830D
:1087E0006E837F83C3CF6F927F928F92AF92BF923F
:1087F000CF92DF92EF92FF920F931F93CF93DF936D
:1088000000D000D01F921F92CDB7DEB73C016A01A5
:108810007B01590140FF03C0E894C0F8D3F8D3FCB2
:108820000DC00E944B2D663971058105910530F010
:108830008091B4079091B507059729F5B701A60176
:108840004427507766277727C3010E94AB1B60E956
:108850007BE087EE9AE00E94C48C8FEF9FEF289612
:108860000FB6F894DEBF0FBECDBFDF91CF911F9141
:108870000F91FF90EF90DF90CF90BF90AF908F90CF
:108880007F906F90089519821A821B821C821D822C
:108890001E821F8218868A81807F8A8340E050E38F
:1088A000B301CE0101960E94774340E050E760E0BB
:1088B00070E0C3010E94D41BC62AD72AE82AF92AED
:1088C0008824839409811A812B813C814D815E81AA
:1088D0006F817885C3010E94B533C1CF8F929F927B
:1088E000AF92BF92CF92DF92EF92FF920F931F93BE
:1088F000CF93DF9300D000D01F921F92CDB7DEB789
:108900006D7F6130710509F4B7C0FC01E280F3802E
:10891000E114F10409F4B0C08C01C7010E941341B5
:108920004B015C0161E070E0C7010E94DA1F811415
:108930009104A104B10409F49FC020E030E04AE7AB
:1089400054E40E94BFD60E9432D96B017C01C1144D
:10895000D104E104F10409F48FC00E9430AC68191D
:1089600079098A099B096C157D058E059F0508F418
:1089700083C0F801A280B38070E060E0C5010E946E
:10898000DA1F20E030E048EC52E40E94BFD60E949B
:1089900032D96B017C014FEF5FEFBA0180E00E949A
:1089A000C329AB01BC01C5010E94C94019821A82CA
:1089B0001B821C821D821E821F8218868A81807FF4
:1089C0008A83F8016281738140E050E3CE01019611
:1089D0000E947743CE0101960E94F1154B015C0184
:1089E00066EA74E087EE9AE00E946D8CB501A401FE
:1089F00087EE9AE00E9448A165EB74E087EE9AE06A
:108A00000E946D8CB701A60187EE9AE00E9448A1F2
:108A100087EE9AE00E94F68AC80CD91CEA1CFB1C5F
:108A20008A81807F86608A83CD82DE82EF82F886AB
:108A3000F8016281738140E050E2CE0101960E940C
:108A4000A73E69EB74E087EE9AE00E946D8CB70157
:108A5000A60187EE9AE00E9448A187EE9AE00E9464
:108A6000F68A30E020E040E050E260E070E0F8019B
:108A7000828193810E94F34390E080E028960FB6B4
:108A8000F894DEBF0FBECDBFDF91CF911F910F9144
:108A9000FF90EF90DF90CF90BF90AF909F908F901E
:108AA00008950F931F93CF93DF9300D000D01F92B0
:108AB0001F92CDB7DEB719821A821B821C821D82DB
:108AC0001E821F8218862A81207F2A83FC01028150
:108AD0001381C8010E94C341813041F020F08230EF
:108AE00011F0853081F490E080E002C081E090E0F8
:108AF00028960FB6F894DEBF0FBECDBFDF91CF91A1
:108B00001F910F91089540E050E2B801CE01019607
:108B10000E947743CE0101960E94529DE9CF0F93A8
:108B20001F93CF93DF93DC011B960D911C910115D0
:108B3000110519F1EC010E94AFA10097F1F0D801E5
:108B4000ED91FC91DC0112968D919C91C817D9078B
:108B500059F40684F785E02D70E060E0C801DF91EC
:108B6000CF911F910F9119940280F381E02DC801DC
:108B7000DF91CF911F910F911994DF91CF911F91A8
:108B80000F9108958F929F92AF92BF92CF92DF92F2
:108B9000EF92FF920F931F93CF93DF93CDB7DEB782
:108BA000CF55D1090FB6F894DEBF0FBECDBF8C01F3
:108BB0006B016115710519F04115510579F56FE2E9
:108BC00070E187EE9AE00E94C48C66E270E187EE65
:108BD0009AE00E94C48CB80187EE9AE00E946D8CE6
:108BE00064E270E187EE9AE00E94C48C87EE9AE01E
:108BF0000E94F68AC15ADF4F0FB6F894DEBF0FBE4F
:108C0000CDBFDF91CF911F910F91FF90EF90DF903B
:108C1000CF90BF90AF909F908F900895460F571FB1
:108C2000DA011C920E944B2D4B016EE170E187EE40
:108C30009AE00E94C48CB40187EE9AE00E9452A18F
:108C40006BE170E187EE9AE00E94C48CB80187EE78
:108C50009AE00E946D8C68E170E187EE9AE00E94D4
:108C6000C48CBAE38B16B1E09B064CF46BE070E168
:108C700080E49AE00E94C48C80E49AE0B9CF69E075
:108C800070E187EE9AE00E94C48CB60187EE9AE00C
:108C90000E946D8C67E070E187EE9AE00E94C48CC0
:108CA00087EE9AE00E94F68A1A821982FE013396B4
:108CB0008EE3DF011D928A95E9F78091B4079091C8
:108CC000B507059791F563E070E0C8010E94DA2CC2
:108CD0007C01892BD1F5E091B909F091BA09808125
:108CE00080FF88CF61E070E0C8010E94DA2C892BF8
:108CF00009F480CF64E270E0C8010E94CCDC892BCB
:108D000009F078CF69EE7FE087EE9AE00E94C48C8C
:108D1000B80187EE9AE00E946D8C87EE9AE00E947F
:108D2000F68AC8010E94C8A865CF61E070E0C8015A
:108D30000E94DA2C7C01892B09F465C04FE350E0D6
:108D4000B801CE0101960E94BDDCA12CBB24B394D6
:108D5000E00EF11E60EE7FE0C7010E9464D0892B17
:108D600009F45EC064E270E0C8010E94CCDC892B8B
:108D700009F040CFB11003C0AA2009F43BCF4091C5
:108D8000B6075091B707B701CE018F5B9F4F0E9486
:108D90002C40CE018F5B9F4F0E949A3E182F882354
:108DA00059F0B601CE018F5B9F4F0E9415A411E0D0
:108DB000181619060CF010E0CE018F5B9F4F0E9431
:108DC0008F45112309F416CF8981882309F412CF26
:108DD0008091B4079091B507059709F40BCF62EC29
:108DE0007FE087EE9AE00E94C48CBE016F5F7F4FE8
:108DF00087EE9AE00E946D8C87EE9AE00E94F68AD8
:108E0000CE0101968FCF62E070E0C8010E94DA2C9B
:108E10007C01892B09F4EECEAA24A394B12C98CF1F
:108E2000F60101900020E9F73197EC19FD0932971E
:108E300008F498CFC8010E94C8A8B11003C0AA20A6
:108E400009F4D8CEC6010E949590D4CECF93DF937B
:108E5000EC01598348837B836A831C861B861D86AD
:108E60001E8E1D8E0E949A3E882329F0CE01DF912E
:108E7000CF910C944D3FDF91CF9108952F923F9267
:108E80004F925F926F927F928F929F92AF92BF921A
:108E9000CF92DF92EF92FF920F931F93CF93DF93C6
:108EA000CDB7DEB7A4970FB6F894DEBF0FBECDBF27
:108EB000FC016115710509F4D0C0DB0118969C9185
:108EC0009F70953009F0C9C0EBA20AA319013A01BD
:108ED000F9A3E8A3FB01468057808091B0078F5F1C
:108EE0008093B007FE2DF160FCA34114510409F4F6
:108EF000AFC0D20118968C918F70843049F018F071
:108F0000873008F491C0D20112964D905C90EDCF5D
:108F1000F20161857285A8A1B9A18D919C910E94F1
:108F2000CB9C4C01009779F3FC0180858F708530D4
:108F300051F74091B6075091B707B401CE010196A1
:108F40000E9426476114710419F1CE0101960E9416
:108F50009A3E8823E9F0AAA0CCA07101D3010C911C
:108F600011961C91119712962C91129713963C9181
:108F7000139714964C91149715965C911597169625
:108F80006C91169717967C91CE0101960E946E4ABD
:108F90008B858730A9F561E0C4010E94439DEBA059
:108FA0000AA19101A301BC0188A199A10E943E4799
:108FB00061147104A1F5882391F18091B00781506B
:108FC0008093B007CE0101960E948F4581E0A49660
:108FD0000FB6F894DEBF0FBECDBFDF91CF911F91CA
:108FE0000F91FF90EF90DF90CF90BF90AF909F9048
:108FF0008F907F906F905F904F903F902F9008954B
:109000006114710461F4CE0101960E949A3E882396
:1090100031F0CE0101960E942F48892B71F6CE01C6
:1090200001960E948F456FCF912C812CB12CA12CE1
:10903000D12CC12CF301E080F180028113812481C5
:109040003581468157816FEFC2010E94735C5BCF0F
:109050008091B00781508093B00780E0B8CFCF9265
:10906000DF92EF92FF920F931F93CF93DF9300D085
:1090700000D01F921F92CDB7DEB76C0119821A8201
:109080001B821C821D821E821F8218868A81807F1D
:109090008A8362E47BE087EE9AE00E94C48CD6016A
:1090A0001296ED91FC916081718187EE9AE00E94A9
:1090B0006D8C60E47BE087EE9AE00E94C48CC60170
:1090C0000E949A3E81111CC067E37BE087EE9AE024
:1090D0000E94C48C87EE9AE00E94F68A0FEF1FEF81
:1090E000C80128960FB6F894DEBF0FBECDBFDF9142
:1090F000CF911F910F91FF90EF90DF90CF90089547
:10910000C6010E94C341F82EF6018385948500971D
:1091100091F0DC01ED91FC910288F389E02D199525
:109120008C0197FD08C081E00115110509F480E06C
:109130000E945D1CD5CFF6018285873009F431C0CD
:10914000EFEFEF0DE63108F02CC0F0E08827E45592
:10915000F74B8F4F0C942ED8C248CB48D148D148FA
:10916000CB48C248D148D148D148D148D148D1484C
:10917000D148C248D148D148D148D148C248C24854
:10918000C248C24868E17BE087EE9AE00E94C48C46
:1091900001E010E0A5CF80E00E945D1C10E000E03F
:1091A0009FCF40E050E2B601CE0101960E94774386
:1091B000D6011A968C911A97873071F160F483303A
:1091C00009F456C0843061F068E27BE087EE9AE0F3
:1091D0000E94C48CE3CF883009F44AC08930A1F7DB
:1091E000CE0101960E94529D8C016DE17BE087EEDD
:1091F0009AE00E94C48CB80187EE9AE00E9452A1C6
:1092000087EE9AE00E94F68A91E080E0012B09F453
:1092100090E0092F182F64CF1496ED91FC91808572
:109220008F7010E000E0853001F765E37BE087EEAA
:109230009AE00E94C48CF60164817581E12C00E003
:1092400030E020E050E040E0C6010E943E47F82EAA
:10925000082F10E062E37BE087EE9AE00E94C48C66
:109260008F2D0E945D1C87EE9AE00E94F68A38CF0F
:10927000CE0101960E945E378B01B7CF4F925F926D
:109280006F927F928F929F92AF92BF92CF92DF9216
:10929000FF920F931F93CF93DF9300D000D01F92C4
:1092A0001F92CDB7DEB76130710509F481C0FC01B2
:1092B000628173816115710509F47AC08C0119828C
:1092C0001A821B821C821D821E821F8218868A813E
:1092D000807F8A8340E050E2CE0101960E9477436E
:1092E000CE0101960E94529D6C01F801828193810A
:1092F0000E9413412B013C01F801278130854185F3
:109300005285D6010E94EFD72FEF30E040E050E0C9
:109310000E94A3D749015A010E9430ACFF24F39464
:1093200081149104A104B10461F0641975098609DE
:109330009709FF24F394681579058A059B0508F4BD
:10934000F12C411451046104710491F1F8018780FA
:109350009084A184B2840E9430ACF80181149104FD
:10936000A104B10451F064197509860997096815BB
:1093700079058A059B0508F449C0A280B3804FEFA8
:109380005FEFBA0180E00E94C329AB01BC01C501B7
:109390000E94C940CD2861F0F80184810E948F1499
:1093A000F8019681891304C061E0C8010E94D04190
:1093B00090E080E028960FB6F894DEBF0FBECDBFD8
:1093C000DF91CF911F910F91FF90DF90CF90BF90D1
:1093D000AF909F908F907F906F905F904F90089587
:1093E000FF20D9F060E0C8010E94D041F8018281DD
:1093F00093810E942F48892BD9F640E050E0BA01B2
:10940000F801828193810E94C940D2CF84810E9459
:109410008F14F80196818913E3CFCD2849F2F80122
:1094200084810E948F14F80196818913C1CFF110B5
:10943000BFCFBACFCF93DF93EC016CE77AE187EE31
:109440009AE00E94C48C67E77AE187EE9AE00E9476
:10945000C48C6C817D8187EE9AE00E9452A161E705
:109460007AE187EE9AE00E94C48C87EE9AE00E942F
:10947000F68A61E08C810E948CAA6E818C810E94A8
:109480005EAA8A819B81009729F040E050E0BA01F2
:109490000E94C940E881F9810484F585E02D62E0ED
:1094A000CE0119958A819B81009799F00E942F48DF
:1094B0001816190674F40A80DB81C02D4FEF5FEF98
:1094C000BA0180E00E94C329AB01BC01CE010E9419
:1094D000C94081E090E0DF91CF9108952F923F92B3
:1094E0004F925F926F927F928F929F92AF92BF92B4
:1094F000CF92DF92EF92FF920F931F93CF93DF9360
:10950000CDB7DEB7C95DD1090FB6F894DEBF0FBE87
:10951000CDBF1C01C754DF4F0883C95BD040C65480
:10952000DF4F1883CA5BD040C554DF4F2883CB5B25
:10953000D040C454DF4F3883CC5BD040C354DF4F9E
:109540004883CD5BD040C254DF4F5883CE5BD040C0
:10955000C154DF4F6883CF5BD040C054DF4F788366
:10956000C05CD040CF53DF4FF982E882C15CD0406D
:10957000CD52DF4FC882C35DD040C053DF4FA882B9
:10958000C05DD0400E944B2D6B01CC52DF4F7983E0
:109590006883C45DD040683C71059CF46FEF7AE04D
:1095A00080E49AE00E94C48CB60180E49AE00E94B4
:1095B00052A180E49AE00E94F68A2FEF3FEF0C94CC
:1095C0006F550E9430ACCA52DF4F688379838A831B
:1095D0009B83C65DD040C554DF4F8881CB5BD040B4
:1095E000A82FB0E0C553DF4FB983A883CB5CD04030
:1095F000E091B407F091B507CF52DF4FF983E883CC
:10960000C15DD040CF53DF4FE881F981C15CD040CC
:10961000309721F0808181110C94135AD1011D964D
:109620008C91882341F0C1010D96CF53DF4F998370
:109630008883C15CD040C553DF4FE881F981CB5CA2
:10964000D040EF2B11F00C946F5ACF53DF4FE881CD
:10965000F981C15CD040309711F00C941C5AD101B3
:109660005D960D90BC91A02DC553DF4FB983A883A3
:10967000CB5CD040AB2B11F40C946F5AC554DF4F28
:109680008881CB5BD04081110C946F5AC553DF4F5A
:109690006881CB5CD040CE0187549F4F0E947133CC
:1096A000CF55DF4F2883C15AD040CE55DF4F388386
:1096B000C25AD040CD55DF4F4883C35AD040CC5515
:1096C000DF4F5883C45AD040CB55DF4F6883C55A0B
:1096D000D040CA55DF4F7883C65AD040C955DF4FB6
:1096E0008883C75AD040C855DF4F9883C85AD040A6
:1096F0000C946F5AD10112968D919C91892B09F48B
:109700005CCFC553DF4FE881F981CB5CD040319706
:10971000A1F4C654DF4F8881CA5BD0408F70F1E05E
:10972000C153DF4FF883CF5CD040811128C0C153B3
:10973000DF4F1882CF5CD04022C0C553DF4F088175
:109740001981CB5CD040012B09F044C0C754DF4FD6
:109750008881C95BD040882309F44EC0885082308C
:1097600008F44AC0C153DF4F1882CF5CD04081E07B
:1097700090E0C553DF4F99838883CB5CD040C754BA
:10978000DF4F1881C95BD040112309F45DC040E070
:1097900052E060E070E0C1010E94D41B672B682B8F
:1097A000692B09F451C01C3009F44EC06CEB7AE00F
:1097B00080E49AE00E94C48C80E49AE00E94F68AD9
:1097C000AAEFBFEFC953DF4FB983A883C75CD0406E
:1097D0000C94C85AC553DF4F28813981CB5CD040E7
:1097E0002430310509F4A3CF2930310509F49FCF86
:1097F0002330310509F469C0C654DF4F8881CA5B44
:10980000D0408F7009F461C040E054E060E070E047
:10981000C1010E94D41B672B682B692B09F455C02A
:1098200067EA7AE080E49AE00E94C48C80E49AE0DF
:109830000E94F68AEAEFFFEFC953DF4FF983E8830E
:10984000C75CD0400C94C85AC553DF4F08811981BA
:10985000CB5CD04004301105E9F5C053DF4FE88000
:10986000C05DD040C754DF4F0881C95BD040C654AB
:10987000DF4F1881CA5BD040C554DF4F2881CB5BD6
:10988000D040C454DF4F3881CC5BD040C354DF4F4D
:109890004881CD5BD040C254DF4F5881CE5BD04071
:1098A000C154DF4F6881CF5BD040C054DF4F788117
:1098B000C05CD040C1010E94A237C953DF4F9983D9
:1098C0008883C75CD0400C94C85AC153DF4F1882BC
:1098D000CF5CD040CD52DF4F1881C35DD0401330F4
:1098E00091F4D1011A968C91873069F469E87AE095
:1098F00087EE9AE00E94C48C87EE9AE00E94F68A76
:10990000E9EFFFEF99CF88E0FE01E754FF4FDE015A
:10991000AF54BF4F01900D928A95E1F7E114F10425
:1099200009F451C068E37CE0C7010E9464D0892B30
:1099300009F450C062E47CE0C7010E9464D0892B26
:1099400009F451C060E67CE0C7010E9464D0892B15
:1099500009F452C06AE67CE0C7010E9464D0892BFA
:1099600009F453C066EF7CE0C7010E9464D0892BE4
:1099700009F454C060E07DE0C7010E9464D0892BE7
:1099800009F46CC06AEB7CE0C7010E9464D0892BAB
:1099900009F467C064EC7CE0C7010E9464D0892BA5
:1099A00009F462C06AE07DE0C7010E9464D0892B9F
:1099B00009F45DC06CEE7CE0C7010E9464D003E155
:1099C00010E0892B69F1C353DF4F19821882CD5CF7
:1099D000D0402CC021E030E0C353DF4F39832883CF
:1099E000CD5CD04023C082E090E0C353DF4F998329
:1099F0008883CD5CD0401AC0A5E0B0E0C353DF4FF0
:109A0000B983A883CD5CD04011C0E6E0F0E0C35339
:109A1000DF4FF983E883CD5CD04008C004E110E05B
:109A2000C353DF4F19830883CD5CD040C754DF4F49
:109A30001881C95BD040143009F42BC3D8F411232A
:109A400009F47FC0412C512C32010FEF1FEFC95395
:109A5000DF4F19830883C75CD040B5C325E130E0F0
:109A6000BBCF8EE090E0C1CFAFE0B0E0C7CFE6E182
:109A7000F0E0CDCF88EF810F823020F788E0FE0143
:109A8000E754FF4FDE01119601900D928A95E1F7A0
:109A9000C654DF4F8881CA5BD0408F7009F4AAC3D7
:109AA000CE0187549F4F0E94F1156B017C01C114B8
:109AB000D104E104F10409F49DC3193041F4F09498
:109AC000E094D094C094C11CD11CE11CF11CB101E4
:109AD000CE0187549F4F0E941DA260E0CE018754A3
:109AE0009F4F0E949333A2962FAFA297A3963FAFAA
:109AF000A397A4964FAFA497A5965FAFA597A696F8
:109B00006FAFA697A7967FAFA797A8968FAFA89796
:109B1000A9969FAFA997C553DF4FA881B981CB5CA8
:109B2000D040AA30B10509F442C50CF069C31097C2
:109B300009F404C4129709F4C0C3412C512C32011A
:109B400094C519821A821B821C821D821E821F826A
:109B500018868A81807F8A83C654DF4F8881CA5BDA
:109B6000D0408F7009F489C2C553DF4F0881198135
:109B7000CB5CD0400A30110509F432C25CF4011507
:109B8000110579F10230110509F4C3C0412C512CA3
:109B900032011DC2C553DF4F28813981CB5CD040D3
:109BA0002B30310509F4B5C12C30310579F7B101FD
:109BB000CE0101960E941DA2CE0187549F4F0E94A4
:109BC0003C16BC01CE0101960E94AF3988E0FE012F
:109BD0003196DE01A754BF4F01900D928A95E1F7AF
:109BE000F1C1EF2859F064E77AE087EE9AE00E942D
:109BF000C48C87EE9AE00E94F68AC8CFC1010E9409
:109C00002F481816190614F00C94FD59CE018754EC
:109C10009F4F0E945E37672B682B692B09F06FC13D
:109C200062E0CE0187549F4F0E949333C756DF4FA7
:109C30002883C959D040C656DF4F3883CA59D0400F
:109C4000C556DF4F4883CB59D040C456DF4F5883A9
:109C5000CC59D040C356DF4F6883CD59D040C2564F
:109C6000DF4F7883CE59D040C156DF4F8883CF591C
:109C7000D040C056DF4F9883C05AD040442443940C
:109C800030E1532E612C712C31E0CD53DF4F3883FE
:109C9000C35CD040AA24A39446C061E0CE0187549F
:109CA0009F4F0E949333CF56DF4F2883C159D04036
:109CB000CE56DF4F3883C259D040CD56DF4F488350
:109CC000C359D040CC56DF4F5883C459D040CB56EF
:109CD000DF4F6883C559D040CA56DF4F7883C659D5
:109CE000D040C956DF4F8883C759D040C856DF4F90
:109CF0009883C859D0404424439420E1522E612CCB
:109D0000712C81E0CD53DF4F8883C35CD040A12C00
:109D10000AC0412C512C3201CD53DF4F1882C35C55
:109D2000D040AA24AA94B101CE0101960E941DA29E
:109D30008A819CE0980F9F70923058F4C654DF4F90
:109D40009881CA5BD0409F70923019F4807F826006
:109D50008A83D1011A969C91973069F4C654DF4FDB
:109D60008881CA5BD0408F708250843020F48A8111
:109D7000807F82608A83F101A385B485892F90E07A
:109D8000109741F0ED91FC911197008CF18DE02D31
:109D9000CD0119957C01C754DF4F0881C95BD040C4
:109DA000C654DF4F1881CA5BD040C554DF4F2881AD
:109DB000CB5BD040C454DF4F3881CC5BD040C35420
:109DC000DF4F4881CD5BD040C254DF4F5881CE5B1E
:109DD000D040C154DF4F6881CF5BD040C054DF4FCB
:109DE0007881C05CD040CE0101960E94E939C75706
:109DF000DF4F2883C958D040C657DF4F3883CA5831
:109E0000D040C557DF4F4883CB58D040C457DF4FB1
:109E10005883CC58D040C357DF4F6883CD58D040CB
:109E2000C257DF4F7883CE58D040C157DF4F888369
:109E3000CF58D040C057DF4F9883C059D040CE0193
:109E400001960E942933CD53DF4FF881C35CD04087
:109E5000FF2341F1C654DF4F8881CA5BD0408F7029
:109E60009FE0980F9F70923020F08A5F8F70823051
:109E7000C8F48A818F7081508230A0F42D8130E047
:109E8000AFEFB0E00E94F7D72FEF611504E670073F
:109E90008105910534F424E630E040E050E00E9472
:109EA000C5D72D8388E0FE013196DE01A754BF4F50
:109EB00001900D928A95E1F718E2512AB12C2FEF0B
:109EC0003FEFC953DF4F39832883C75CD040D101AE
:109ED0001A968C911A97873009F0A0C5CC52DF4FA3
:109EE000E881F981C45DD040EE35F1400CF03DC40D
:109EF00064E27AE080E49AE00E94C48C5ACB412C60
:109F0000512C320191E0CD53DF4F9883C35CD04098
:109F1000C1CEB101CE0101960E941DA2C254DF4FF5
:109F20009881CE5BD0408A81282F2F7041F022305B
:109F300049F0412C512C3201BB24B39449C0807F9D
:109F400082608A83892F90E08536910514F084E63B
:109F500090E08E8388E0FE013196DE01A754BF4F6A
:109F600001900D928A95E1F762E0CE0187549F4FF0
:109F70000E947133CF57DF4F2883C158D040CE574E
:109F8000DF4F3883C258D040CD57DF4F4883C35886
:109F9000D040CC57DF4F5883C458D040CB57DF4F09
:109FA0006883C558D040CA57DF4F7883C658D04021
:109FB000C957DF4F8883C758D040C857DF4F9883B1
:109FC000C858D040412C98E2592E612C712CB12CEC
:109FD000CD53DF4F1882C35CD040AA24AA946FCF20
:109FE000B101CE0101960E941DA2C154DF4F6881CC
:109FF000CF5BD040C054DF4F7881C05CD0407170DF
:10A00000CE0101960E94593ECD53DF4F8883C35C39
:10A01000D040412C512C3201BB24B3948823E9F267
:10A0200088E0FE013196DE01A754BF4F01900D92EA
:10A030008A95E1F762E0CE0187549F4F0E94713309
:10A04000EA962FAFEA97EB963FAFEB97EC964FAFC0
:10A05000EC97ED965FAFED97EE966FAFEE97EF96BC
:10A060007FAFEF97C158DF4F8883CF57D040C0589C
:10A07000DF4F9883C058D040A5CF412C512C3201DE
:10A080008FEF9FEFC953DF4F99838883C75CD04020
:10A090009AC0C553DF4FA881B981CB5CD0401997D6
:10A0A00009F471C0C1010E942F4818161906B4F5B1
:10A0B00062E0CE0187549F4F0E949333E2962FAF08
:10A0C000E297E3963FAFE397E4964FAFE497E596C8
:10A0D0005FAFE597E6966FAFE697E7967FAFE797B6
:10A0E000E8968FAFE897E9969FAFE99744244394A9
:10A0F00080E1582E612C712CEFEFFFEFC953DF4F39
:10A10000F983E883C75CD040B12CF1E0CD53DF4F39
:10A11000F883C35CD040AA24A394D9CE61E0CE01D9
:10A1200087549F4F0E949333AA962FAFAA97AB965E
:10A130003FAFAB97AC964FAFAC97AD965FAFAD97D7
:10A14000AE966FAFAE97AF967FAFAF97E0968FAFFB
:10A15000E097E1969FAFE1974424439400E1502EAD
:10A16000612C712C0FEF1FEFC953DF4F1983088348
:10A17000C75CD040B12C11E0CD53DF4F1883C35CD6
:10A18000D040A12CA4CE40E051E060E070E0C101DD
:10A190000E94D41B672B682B692BE1F040E051E053
:10A1A00060E070E0C1010E94821B4424439410E4EB
:10A1B000512E612C712C21E030E0C953DF4F3983DF
:10A1C0002883C75CD040B12CCD53DF4F1882C35CCD
:10A1D000D040EAC140E051E060E070E0C1010E947F
:10A1E000AB1B44244394B0E45B2E612C712C81E0C2
:10A1F00090E048CFA5E0CA2ED12CE12CF12C5DCC0B
:10A20000C553DF4FE881F981CB5CD040EB30F105DD
:10A2100009F44CC23C9709F090CCC654DF4F8881BA
:10A22000CA5BD0408F70823009F092C2C701B6017C
:10A2300024E630E040E050E00E94C5D7C054DF4F34
:10A240008881C05CD040869590E0280F391F121697
:10A25000130614F021E030E02536310514F024E631
:10A2600030E0220FC054DF4F8881C05CD040817045
:10A27000282BC054DF4F2883C05CD04062E0CE0161
:10A2800087549F4F0E9471332A962FAF2A972B969F
:10A290003FAF2B972C964FAF2C972D965FAF2D97F6
:10A2A0002E966FAF2E972F967FAF2F9760968FAF1A
:10A2B000609761969FAF6197D3C1CD53DF4F1882EE
:10A2C000C35CD040D1011B968D919C911C97009747
:10A2D00009F03BC01A968C9190E0E0E58E2E912C0F
:10A2E000A12CB12C8530910549F0812C912C540181
:10A2F000449721F0812C912C54018A943E01B9EBB2
:10A300006B0E711CD3011196EC911197EF70E15017
:10A31000EB3008F034C1F0E023018827ED56FE4A07
:10A320008F4F0C942ED8AD51AD51BF52BF52BF527A
:10A330009052525252525252E151E151F1E0CD53FA
:10A34000DF4FF883C35CD040BDCFDC01ED91FC91C1
:10A35000008CF18DE02D1995C0CFF3011481C70158
:10A36000B60124E630E040E050E00E94C5D7DA01B3
:10A37000C901810F911DA11DB11DB7FF03C080E070
:10A3800090E0DC018F3F9105A105B10529F024F093
:10A390008FEF90E0A0E0B0E0C354DF4F8883CD5B47
:10A3A000D0406EEC74E087EE9AE00E946D8CC201A2
:10A3B0000E942933412C78E2572E612C712CB12C4C
:10A3C000EBC014960D911D912D913C911797C95397
:10A3D000DF4F088319832A833B83C75CD040B4E6F0
:10A3E000CB16D104E104F10484F5A4E6B0E0A901A0
:10A3F00098010E94E4D7C60ED71EE81EF91E8114EC
:10A400009104A104B104B9F0A50194010E94E4D71C
:10A41000362F272FB701A60177FF03C040E050E099
:10A42000BA01C32ED22E7C014C155D056E057F0549
:10A4300014F46A017B01F301C482D582E682F782BB
:10A440008181807F86608183ACCFC701B60124E61D
:10A4500030E040E050E00E94C5D7C953DF4F88810B
:10A460009981AA81BB81C75CD040280F391F4A1F40
:10A470005B1F81149104A104B10461F057FF03C074
:10A4800020E030E0A90182169306A406B50614F474
:10A49000A5019401D20114962D933D934D935C93A5
:10A4A00017977FCFF30164817581868197810E9420
:10A4B0002BD9C953DF4F688379838A839B83C75C19
:10A4C000D040C701B60124E630E040E050E00E94F1
:10A4D000C5D7C953DF4F688179818A819B81C75C69
:10A4E000D040620F731F841F951F81149104A10433
:10A4F000B10461F097FF03C060E070E0CB01861605
:10A500009706A806B90614F4C501B4010E9460D6E6
:10A51000D30114966D937D938D939C93179741CFA0
:10A52000F30184819581A681B781C80ED91EEA1EE8
:10A53000FB1E81149104A104B104C9F0A4E6B0E0AB
:10A54000A50194010E94E4D7362F272FB701A60159
:10A5500077FF03C040E050E0BA01C32ED22E7C0149
:10A560004C155D056E057F0514F46A017B01D3016E
:10A570001496CD92DD92ED92FC92179712CF88E05F
:10A58000FE013196D30101900D928A95E1F7412C9D
:10A59000512C3201BB24B394EFEFFFEFC953DF4FCF
:10A5A000F983E883C75CD040AA24AA9490CCC6540F
:10A5B000DF4F8881CA5BD0408F70823009F057C06E
:10A5C000C701B60124E630E040E050E00E94C5D764
:10A5D000C154DF4F8881CF5BD040C054DF4F6881CA
:10A5E000C05CD040962F9170280F391F2E36B1E0F5
:10A5F0003B072CF437FF05C02DE631E002C030E008
:10A6000020E0C154DF4F2883CF5BD040C054DF4FE0
:10A610008881C05CD04030FB80F9C054DF4F888314
:10A62000C05CD04062E0CE0187549F4F0E947133DE
:10A630006A962FAF6A976B963FAF6B976C964FAF4A
:10A640006C976D965FAF6D976E966FAF6E976F96C6
:10A650007FAF6F97A0968FAFA097A1969FAFA1975E
:10A66000412C68E2562E612C712CB12C19C088E067
:10A67000FE013196DE01A754BF4F01900D928A95DD
:10A68000E1F768E67AE080E49AE00E94C48C80E416
:10A690009AE00E94F68A412C512C3201BB24B394DB
:10A6A000CD53DF4F1882C35CD04076CFC654DF4F06
:10A6B0008881CA5BD0408F708230E9F5C701B6014E
:10A6C00024E630E040E050E00E94C5D7C254DF4F9E
:10A6D0008881CE5BD04090E0280F391F37FF02C041
:10A6E00030E020E02536310514F024E630E0C25495
:10A6F000DF4F2883CE5BD04062E0CE0187549F4F6E
:10A700000E94713362962FAF629763963FAF639753
:10A7100064964FAF649765965FAF659766966FAF27
:10A72000669767967FAF679768968FAF68976996C9
:10A730009FAF699795CF88E0FE013196DE01A7545F
:10A74000BF4F01900D928A95E1F76CE57AE09BCFBF
:10A7500088E0FE013196DE01A754BF4F01900D92B3
:10A760008A95E1F760E57AE08ECFCD52DF4F3881F0
:10A77000C35DD04030FD77C01496ED91FC9180858B
:10A780008F70853009F06FC0CF52DF4FE881F981BB
:10A79000C15DD040359709F466C0C553DF4F0881CD
:10A7A0001981CB5CD0400130110509F0B6C7C75400
:10A7B000DF4F8881C95BD0408A50823008F008C7DB
:10A7C0006CE07AE087EE9AE00E94C48CD101129688
:10A7D000ED91FC916081718187EE9AE00E946D8C11
:10A7E00087EE9AE00E94F68AC754DF4F8881C95BE2
:10A7F000D0408A3071F08B30C1F030E020E040E092
:10A8000050E460E070E0C1010E94F34301E010E019
:10A81000B9C640E051E060E070E0C1010E94821BD7
:10A820006AE0C1010E94F81BE8CFC053DF4FB88136
:10A83000C05DD040B1110EC063EF79E080E49AE0D2
:10A840000E94C48C80E49AE00E94F68AEBEFFFEF4E
:10A850000C941C4C40E051E060E070E0C1010E94AB
:10A86000AB1B6BE0DECF10E0C353DF4F2881398193
:10A87000CD5CD040232B09F441C7CF53DF4F198261
:10A880001882C15CD0403AC7863009F454C787307B
:10A8900009F041C7C1010E94C341082F863009F069
:10A8A00062C067EC79E087EE9AE00E94C48C66E0B3
:10A8B00070E087EE9AE00E9452A187EE9AE00E9433
:10A8C000F68A62E0CE0187549F4F0E94933329AFEE
:10A8D0003AAF4BAF5CAF6DAF7EAF8FAF21969FAFFE
:10A8E00021973DC0C1010E94C341853021F083E022
:10A8F00090E00C945D4C6EED79E087EE9AE00E945A
:10A90000C48C65E070E087EE9AE00E9452A187EE69
:10A910009AE00E94F68AB101CE0187549F4F0E94AF
:10A920001DA261E0CE0187549F4F0E94933322966F
:10A930002FAF229723963FAF239724964FAF2497AC
:10A9400025965FAF259726966FAF269727967FAF00
:10A95000279728968FAF289729969FAF29976894B5
:10A9600040F854F8D8C669EA79E087EE9AE00E9488
:10A97000C48C602F70E087EE9AE00E9452A187EEAF
:10A980009AE00E94F68AA3E0B0E00C94E24BAA2081
:10A9900009F4E7C66FE879E087EE9AE00E94C48C7C
:10A9A000E3E0F0E00C941C4C6AE779E087EE9AE073
:10A9B0000E94C48C03E010E0E5C52FEFA2120DC089
:10A9C000C1010E942F48181619064CF06DE579E078
:10A9D00087EE9AE00E94C48C8ACFAA20B9F362E085
:10A9E000CE0187549F4F0E94933329A73AA74BA7C4
:10A9F0005CA76DA77EA78FA798AB689440F854F822
:10AA000035E0932EC7C640E050E2B101CE01875435
:10AA10009F4F0E9477438111DCC6DDC6BFEFAB12AA
:10AA200065C0C1010E942F48AA24A39418161906D4
:10AA30000CF45FC0A12C6FE479E087EE9AE00E94ED
:10AA4000C48CEA2C0A2C000CFF08B70187EE9AE0B0
:10AA50000E9452A168E479E087EE9AE00E94C48CDB
:10AA6000CD53DF4FF881C35CD0406F2F70E087EE8D
:10AA70009AE00E9452A187EE9AE00E94F68ACF5394
:10AA8000DF4F88809980C15CD04081149104F1F13E
:10AA9000C1010E94C341C82ED12CC114D10409F4B4
:10AAA0006701C353DF4F08811981CD5CD040011588
:10AAB000110509F453C0C016D10611F16CE279E01A
:10AAC00087EE9AE00E94C48CB60187EE9AE00E945D
:10AAD00052A187EE9AE00E94F68A2DEF3FEFC9530C
:10AAE000DF4F39832883C75CD04052C5AA2009F4C0
:10AAF000A2CFE1E0CD53DF4FE883C35CD0409BCFD2
:10AB0000CF53DF4F19821882C15CD040C754DF4F4A
:10AB10009880C95BD040B6E1B91508F4E5C1E92DCC
:10AB2000F0E08827E956FA4A8F4F0C942ED8F15559
:10AB30002A571B572D56F155FC56BE567556F155E2
:10AB4000F155705770578F578F574C574C57745754
:10AB5000745774574C574C574C574C57D1011B9650
:10AB60008D919C91009709F4D1CFDC01ED91FC917E
:10AB70000088F189E02DC053DF4FA880C05DD04030
:10AB8000CD53DF4FC880C35CD0407401C754DF4F42
:10AB90000881C95BD040C654DF4F1881CA5BD040E2
:10ABA000C554DF4F2881CB5BD040C454DF4F388180
:10ABB000CC5BD040C354DF4F4881CD5BD040C25402
:10ABC000DF4F5881CE5BD040C154DF4F6881CF5BEF
:10ABD000D040C054DF4F7881C05CD04019950C94B0
:10ABE0005D4C912CC153DF4F2881CF5CD040222394
:10ABF00009F404C6C053DF4FC880C05DD040CF54B5
:10AC0000DF4F0881C15BD040CE54DF4F1881C25B5B
:10AC1000D040CD54DF4F2881C35BD040CC54DF4FB0
:10AC20003881C45BD040CB54DF4F4881C55BD040F6
:10AC3000CA54DF4F5881C65BD040C954DF4F68818A
:10AC4000C75BD040C854DF4F7881C85BD040C1019A
:10AC50000E947838E89455F8D1C5C1010E94C341DB
:10AC6000853009F044CE67E179E087EE9AE00E94F2
:10AC7000C48C65E070E087EE9AE00E9452A187EEF6
:10AC80009AE00E94F68AB101CE0187549F4F0E943C
:10AC90001DA2F10182858530C9F46EE0CE01875492
:10ACA0009F4F0E94933329A33AA34BA35CA36DA3A8
:10ACB0007EA38FA398A7689440F854F8912CF1E0F4
:10ACC000CD53DF4FF883C35CD0408CCF61E0CE0121
:10ACD00087549F4F0E949333298F3A8F4B8F5C8FFD
:10ACE0006D8F7E8F8F8F98A3E6CFC1010E94C341E5
:10ACF000182F863081F560E079E087EE9AE00E94B7
:10AD0000C48C66E070E087EE9AE00E9452A187EE64
:10AD10009AE00E94F68A62E0CE0187549F4F0E941B
:10AD20009333298B3A8B4B8B5C8B6D8B7E8B8F8B0C
:10AD3000988F40E050E068E070E0C1010E94821B03
:10AD4000689440F854F8912C01E0CD53DF4F08830C
:10AD5000C35CD04047CF62EE78E087EE9AE00E9475
:10AD6000C48C612F70E087EE9AE00E9452A187EEBA
:10AD70009AE00E94F68A23E030E0B1CE40E051E054
:10AD800060E070E0C1010E94D41B672B682B692B27
:10AD900061F5A11027C0B101CE0187549F4F0E94D9
:10ADA0001DA261E0CE0187549F4F0E9493332987F3
:10ADB0003A874B875C876D877E878F87988B40E0CB
:10ADC00050E068E070E0C1010E94AB1B689440F85D
:10ADD00054F826E0922E31E0CD53DF4F3883C35C28
:10ADE000D04000CF68EC78E0F3CD63EB78E087EEFD
:10ADF0009AE00E94C48CC7CDAA20D1F062E0CE01B7
:10AE000087549F4F0E94933329833A834B835C83FB
:10AE10006D837E838F839887689440F854F895E01B
:10AE2000992EB1E0CD53DF4FB883C35CD040DACE6A
:10AE300066E978E0B1CDC554DF4F8881CB5BD04067
:10AE4000823008F073C0C1010E94C341853009F00F
:10AE500032CF4DCDC554DF4F8881CB5BD04082309F
:10AE600008F02CCFAA20C1F06DE778E087EE9AE0D9
:10AE70000E94C48C61E0C1010E94F81BCF53DF4FD8
:10AE800028813981C15CD04040E058E160E070E049
:10AE9000C1010E94F3438ECDC554DF4F8881CB5B47
:10AEA000D040823008F04FCF992009F447C0C654F3
:10AEB000DF4F8881CA5BD0408F7031F4B101CE0181
:10AEC00087549F4F0E941DA2689440F810E3512AB6
:10AED000912C21E0CD53DF4F2883C35CD04082CE3C
:10AEE000689456F8912C77CFC654DF4F8881CA5B9F
:10AEF000D0408F7051F4689454F8912C81E0CD5378
:10AF0000DF4F8883C35CD0406DCE90E3592A912CEB
:10AF1000A1E0CD53DF4FA883C35CD04063CE912C1A
:10AF2000412C80E4582E612C712C7BCF912CE1E0D8
:10AF3000CD53DF4FE883C35CD04054CE11E0CD53F6
:10AF4000DF4F1883C35CD0404DCEF10183859485DB
:10AF5000892B09F4CBC0411451046104710439F008
:10AF6000A201B101CE0187549F4F0E94A73ED1019B
:10AF70001B968D919C91CF53DF4FE880F980C15C87
:10AF8000D040DC01ED91FC910088F189E02DC053A7
:10AF9000DF4FA880C05DD040CD53DF4FC880C35C79
:10AFA000D040C754DF4F0881C95BD040C654DF4F43
:10AFB0001881CA5BD040C554DF4F2881CB5BD0409D
:10AFC000C454DF4F3881CC5BD040C354DF4F48813D
:10AFD000CD5BD040C254DF4F5881CE5BD040C154CE
:10AFE000DF4F6881CF5BD040C054DF4F7881C05CB9
:10AFF000D0401995C953DF4F99838883C75CD040EF
:10B00000F10183859485DC01ED91FC91008CF18D3B
:10B01000E02D1995059711F4689440F856FCC5C1C8
:10B02000992021F0692DC1010E94F81BCF52DF4FFA
:10B03000A881B981C15DD040159709F425C430E0DD
:10B0400020E0B301A201C1010E94F343C153DF4FCD
:10B05000B881CF5CD040BB2309F416C4CF53DF4F77
:10B0600088819981C15CD040892B09F40DC460E2CC
:10B0700078E087EE9AE00E94C48C87EE9AE00E9406
:10B08000F68ACF53DF4FA880B980C15CD040812CB5
:10B0900073016201CF54DF4F0881C15BD040CE54B1
:10B0A000DF4F1881C25BD040CD54DF4F2881C35B96
:10B0B000D040CC54DF4F3881C45BD040CB54DF4FFD
:10B0C0004881C55BD040CA54DF4F5881C65BD04031
:10B0D000C954DF4F6881C75BD040C854DF4F7881C7
:10B0E000C85BD040C1010E94B533CEC38285853094
:10B0F00009F484C0863009F093CFC754DF4FD8805D
:10B10000C95BD040DD2009F479C0C1010E94FBA1D8
:10B110007C01411451046104710439F0A201B101B0
:10B12000CE0187549F4F0E94A73EE114F10409F419
:10B1300077CF10E000E0F7FE05C0F194E194F1084C
:10B1400001E010E0C70101978634910508F068CF4F
:10B15000CE2C61E08E2D0E948CAAEFEFED0DE63132
:10B1600008F049C0F0E08827E754F74A8F4F0C9465
:10B170002ED8CF58D158FB58FB58D158CF58D1585A
:10B18000FB58FB58FB58FB58FB58FB58CF58CF587F
:10B19000FB58FB58FB58CF58FB58CF58CF58F1E01D
:10B1A0000F27602F8C2D0E945EAA68E578E087EE5D
:10B1B0009AE00E94C48CB70187EE9AE00E9452A1E7
:10B1C00066E578E087EE9AE00E94C48CB80187EECD
:10B1D0009AE00E9452A187EE9AE00E94F68A689453
:10B1E00040F854F801E010E0C953DF4F1983088399
:10B1F000C75CD04015CF0FEF1FEFD7CF41145104DC
:10B200006104710439F0A201B101CE0187549F4F4E
:10B210000E94A73EC553DF4F28813981CB5CD040C7
:10B220002230310509F4BDC02330310581F02130D1
:10B23000310509F0F5CE689440F854F821E030E08B
:10B24000C953DF4F39832883C75CD040E9CEC101A1
:10B250000E9413416B017C01892B61F566E478E063
:10B2600086E39AE00E94C48CD1011296ED91FC9184
:10B270006081718186E39AE00E946D8C6AED74E0D2
:10B2800086E39AE00E946D8C2AE030E0B701A601C7
:10B2900086E39AE00E94E78B86E39AE00E94F68AB2
:10B2A000D1011296ED91FC916081718180EE94E064
:10B2B0000E941CADCE0187549F4F0E94183720E09A
:10B2C00030E048EC52E40E94BFD60E942BD9C9530B
:10B2D000DF4F688379838A839B83C75CD040C953DF
:10B2E000DF4FC880D980C75CD0404FEF5FEF60E090
:10B2F00070E088E00E94C329CD53DF4F68837983D3
:10B300008A839B83C35CD040CD53DF4FE880F980B4
:10B31000C35CD0406FE378E087EE9AE00E94C48C73
:10B32000D1011296ED91FC916081718187EE9AE0D6
:10B330000E946D8C6BE378E087EE9AE00E94C48CEB
:10B34000C953DF4F68817981C75CD04087EE9AE0AE
:10B350000E9452A166E378E087EE9AE00E94C48CD6
:10B36000CD53DF4F488159816A817B81C35CD040D6
:10B37000662777272AE087EE9AE00E94AA8A87EE5E
:10B380009AE00E94F68AB701A601C1010E94C94055
:10B39000E1E0F0E0C953DF4FF983E883C75CD040B8
:10B3A0003FCE689440F855F81DCF81E090E0C95336
:10B3B000DF4F99838883C75CD04032CECF52DF4FB6
:10B3C000E881F981C15DD040359709F45DC240E064
:10B3D00050E4B101CE0187549F4F0E94A73E30E058
:10B3E00020E040E050E460E070E0C1010E94F343DF
:10B3F0004BC2ACEFBFEF0C94E24BCE0187549F4F92
:10B400000E945E372B013C01411451046104710418
:10B4100011F00C944D4EB1E0CD53DF4FB883C35CB7
:10B42000D0400C94874EC553DF4F08811981CB5C07
:10B43000D040012B09F053C08081882311F40C9473
:10B440002F4BCE018F539F4F0E94773EC553DF4F46
:10B4500099838883CB5CD040C554DF4F8881CB5B18
:10B46000D040811132C0C553DF4F6881CB5CD040E2
:10B47000CE0187549F4F0E947133C755DF4F2883F9
:10B48000C95AD040C655DF4F3883CA5AD040C55537
:10B49000DF4F4883CB5AD040C455DF4F5883CC5A36
:10B4A000D040C355DF4F6883CD5AD040C255DF4FDF
:10B4B0007883CE5AD040C155DF4F8883CF5AD040D1
:10B4C000C055DF4F9883C05BD040C553DF4FE88144
:10B4D000F981CB5CD040EF2B11F40C942F4B64EF2F
:10B4E0007AE087EE9AE00E94C48CB60187EE9AE07B
:10B4F0000E9452A16DEE7AE087EE9AE00E94C48C21
:10B50000D1011296ED91FC916081718187EE9AE0F4
:10B510000E946D8C67EE7AE087EE9AE00E94C48C00
:10B52000CF53DF4F68817981C15CD04087EE9AE0CC
:10B530000E946D8C65EE7AE087EE9AE00E94C48CE2
:10B54000CE0187549F4F0E942933CF53DF4FE880AD
:10B55000F980C15CD040E114F10411F40C947A4BF1
:10B56000F7018081843211F00C947A4B61ED7AE01E
:10B5700087EE9AE00E94C48C87EE9AE00E94F68AD9
:10B580000CEF1FEFC953DF4F19830883C75CD0400E
:10B59000C953DF4F88819981C75CD040C752DF4FC4
:10B5A0000FB6F894DEBF0FBECDBFDF91CF911F91D4
:10B5B0000F91FF90EF90DF90CF90BF90AF909F9052
:10B5C0008F907F906F905F904F903F902F90089555
:10B5D0001FEFA11212C0C1010E942F48AA24A394F8
:10B5E000181619060CF0A12CC553DF4F288139819C
:10B5F000CB5CD0402130310599F4C754DF4F8881AE
:10B60000C95BD040863061F440E051E060E070E01A
:10B61000C1010E94D41B672B682B692B09F081C0E4
:10B62000CF53DF4F28813981C15CD040D1011496BE
:10B630006D917C91CD52DF4FE880C35DD040C05307
:10B64000DF4F0881C05DD040AE0147545F4FC1015C
:10B650000E943E47C153DF4FB881CF5CD04010E01D
:10B66000BB23C1F1C053DF4FC880C05DD040EE2482
:10B67000EA94FE2CCF54DF4F0881C15BD040CE54FA
:10B68000DF4F1881C25BD040CD54DF4F2881C35BB0
:10B69000D040CC54DF4F3881C45BD040CB54DF4F17
:10B6A0004881C55BD040CA54DF4F5881C65BD0404B
:10B6B000C954DF4F6881C75BD040C854DF4F7881E1
:10B6C000C85BD040C1010E947838C153DF4F188158
:10B6D000CF5CD040CF53DF4F88819981C15CD0408F
:10B6E000892B09F4C1C8C353DF4FE881F981CD5CD0
:10B6F000D040EF2B09F0C1C8689440F8C754DF4F21
:10B700008881C95BD040853009F457C908F0BCC8AE
:10B71000833009F4E7C8912C3DC02FEFA21280CFEF
:10B720005ACFC353DF4F88819981CD5CD04010E060
:10B73000892B09F0A2C840E051E060E070E0C1014F
:10B740000E94D41B672B682B692B09F02DC9BFEF12
:10B75000AB121DC9C1010E942F48181619060CF41E
:10B7600019C9B101CE0187549F4F0E941DA261E00B
:10B77000CE0187549F4F0E94933329AB3AAB4BAB1A
:10B780005CAB6DAB7EAB8FAB98AF689440F854F870
:10B7900046E0942ED301C201689440F8C554DF4FAF
:10B7A0002881CB5BD040223060F4C754DF4F288122
:10B7B000C95BD040222329F02C013D01689440F858
:10B7C00054F8C654DF4F8881CA5BD0408F7009F4AB
:10B7D0001AC9689455F8112311F0E89455F8A2019C
:10B7E000B101CE0187549F4F0E94A73EA1E0B0E077
:10B7F000C953DF4FB983A883C75CD040B110F9CDDE
:10B80000D1011B968D919C91009709F49ECBDC0190
:10B81000ED91FC910488F589E02DC754DF4F088134
:10B82000C95BD040C654DF4F1881CA5BD040C554B5
:10B83000DF4F2881CB5BD040C454DF4F3881CC5BD5
:10B84000D040C354DF4F4881CD5BD040C254DF4F5E
:10B850005881CE5BD040C154DF4F6881CF5BD04070
:10B86000C054DF4F7881C05CD040199581116DCBF9
:10B870006DE578E080E49AE00E94C48C80E49AE070
:10B880000E94F68A56FC9ACD65E178E087EE9AE050
:10B890000E94C48CC953DF4F68817981C75CD04056
:10B8A00087EE9AE00E9452A16EE078E087EE9AE07F
:10B8B0000E94C48C0E9430ACAB01BC01CA52DF4F65
:10B8C000088119812A813B81C65DD040401B510B04
:10B8D000620B730B87EE9AE00E9448A187EE9AE014
:10B8E0000E94F68A55CE2F923F924F925F926F92AE
:10B8F0007F928F929F92AF92BF92CF92DF92EF9200
:10B90000FF920F931F93CF93DF93CDB7DEB7CB5743
:10B91000D1090FB6F894DEBF0FBECDBFE296EFAEF1
:10B92000E297E396FFAEE397E4960FAFE497E596D0
:10B930001FAFE597E6962FAFE697E7963FAFE797FD
:10B94000E8964FAFE897E9965FAFE997009709F45B
:10B9500053C024012B2CEC96AFAEEC97EB96DFAEE8
:10B96000EB97EA96CFAEEA97362E8C0180910102D2
:10B97000893020F4809100028930A0F180E091E0CC
:10B980000E942BCE7C01892B69F11C821B821E82B6
:10B990001D828FEF9FEF98878F838DE992E09A83C6
:10B9A00089831A861986FC86EB8680E091E0988B65
:10B9B0008F871E861D86B801CE0101960E94CCA2FB
:10B9C0006FEE74E087EE9AE00E946D8CB70187EE0F
:10B9D0009AE00E946D8C87EE9AE00E94F68AC70179
:10B9E0000E94C7CEF80180858F70843009F45FC152
:10B9F00028F4882309F464C180E02FC0853009F45D
:10BA000046C08630C9F767E374E0C8010E94CB9C4A
:10BA10003C01009709F476C0912C812CB12CA12C0B
:10BA2000D12CC12CE296EFACE297E396FFACE39702
:10BA3000E4960FADE497E5961FADE597E6962FAD3A
:10BA4000E697E7963FADE797E8964FADE897E9961A
:10BA50005FADE997632D0E94735CC558DF4F0FB649
:10BA6000F894DEBF0FBECDBFDF91CF911F910F9134
:10BA7000FF90EF90DF90CF90BF90AF909F908F900E
:10BA80007F906F905F904F903F902F90089580919E
:10BA9000B0078F5F8093B007668077806114710470
:10BAA00059F14201EC96AFACEC97B22CEA96CFACD0
:10BAB000EA97EB96DFACEB97E296EFACE297E39672
:10BAC000FFACE397E4960FADE497E5961FADE597DD
:10BAD000E6962FADE697E7963FADE797E8964FAD30
:10BAE000E897E9965FADE997632DC3010E94735C07
:10BAF000F30162807380D2CF8091B0078150809330
:10BB0000B0077ACF65EF74E0C8010E94CB9C2C018E
:10BB10006AEF74E0C8010E94CB9C7C016FEF74E077
:10BB2000C8010E94CB9C332039F0F1E03F1609F4A4
:10BB30009FC0D12CC12C0CC063E075E0C8010E94ED
:10BB4000CB9C3C0168E075E0C8010E94CB9C6C0175
:10BB50006114710409F43801C114D10409F46801B5
:10BB60004114510431F4EA964FACEA97EB965FAC7E
:10BB7000EB97E114F10421F4EC96EFACEC97F22C86
:10BB80006114710409F4A5C0F30180858F708430BD
:10BB900009F09FC061847284C114D10409F49CC06F
:10BBA000F60180858F70843009F096C0C184D284FC
:10BBB00010E000E04114510409F4F3C06114710471
:10BBC00009F4B1C06AE27CE187EE9AE00E94C48C7D
:10BBD000F2016185728587EE9AE00E946D8C65E2C4
:10BBE0007CE187EE9AE00E94C48CB30187EE9AE074
:10BBF0000E946D8C87EE9AE00E94F68ACE018F58E3
:10BC00009F4F0E942933E114F10409F0D3C0F201DF
:10BC100080858F70843009F083C14091B6075091C0
:10BC2000B70761857285CE0101960E942C40CE0136
:10BC300001960E949A3E8823B1F00E944B2D6B0121
:10BC4000683C71050CF083C064EE7BE180E49AE00F
:10BC50000E94C48CB60180E49AE00E9452A180E464
:10BC60009AE00E94F68ACE0101960E948F4558C143
:10BC70006DE075E0C8010E94CB9C3C0162E175E07B
:10BC8000C8010E94CB9C6C016114710409F04AC187
:10BC900063E075E0C8010E94CB9C3C01C114D10453
:10BCA00009F450CF892B09F05BCF380159CFD12C43
:10BCB000C12C712C612CF12CE12C512C412C48CF42
:10BCC000D12CC12C712C612CF12CE12C512C412C4C
:10BCD00047CF712C612C60CF00E020E030E340E1E1
:10BCE00050E0BE016F597F4FCE018F589F4F0E9489
:10BCF0006B206C01E4960FADE49710E0011511057F
:10BD000009F058CFE2968FADE297811109C0E39612
:10BD10008FADE3978F7009F44DCF02E010E04ACF6A
:10BD200001E010E047CF6BE17CE187EE9AE00E94F2
:10BD3000C48CF2016185728587EE9AE00E946D8C59
:10BD400066E17CE187EE9AE00E94C48C57CF6114D3
:10BD5000710431F0B301CE0101960E9415A483CF86
:10BD6000A12CC12CF12CE12CE2960FADE297E396C9
:10BD70001FADE397E4962FADE497E5963FADE597C9
:10BD8000E6964FADE697E7965FADE797E8966FAD1D
:10BD9000E897E9967FADE997CE0101960E946E4A39
:10BDA00062CFE114F10409F4BBC0C114D10409F459
:10BDB000B7C004C0C114D10409F429CFF7018085AC
:10BDC0008F70843009F0A8C08185928525961FAEBA
:10BDD0001EAE259748EE53E060E070E029964CAF28
:10BDE0005DAF6EAF7FAF299723EB32E023963FAF75
:10BDF0002EAF23972F969FAF8EAF2F9761961FAED2
:10BE00001EAE619763961FAE1EAE639765961FAE1A
:10BE10001EAE659767961FAE1EAE679769961FAFF9
:10BE20000EAF69976A961FAE6A9740E450E0BE0174
:10BE30006F5F7F4FCE018F5B9F4F0E94719E21E00D
:10BE400030E02C0F3D1F820F931FFC0110826EE02B
:10BE50007CE187EE9AE00E94C48CF70161857285CF
:10BE600087EE9AE00E946D8C67E175E087EE9AE0BC
:10BE70000E946D8CBE016F5F7F4F87EE9AE00E943B
:10BE80006D8C69E07CE187EE9AE00E94C48CB6017B
:10BE900087EE9AE00E946D8C87EE9AE00E94F68A07
:10BEA0000E94E99C8823C1F18091AF07811134C0C1
:10BEB0006FE270E0CE0101960E9484DC892B51F480
:10BEC000F7012185328543E050E060E4CE01019620
:10BED0000E94462C62E07CE187EE9AE00E94C48CCE
:10BEE000BE016F5F7F4F87EE9AE00E946D8C6DEF11
:10BEF0007BE187EE9AE00E94C48CB60187EE9AE05F
:10BF00000E946D8C87EE9AE00E94F68A41E0B601AD
:10BF1000CE0101960E94FEAC4114510409F077CE87
:10BF200081E09BCD892B09F01BCE0CCE2F923F9246
:10BF30004F925F926F927F928F929F92AF92BF9239
:10BF4000CF92DF92EF92FF920F931F93CF93DF93E5
:10BF5000CDB7DEB767970FB6F894DEBF0FBECDBF83
:10BF60001C017C8B6B8B40E050E860E070E00E942D
:10BF7000D41B672B682B692B09F45DC019821A82C8
:10BF80001B821C821D821E821F8218868A81807FEE
:10BF90008A8340E050E3B101CE0101960E947743CD
:10BFA000D1011B968D919C91892B09F444C040E0EE
:10BFB00050E860E070E0C1010E94821B6AE57BE00E
:10BFC00087EE9AE00E94C48CF10183859485DC01A0
:10BFD000ED91FC910088F189E02DA12CCC24C39433
:10BFE000F12CE12C09811A812B813C814D815E81EC
:10BFF0006F81788519958F3F9807E9F0D1011296E6
:10C00000ED91FC9160817181892B09F0C5C087EEAB
:10C010009AE00E946D8C68E57BE087EE9AE00E94D2
:10C02000C48C60E57BE087EE9AE00E94C48C87EECA
:10C030009AE00E94F68A65E0F101828193810E9474
:10C04000439D9A8B898B009709F4DAC0DC0118961E
:10C05000BC91BD8B9B2E92943FE09322FC014184C6
:10C060005284638474840E9430AC992009F4C8C05F
:10C07000461A570A680A790A19861A861B861C8688
:10C0800099861A85107F1A601A874D865E866F869C
:10C09000788A8B899C89049769F588248394B12CCC
:10C0A000A12CC12CD12C20E1E22EF12C092D2B85C5
:10C0B0003C854D855E856F857889C1010E94B533C9
:10C0C000C301B20128EE33E040E050E00E94C5D742
:10C0D000BA01A9012AE030E087EE9AE00E94E78BDE
:10C0E00061E87BE087EE9AE00E94C48C87EE9AE0DC
:10C0F0000E94F68A77FE84C092E0491651046104DA
:10C1000090E879060CF47CC00E944B2D2B017F8BAC
:10C110006E8B88248394B12CA12CC12CD12C90E15E
:10C12000E92EF12C09851A852B853C854D855E8588
:10C130006F857889C1010E94B533AE89BF89A83C5B
:10C14000B105BCF568E67BE080E49AE00E94C48C0F
:10C15000B20180E49AE00E9452A180E49AE00E9439
:10C16000F68A8FEF9FEF67960FB6F894DEBF0FBE8B
:10C17000CDBFDF91CF911F910F91FF90EF90DF9096
:10C18000CF90BF90AF909F908F907F906F905F9077
:10C190004F903F902F90089587EE9AE00E946D8C0B
:10C1A0006EE47BE087EE9AE00E94C48C6AE47BE058
:10C1B0003ACFE989FA8980858F70808719821A823F
:10C1C0001B821C821D821E821F8218868A81807FAC
:10C1D0008A8399828D898F70AA24A394873009F06D
:10C1E000A12C82E0C82EF12CE12C09811A812B812F
:10C1F0003C814D815E816F817885C1010E946E4ACC
:10C200008B899C89019701F540E050E360E070E084
:10C21000C1010E94D41BAB01BC0141155105610550
:10C22000710591F08091B4079091B507069761F47C
:10C2300030E020E0C1010E94F34340E050E360E0C1
:10C2400070E0C1010E94821BD1011B968D919C91CF
:10C25000009719F490E080E086CFDC01ED91FC912D
:10C260000284F385E02D1995892BA1F3F1018385D3
:10C270009485DC01ED91FC910480F581E02D6B89C2
:10C280007C89199570CF6F927F928F929F92AF9217
:10C29000BF92CF92DF92EF92FF920F931F93CF93B3
:10C2A000DF93CDB7DEB7C854D1090FB6F894DEBF1F
:10C2B0000FBECDBF3C014B01FC010081118165EF38
:10C2C00074E0C8010E94CB9C5C016AEF74E0C80175
:10C2D0000E94CB9C6C016FEF74E0C8010E94CB9C64
:10C2E000A114B10431F4C114D10419F4892B09F457
:10C2F000CEC06AE175E0C8010E94CB9C7C016FE171
:10C3000075E0C8010E94CB9C8C016CEB77E087EE56
:10C310009AE00E94C48CF301638187EE9AE00E9448
:10C320004BA16AEB77E087EE9AE00E94C48CB401DF
:10C3300087EE9AE00E9452A187EE9AE00E94F68A68
:10C34000C114D10409F455C0F60180858F70843082
:10C3500009F04FC06185728540E450E0CE0101963E
:10C360000E94BDDC0E94E99C882309F442C08091B0
:10C37000AF0781113EC06FE270E0CE0101960E94CE
:10C3800084DC892B51F4F6012185328543E050E0AD
:10C3900060E4CE0101960E94462C8114910409F4B8
:10C3A000B5C0E114F10409F088C041E064E275E031
:10C3B000CE0101960E94FEAC64EB77E087EE9AE036
:10C3C0000E94C48CBE016F5F7F4F87EE9AE00E948F
:10C3D0006D8C61EB77E087EE9AE00E94C48C64E29A
:10C3E00075E087EE9AE00E946D8C87EE9AE00E94DD
:10C3F000F68AA114B10409F44AC0F50180858F7052
:10C40000843009F044C04091B6075091B707618568
:10C410007285CE0101960E942C40CE0101960E94A9
:10C420009A3E882381F1892809F4B7C0F701EF28E3
:10C4300009F0CCC025961CAE1DAE1EAE1FAE2597D2
:10C4400029961CAE1DAE1EAE1FAE299723961FADBA
:10C450002397107FA12CC12CF12CE12C01E0249614
:10C460002FAD249725963FAD259740E027965FADE9
:10C47000279728966FAD289729967FAD2997CE01EB
:10C4800001960E946E4ACE0101960E948F45C85BBC
:10C49000DF4F0FB6F894DEBF0FBECDBFDF91CF9157
:10C4A0001F910F91FF90EF90DF90CF90BF90AF90D2
:10C4B0009F908F907F906F900895F70180858F7087
:10C4C000843009F096CF61857285FB0180818823D5
:10C4D00009F48FCF41E0CE0101960E94FEAC6BEAD9
:10C4E00077E087EE9AE00E94C48CBE016F5F7F4FB9
:10C4F00087EE9AE00E946D8C68EA77E087EE9AE01A
:10C500000E94C48CF701618572856BCF01151105FE
:10C51000E9F441E067E275E0CE0101960E94FEACCD
:10C5200062EA77E087EE9AE00E94C48CBE016F5FFA
:10C530007F4F87EE9AE00E946D8C6FE977E087EE7F
:10C540009AE00E94C48C67E275E04BCFF8018085C9
:10C550008F70843009F04DCF61857285FB01808139
:10C56000882309F446CF41E0CE0101960E94FEAC3B
:10C5700069E977E087EE9AE00E94C48CBE016F5FA4
:10C580007F4F87EE9AE00E946D8C66E977E087EE38
:10C590009AE00E94C48CF801B6CFF801012BB1F4E7
:10C5A00025961CAE1DAE1EAE1FAE259729961CAE5D
:10C5B0001DAE1EAE1FAE299723961FAD2397107F89
:10C5C000A12CC12CF12CE12C02E049CF80858F7089
:10C5D000843009F058CF61857285FB018081882302
:10C5E00009F451CFCE0101960E9415A44CCFEF92D1
:10C5F000FF920F931F93CF93DF93EC018B011E8269
:10C600001D821A821B821C82E880F980E114F104E9
:10C6100059F18091DD069091DE06892B29F1672B77
:10C6200009F48701F80180858F708630E9F46BE2A8
:10C6300075E0C8010E94CB9C009719F0FC01818530
:10C640008A836AE676E0C8010E94CB9CFC01892BB4
:10C6500061F180858F70823071F0853079F0F9E07A
:10C66000EF0EF11CFE82ED82DF91CF911F910F91B1
:10C67000FF90EF90089581858B83F1CF0680F7813D
:10C68000E02D309761F380858F70823041F781858E
:10C690008B830680F781E02D309709F380858F70BA
:10C6A0008230E9F681858C83DACFF801808191812F
:10C6B0000E94F8CFE1CF0F931F93CF93DF93CDB7B5
:10C6C000DEB76F970FB6F894DEBF0FBECDBF2091D7
:10C6D000DD063091DE06232B09F40BC12091B00753
:10C6E000022E000C330B82179307B4F462E07FE054
:10C6F00080E49AE00E94C48C80E49AE00E94F68A6A
:10C7000080E06F960FB6F894DEBF0FBECDBFDF910D
:10C71000CF911F910F9108956CEE7EE087EE9AE025
:10C720000E94C48C87EE9AE00E94F68A8091D2061D
:10C730008F5F8093D20667EA7EE086E39AE00E94EC
:10C74000C48C86E39AE00E94F68AE091B207F091E9
:10C75000B307309709F18091B0078F5F8093B007DE
:10C76000068117810115110591F0D80118968C9159
:10C770008F70863041F41A83098370E060E0CE0147
:10C7800001960E94F762F80102811381EBCF80913C
:10C79000B00781508093B007E091B607F091B707DA
:10C7A0003097A1F10681178101151105C9F1D80152
:10C7B00018968C918F70853029F5C8010E94EBA1E5
:10C7C000882301F14091B6075091B707F8016081C5
:10C7D0007181CE0101960E942C40CE0101960E94EB
:10C7E0009A3E882359F08C859D85009739F0DC01AD
:10C7F000ED91FC910084F185E02D1995CE01019613
:10C800000E948F45F80102811381CECF6CED7EE04E
:10C8100087EE9AE00E94C48C87EE9AE00E94F68A26
:10C820001092AE071092AD0764ED7EE087EE9AE0BD
:10C830000E94C48C87EE9AE00E94F68A64E670E05B
:10C8400080E090E00E94FDAB10923A071092A8079A
:10C850006CEB7EE087EE9AE00E94C48C0E944B2D28
:10C86000AB01BC0187EE9AE00E9448A18091DD06F1
:10C870009091DE06009711F00E9436A71092DE0616
:10C880001092DD061092B3071092B2071092B7070C
:10C890001092B60710923C0710923B071092D406F4
:10C8A0001092D3061092A6071092A5071092A40723
:10C8B0001092A3071092A2071092B9071092B8071E
:10C8C00067EB7EE087EE9AE00E94C48C0E944B2DBD
:10C8D000AB01BC0187EE9AE00E9448A187EE9AE086
:10C8E0000E94F68A1092A7078091D2068150809309
:10C8F000D20681E006CF2F923F924F925F927F92B5
:10C900008F929F92AF92BF92CF92DF92EF92FF925F
:10C910000F931F93CF93DF93CDB7DEB7A9970FB6D1
:10C92000F894DEBF0FBECDBF6C01F62E1A0149018F
:10C93000DC018D919C911197892B09F4C6C0159645
:10C94000ED91FC91309709F4C0C080818071BFEFF8
:10C950006B13BDC0C9F481E0A9960FB6F894DEBF91
:10C960000FBECDBFDF91CF911F910F91FF90EF9040
:10C97000DF90CF90BF90AF909F908F907F905F900F
:10C980004F903F902F9008954330510521F3F1804F
:10C99000F2942FE0F2226CE877E087EE9AE00E94B2
:10C9A000C48CD60113966C9187EE9AE00E944BA13D
:10C9B0006AE877E087EE9AE00E94C48CD60115966B
:10C9C000ED91FC9161816F7087EE9AE00E944BA11E
:10C9D00067E877E087EE9AE00E94C48C6F2D87EEBF
:10C9E0009AE00E944BA187EE9AE00E94F68AD60157
:10C9F0001596ED91FC9181818F70F81609F462C053
:10CA0000008103FB002700F9198E1A8E1B8E1C8EE5
:10CA10001D8E1E8E1F8E18A28A8D807F8A8FD60152
:10CA20001596ED91FC9181818F708F1579F1B3E0AE
:10CA30002B16310459F165E877E087EE9AE00E9401
:10CA4000C48CF601638187EE9AE00E944BA163E8F3
:10CA500077E087EE9AE00E94C48CD6011596ED919E
:10CA6000FC9161816F7087EE9AE00E944BA160E8B3
:10CA700077E087EE9AE00E94C48C6F2D87EE9AE0F3
:10CA80000E944BA187EE9AE00E94F68ABFE0BF1594
:10CA900008F455C1EF2DF0E08827EE5AFA498F4F80
:10CAA0000C942ED86B65AB65F76562666D66F765AD
:10CAB000D065F76570667C66E4657F668A669F660A
:10CAC0009F668D6680818F7E808380E045CF88233E
:10CAD00009F49ACFFACFF601A580B680D501119658
:10CAE0008C918F70853009F42AC168F48230D9F0B6
:10CAF0006FE175E0C4010E94CB9C2C01712CEE20EB
:10CB000009F491C0A7C08730D1F08A3089F764E377
:10CB100075E0C4010E94CB9C2C01F501708072FA73
:10CB2000772470F8ECCF6EE275E0C4010E94CB9CD4
:10CB30002C01F501708070FA772470F8E0CF6DE277
:10CB400075E0C4010E94CB9C2C01D5017C9071FA48
:10CB5000772470F8D4CF6AE175E0C4010E94CB9CC1
:10CB60002C01D6011596ED91FC91808180FB7724F4
:10CB700070F8982F9E7F80FF91609083411451043C
:10CB800009F0BDCF61E0CE0149960E949333298B15
:10CB90003A8B4B8B5C8B6D8B7E8B8F8B988FAFCF53
:10CBA0006BE375E0C4010E94CB9C2C01D601159665
:10CBB000ED91FC91808181FB772470F8982F9D7F07
:10CBC00081FF926090839BCF61E475E0C4010E9475
:10CBD000CB9C2C01D6011596ED91FC91808182FBB6
:10CBE000772470F8982F9B7F82FF9460EBCF6FE1E2
:10CBF00075E0C4010E94CB9C2C01892B69F462E092
:10CC0000CE0149960E94933329873A874B875C87E8
:10CC10006D877E878F87988BEE2009F48EC0BFE0EA
:10CC2000712CFB1217C0E3E02E16310409F48AC000
:10CC3000602F70E0C6010E944361D6011596ED9108
:10CC4000FC9180818F7E8083BFE0FB1203C0EE20C9
:10CC500009F481CE65EF74E0C4010E94CB9C8C0185
:10CC60006AEF74E0C4010E94CB9C5C016FEF74E03A
:10CC7000C4010E94CB9C99A788A7A114B10481F498
:10CC80000115110569F460E0CE0149960E949333C5
:10CC900029833A834B835C836D837E838F8398875C
:10CCA000D6011596ED91FC914114510409F05BC039
:10CCB000898D811158C0BFE0FB126AC080818F7ED0
:10CCC000808349CE67E475E0C4010E94CB9C2C01AF
:10CCD000D6011596ED91FC912DCF6CE475E0F4CF63
:10CCE00062E575E0C4010E94CB9C2C01D60115962B
:10CCF000ED91FC9170802BCF68E575E0F3CF6FE587
:10CD000075E0C4010E94CB9C2C01D6011596ED91D3
:10CD1000FC9104CF65E675E0F4CF712C512C412CC9
:10CD2000EE2009F480CF6AE175E0011102C06FE1E5
:10CD300075E0C4010E94CB9C2C01712C74CF512C46
:10CD4000412C6ACFD6011596ED91FC9180818061CE
:10CD500000FB83F9808381818F709F2D9295907F56
:10CD6000892B818371CF83E028163104C9F4818136
:10CD70008F708F1509F4EFCD9FE0F91609F4EBCD14
:10CD8000F29490EFF9228F2981838081806198CF7E
:10CD90009F2D9F70F92E8181807FF82AF1828ECF9E
:10CDA000AFE0FA1639F0BF2DBF70FB2E8181807F76
:10CDB000F82AF18280818F7E80836CE675E0C20163
:10CDC0000E94CB9C4C01009709F452C0FC01808565
:10CDD0008F70843029F0853031F0823009F048C0FE
:10CDE000B401C60143C070E060E0C4010E944C2958
:10CDF0006C010097E9F1BC018091B2079091B307F3
:10CE00000E94CB9C9AA389A370E060E0CE0181963A
:10CE10000E94F76265E775E087EE9AE00E946D8CEC
:10CE2000B60187EE9AE00E946D8C6AE775E087EEA6
:10CE30009AE00E946D8C61E070E08EA19FA1892B29
:10CE400011F470E060E087EE9AE00E9452A187EE54
:10CE50009AE00E94F68A8EA19FA1892B49F061E099
:10CE6000C4010E94439DBC01CE0181960E94DE1C3C
:10CE700088A499A46801E98CFA8C0B8D1C8D2D8DEA
:10CE80003E8D4F8D58A1672DC2010E94735C63CD0A
:10CE90002F923F924F925F926F927F928F929F92CA
:10CEA000AF92BF92CF92DF92EF92FF920F931F93B8
:10CEB000CF93DF93CDB7DEB7CB56D1090FB6F89439
:10CEC000DEBF0FBECDBFDC0115962D913C91232B0B
:10CED00009F42AC75B013C016130710509F4EEC514
:10CEE0000CF482C0643071050CF07EC0DC01129637
:10CEF0008C91803409F476C308F06DC0843008F05A
:10CF000073C0873009F470C080919B068F5F809357
:10CF10009B06F301C080D180C114D10491F067E376
:10CF200074E0C6010E94CB9CFC01892B51F09085D6
:10CF30009F709550923028F481859285009709F072
:10CF40006C01E12C00E09601A5016FEFC3010E9486
:10CF50007B64D30112968C91129781FB002700F914
:10CF600013961C919AEC910F903118F0873009F0CC
:10CF70004BC06FE775E0F301808191810E94CB9CEB
:10CF80004C01009709F440C0DC0118968C918F7019
:10CF90008530D1F58091540B181329C08091550B21
:10CFA000803429F58091560B9091570B1C01990FF5
:10CFB0004408550860E0C4010E94439DFC0181853E
:10CFC0009285A385B485281639064A065B060CF0BF
:10CFD00069C010E042C0823409F404C328F090E82C
:10CFE000980F943008F48DCF90E080E09FC61093A6
:10CFF000540B80E48093550B812F0E94C8AA909314
:10D00000570B8093560BD2CF212F30E0F901E35418
:10D01000FC4D8491F901E958FC4D1491F901EF5C44
:10D02000FC4DF490FF2009F43AC081110E94F7A949
:10D03000EF2DF0E0EE0FFF1FED50F94FA591B491E9
:10D04000EC911E2331E020E009F430E0832F922F91
:10D0500011E00817190609F0BCCFF3E0AF16B104D0
:10D0600009F4A6C0D3011596ED91FC91E181EF7012
:10D07000E150EC3008F09CC0F0E08827ED5BF74908
:10D080008F4F0C942ED86368F0699768C168F06977
:10D090000D69F069406960697969B769D76990E09D
:10D0A00080E0D6CF61E0C4010E94439D11E0FC0105
:10D0B00081859285A385B48582159305A405B50560
:10D0C0000CF0CBCF86CF0E9430ACDC01CB01AA277D
:10D0D000BB27F30125813681F90122813381821B2F
:10D0E000930BA109B109AA27BB27883E9340A1054C
:10D0F000B10508F45DC067E475E0D3018D919C91A2
:10D100000E94CB9CEE24E394012F892B41F46CE424
:10D1100075E0C6010E94CB9C892B09F4ACC0960136
:10D1200042E050E063E0C3010E947B6441C00E9482
:10D1300030ACDC01CB01AA27BB27F3012581368166
:10D14000F90122813381821B930BA109B109AA271E
:10D15000BB278C329140A105B10550F1EE24E39438
:10D16000012F960142E050E064E0C3010E947B641D
:10D170000E9430ACD3011596ED91FC9173836283CC
:10D1800017C00E9430ACDC01CB01AA27BB27F301FA
:10D1900025813681F90122813381821B930BA109FC
:10D1A000B109AA27BB2786399105A105B105B0F6BB
:10D1B000D3011596ED91FC91808183FB882780F93E
:10D1C000181709F42DC1D3011596ED91FC918081BA
:10D1D000982F907E09F06CC10E9430ACF301A581BC
:10D1E000B68113967C936E9312971196EC911197DA
:10D1F000EF70112309F4A2C1E23009F46AC108F00A
:10D200005DC1EE2309F494C1EC90E3FAEE24E0F85A
:10D2100001E09601A5016FE07DC10E9430ACDC0108
:10D22000CB01AA27BB27F30125813681F901228191
:10D230003381821B930BA109B109AA27BB27883E22
:10D240009340A105B10508F4B3CF62E575E0C601CE
:10D250000E94CB9CEE24E394012F892B39F468E5DE
:10D2600075E0C6010E94CB9C892B29F0960142E013
:10D2700050E068E058CF960142E050E06DE053CFB7
:10D280000E9430ACDC01CB01AA27BB27F30125812A
:10D290003681F90122813381821B930BA109B109E7
:10D2A000AA27BB278C329140A105B10508F480CF95
:10D2B000EE24E394012F960142E050E069E055CF5F
:10D2C0000E9430ACDC01CB01AA27BB27F3012581EA
:10D2D0003681F90122813381821B930BA109B109A7
:10D2E000AA27BB2786399105A105B10508F460CFAF
:10D2F000DFCF0E9430ACDC01CB01AA27BB27F301B2
:10D3000025813681F90122813381821B930BA1098A
:10D31000B109AA27BB27883E9340A105B10508F4AF
:10D3200047CF6FE575E0C6010E94CB9C892B39F48D
:10D3300065E675E0C6010E94CB9C892B41F0EE2486
:10D34000E394012F960142E050E06BE0ECCE61E403
:10D3500075E0C6010E94CB9CEE24E394012F960158
:10D3600042E050E066E0892B09F088CFDCCE0E94D5
:10D3700030ACDC01CB01AA27BB27F3012581368124
:10D38000F90122813381821B930BA109B109AA27DC
:10D39000BB278C329140A105B10508F409CFEE24DA
:10D3A000E394012F960142E050E06CE0DECE0E9453
:10D3B00030ACDC01CB01AA27BB27F30125813681E4
:10D3C000F90122813381821B930BA109B109AA279C
:10D3D000BB2786399105A105B10508F4E9CEDFCF59
:10D3E0000E9430ACDC01CB01AA27BB27F3012581C9
:10D3F0003681F90122813381821B930BA109B10986
:10D40000AA27BB2788359240A105B10508F4D0CEE4
:10D41000EE24E394012F960142E050E060E083CED9
:10D420000E9430ACF30185809680DC01CB01AA27F5
:10D43000BB27F40122813381821B930BA109B1091F
:10D44000AA27BB2780339547A105B105F8F0C11481
:10D45000D104E1F0D60118968C918F708630B1F42A
:10D4600063E875E0C6010E94CB9CFC01892B71F03A
:10D4700080858F70823009F073C4618572858385E1
:10D480009485672B682B692B09F09DCEF401808170
:10D490008F718064808380919B06815080939B066E
:10D4A000A3CD61857285838594850E942BD9E9CFB0
:10D4B000982F907E90528F71892BECCFE53049F0F8
:10D4C000E73009F0A1CEE12C01E09601A5016AE068
:10D4D00021C06BE375E0C6010E94CB9C892BA9F4A7
:10D4E00062E575E0C6010E94CB9C892B71F468E56A
:10D4F00075E0C6010E94CB9C892B39F46DE275E082
:10D50000C6010E94CB9C892B99F0E12C01E0960189
:10D51000A50166E0C3010E947B64882309F4BBCFA8
:10D52000D3011596ED91FC91808110FB83F9B2CF68
:10D53000E12C01E09601A50161E0ECCFE150ED3076
:10D5400008F048C0F0E08827E755F5498F4F0C9464
:10D550002ED8B66AEA6ABC6ABC6AEA6AC26AEA6A31
:10D56000E46AE46AE46AE46AE46ABC6AE12C00E022
:10D570009601A50162E0CECFE12C00E09601A50165
:10D5800065E0C8CF6BE375E0C6010E94CB9C892B98
:10D59000A9F462E575E0C6010E94CB9C892B71F469
:10D5A00068E575E0C6010E94CB9C892B39F46DE2D9
:10D5B00075E0C6010E94CB9C892B31F0E12C00E084
:10D5C0009601A50167E0A6CFE12C00E09601A50138
:10D5D00060E0A0CFEC90E3FAEE24E0F881E0E826EA
:10D5E00000E017CEB3E0AB16B10409F4FDCC6FE751
:10D5F00075E0F301808191810E94CB9C8C01D30165
:10D6000013968C919091540B8913E0C09091550B17
:10D61000903409F0DBC08091560B9091570B2C0190
:10D620000115110509F401C1F80120852F7025307D
:10D6300009F0FBC0C8010E94EBA1A2968FAFA29790
:10D64000843008F4CFC063E0C8010E94439DDC0130
:10D6500019968D919C91BAE0EB2EE89E1001E99EFF
:10D66000300C112462E0C8010E94439DFC018185B9
:10D670009285E89E6001E99ED00C1124AC96DFAE45
:10D68000CEAEAC974601DD0CAA08BB0861E0C8012C
:10D690000E94439D7C0160E0C8010E94439DDC0123
:10D6A00019962D913D914D915C911C97A6962CAFAA
:10D6B0003DAF4EAF5FAFA6979201052C000C440B17
:10D6C000550BA6966CAD7DAD8EAD9FADA697261B76
:10D6D000370B480B590BB101032C000C880B990B2D
:10D6E000681979098A099B090E9493D7D70119966D
:10D6F0002D913D914D915C911C97A696CCACDDACE3
:10D70000EEACFFACA6972C193D094E095F09A69611
:10D710002CAF3DAF4EAF5FAFA6970E94C5D7820E2C
:10D72000931EA41EB51EA2962FADA297253009F414
:10D730006BC0EE24E394F12CC101032C000CAA0B66
:10D74000BB0B88159905AA05BB050CF466C0D5016D
:10D75000C401AC96CEACDFACAC979601DD0C440BAB
:10D76000550B82179307A407B5070CF45BC09C0107
:10D77000AD01A2966FADA297623009F06AC0620156
:10D78000550CEE08FF0860E0C8010E94439DFC01B3
:10D7900081859285A385B485C816D906EA06FB065D
:10D7A0000CF4EBC261E0C8010E94439DFC0181853D
:10D7B0009285A385B4858C159D05AE05BF050CF03B
:10D7C00013CCC12CD12C7601C394DAC28093540BB4
:10D7D00090E49093550B0E94C8AA9093570B8093A6
:10D7E000560B1DCF8AE0849D4001859D900C11242D
:10D7F000092C000CAA08BB08AC961FAE1EAEAC9755
:10D80000212CA8E23A2E95CF64E0C8010E94439DE6
:10D81000DC011996ED90FC908FCF44244A94E3E00C
:10D820005E2E97CF512C412CA4CF2AE0289F400197
:10D83000299F900C11249401990C440B550BAC9624
:10D840001FAE1EAEAC97212C68E2362EEE24E39478
:10D85000F12CD3011596ED91FC9162817381C20187
:10D86000861B970B97FF03C0919581959109E81648
:10D87000F90674F08081982F92959695977096305E
:10D8800050F49F5F9295990F907E8F71892B02C003
:10D8900080818F7180838081803AB8F0AC96EEAD44
:10D8A000FFADAC976F01FF0FEE08FF08C216D3065D
:10D8B000E406F50651F0C101330CAA0BBB0B82172D
:10D8C0009307A407B50709F08FCB4616570609F44E
:10D8D0008BCB6D961CAE1DAE1EAE1FAE6D976B96BC
:10D8E0008FAD6B97807F86606B968FAF6B976D96D1
:10D8F0008CAD9DADAEADBFAD6D9765968CAF9DAF58
:10D90000AEAFBFAF6597AAE0B0E00E94E4D76996DA
:10D910006CAF7DAF8EAF9FAF69976FEE76E087EE0D
:10D920009AE00E94C48CD30113966C9187EE9AE022
:10D930000E944BA16DEE76E087EE9AE00E94C48CC7
:10D94000CE018F5A9F4F0E94293367E374E0F301A1
:10D95000808191810E94CB9C912C812CB12CA12C97
:10D96000D12CC12C6296EFAC62976396FFAC6397A3
:10D9700064960FAD649765961FAD659766962FAD5B
:10D98000669767963FAD679768964FAD68976996BB
:10D990005FAD69976FEF0E94735CD3010D911C918D
:10D9A00065EF74E0C8010E94CB9C7C016AEF74E0D3
:10D9B000C8010E94CB9C8C010097E9F1FC01808595
:10D9C0008F708430C1F56185728540E450E0CE01EE
:10D9D00001960E94BDDC6FE270E0CE0101960E94CC
:10D9E00084DC892B59F4D80119962D913C9143E0A0
:10D9F00050E060E4CE0101960E94462C00E020E059
:10DA000030E240E150E0BE016F5B7F4FCE018F5AA4
:10DA10009F4F0E946B200E94E99C882361F08091B7
:10DA2000AF07811108C041E0BE016F5B7F4FCE019F
:10DA300001960E94FEACE114F104C9F1F701808562
:10DA40008F708430A1F54091B6075091B70761857A
:10DA50007285CE0101960E942C40CE0101960E9453
:10DA60009A3E882301F1A12CC12CF12CE12C629665
:10DA70000FAD629763961FAD639764962FAD649761
:10DA800065963FAD659766964FAD669767965FADB5
:10DA9000679768966FAD689769967FAD6997CE0175
:10DAA00001960E946E4ACE0101960E948F45D301D5
:10DAB0001596ED91FC915382428296CAFC018281B7
:10DAC000883009F440C0803109F08ECA0E9430AC21
:10DAD0006B017C01C3010E94AE16C61AD70AE80A80
:10DAE000F90A30E3C31635E7D306E104F10408F47C
:10DAF0007BCA6AEF74E0D3018D919C910E94CB9C0C
:10DB00008C01009709F405C1FC0180858F70843079
:10DB100009F0FFC00E9430AC2AE0AE014F5F5F4FBA
:10DB20000E9408D10E94E99C882309F4F2C08091E8
:10DB3000AF078111EEC0BE016F5F7F4FD80119960C
:10DB40008D919C91E4C00E9430AC6B017C01C301BB
:10DB50000E94AE16C61AD70AE80AF90AF8E9CF16E3
:10DB6000FAE3DF06E104F10408F43ECAD301159696
:10DB7000ED91FC911697818113961C91811155C0EE
:10DB8000163008F03FC08CE0EEE1F2E0DE011196C5
:10DB900001900D928A95E1F7E12FF0E0EE0FFF1F63
:10DBA000CC24C394D12CCC0EDD1EEC0DFD1D60E009
:10DBB00080810E948CAA6EEF76E183E01330C9F079
:10DBC00070F466E077E181E0113099F062E077E18E
:10DBD00082E0123071F06AE077E180E00AC06AEF1B
:10DBE00076E184E0143029F066EF76E185E01530C7
:10DBF00091F70E945AA1D3011596ED91FC9181E015
:10DC00008183F2C961E677E087EE9AE00E94C48CD6
:10DC1000F301638187EE9AE00E944BA164E377E011
:10DC200087EE9AE00E94C48CDFC924E0129FF001C5
:10DC30001124E456F94F80809180A280B38060E384
:10DC400077E087EE9AE00E94C48CD30113966C9122
:10DC500087EE9AE00E944BA16CE177E087EE9AE0B4
:10DC60000E94C48C2AE030E0B501A40187EE9AE05E
:10DC70000E94E78B6AEF74E0F301808191810E943A
:10DC8000CB9C8C01009709F44CC0DC0118968C9158
:10DC900018978F70843009F044C019966D917C916B
:10DCA00040E450E0CE0101960E94BDDC6FE270E0DE
:10DCB000CE0101960E9484DC892B51F4F801218564
:10DCC000328543E050E060E4CE0101960E94462C8C
:10DCD000BF92AF929F928F9282E494E09F938F9332
:10DCE0008E010F5B1F4F1F930F930E9414DD0E9444
:10DCF000E99C0FB6F894DEBF0FBECDBF882349F074
:10DD00008091AF07811105C0B801CE0101960E9434
:10DD10001CAD0E9430ACAB01BC01C3010E94871650
:10DD200063C96DE077E07CCF8FEF9FEFC559DF4F80
:10DD30000FB6F894DEBF0FBECDBFDF91CF911F911C
:10DD40000F91FF90EF90DF90CF90BF90AF909F909A
:10DD50008F907F906F905F904F903F902F9008959D
:10DD6000833009F49ECB813009F090CB6185062E7B
:10DD7000000C770B880B990B84CBC12CD12C76012E
:10DD8000D3011596ED91FC9182819381092E000CAF
:10DD9000AA0BBB0B8C159D05AE05BF0509F424C964
:10DDA000B601C3010E944361D3011596ED91FC9128
:10DDB000D382C28219C9BF92CF92DF92EF92FF92B3
:10DDC0000F931F93CF93DF93CDB7DEB72E970FB688
:10DDD000F894DEBF0FBECDBF2091B2073091B307DC
:10DDE000232B09F4A6C02091B1072111A2C07C0108
:10DDF0008091B1078F5F8093B1078091B0078F5FEB
:10DE00008093B0070E9430AC0091D9061091DA06D9
:10DE10002091DB063091DC06601B710B820B930BAB
:10DE20006B3071058105910508F479C083E0E8162F
:10DE3000F104A9F00E9430AC0091D5061091D606ED
:10DE40002091D7063091D806601B710B820B930B83
:10DE5000BB24B394643671058105910508F4B12C97
:10DE6000E091B207F091B307068117810115110502
:10DE7000C1F1F80180858F70863079F519870887A0
:10DE800070E060E0CE0108960E94F762B701CE0113
:10DE900008960E94486767E374E0C8010E94CB9C23
:10DEA000FC01892BD1F090859F7095509230A8F499
:10DEB000C680D780C114D10481F0DA82C982B8014A
:10DEC000CE0101960E94F762B701CE0101960E9431
:10DED0004867F601C280D380EDCFF801028113813B
:10DEE000C5CFF3E0EF16F10451F00E9430AC60931F
:10DEF000D9067093DA068093DB069093DC06BB208C
:10DF000051F00E9430AC6093D5067093D606809392
:10DF1000D7069093D8061092540B1092550B80910F
:10DF2000B00781508093B0078091B10781508093F2
:10DF3000B1072E960FB6F894DEBF0FBECDBFDF91AE
:10DF4000CF911F910F91FF90EF90DF90CF90BF90F6
:10DF500008958091AF078F5F8093AF07A89583E006
:10DF600090E00E94DB6E0E9406918091AF07815085
:10DF70008093AF070895CF92DF92EF92FF92CF93F5
:10DF8000DF93EC018C85883068F40E94B0980E9481
:10DF900030AC6B017C018C850E94CC98811109C04A
:10DFA00088E08C87DF91CF91FF90EF90DF90CF904A
:10DFB00008950E94A96F61E070E080E090E00E9407
:10DFC000FDAB0E9430ACAB01BC014C195D096E0980
:10DFD0007F098D859E85B0E0A0E0481759076A0744
:10DFE0007B07C8F28C850E94BE98DACF8F929F92F1
:10DFF000BF92CF92DF92EF92FF920F931F93CF9336
:10E00000DF93CDB7DEB7AE970FB6F894DEBF0FBE85
:10E01000CDBF8091DD069091DE06892B09F4E9C41D
:10E020008091B0078111E5C48091B0078F5F809324
:10E03000B0076FE974E186E39AE00E94C48C86E33E
:10E040009AE00E94F68A0091DD061091DE066AE8E9
:10E0500075E0C8010E94CB9C9093B7078093B607E8
:10E0600060E975E0C8010E94CB9C90933C078093C7
:10E070003B0765EB75E0C8010E94CB9C9093B3070A
:10E080008093B20767E975E0C8010E94CB9C90932A
:10E09000D4068093D306009739F1DC011696ED91F2
:10E0A000FC91309709F120852F702530E9F46BE859
:10E0B00074E186E39AE00E94C48C8091D30690912B
:10E0C000D4060E94EBA18093A207682F86E39AE012
:10E0D0000E944BA186E39AE00E94F68AE091D30663
:10E0E000F091D406868197819093A6078093A50727
:10E0F0000E9481316CE975E08091DD069091DE0629
:10E100000E94CB9C9093B9078093B807892B09F4A0
:10E1100042C08091BA0781113EC08091AB079091B7
:10E12000AC07892B09F0DDC16DE374E187EE9AE05D
:10E130000E94C48C87EE9AE00E94F68A8FE090E0FD
:10E140000E942BCE8C0188E1F8018183128210821B
:10E15000168615860E941FA71093AC070093AB0785
:10E16000012B09F08CC06EE274E180E49AE00E9419
:10E17000C48C80E49AE00E94F68A80E081708093EB
:10E18000BA078091BA07882331F06BE774E186E320
:10E190009AE00E94C48C1092AE071092AD07E091F5
:10E1A000B607F091B707309709F4C8C2E680F78048
:10E1B0000091B6071091B7070115110509F4B7C210
:10E1C000E114F10409F4B3C2F70180858F70853042
:10E1D00099F7C7010E94EBA1823070F3A801B70143
:10E1E000CE0101960E942647CE0101960E949A3EDA
:10E1F0008823E1F18C859D85009709F411C2DC012B
:10E20000ED91FC910284F385E02D1995892B49F05D
:10E210008C859D85DC01ED91FC910084F185E02DDC
:10E2200019958C859D85DC01ED91FC910680F78127
:10E23000E02D1995892BD1F0CE0101960E94C341A2
:10E24000882341F040E050E160E070E0CE010196AB
:10E250000E94AB1B8F819885892B41F040E050E2F2
:10E2600060E070E0CE0101960E94AB1BD7011296D0
:10E27000ED90FC90CE0101960E948F4599CF0E94AF
:10E280001FA78091AB079091AC070E94571B882372
:10E2900009F494C06FE074E186E39AE00E94E88C90
:10E2A0008091AB079091AC070E946626E091AB0786
:10E2B000F091AC0781E080838091AB079091AC072F
:10E2C0000E9474266BEF73E1811102C066EE73E168
:10E2D00087EE9AE00E94E88C8091B8079091B90788
:10E2E000892B09F44ACF8091A9079091AA07892B1D
:10E2F00009F0E9C083E190E00E942BCE8C0180916F
:10E30000AB079091AC0721E830E8D80152963C93D6
:10E310002E93519716969C938E93159714961C9254
:10E3200014971C9289E011968C93119781E01296B4
:10E330008C93129713968C931093AA070093A907B6
:10E340000E9430AC6B017C01B0E1CB0EB7E2DB1E6A
:10E35000E11CF11CD8011596ED91FC9116978FEFF9
:10E360008387148613821482158216821782108680
:10E370001186128614961C92BB24B394BE01605E73
:10E380007F4FF801858196810E944E2718160CF068
:10E3900095C00E9430AC6C157D058E059F0508F078
:10E3A0008DC0DE01909698E080E0915019F1ED91DA
:10E3B000E827F0E0E158F34E8491F7CF0E946229FC
:10E3C0008091AB079091AC070E94571B882359F0AE
:10E3D00069EC73E186E39AE00E94C48C86E39AE0DC
:10E3E0000E94F68A79CF6DEA73E180E49AE00E9498
:10E3F000E88CC3CE9FA19813C1CFD8018C91811115
:10E4000038C015968D919C910E947426BE01605E65
:10E410007F4FF801858196810E94472640E064EB9A
:10E42000D80115968D919C910E942126F801858036
:10E430009680C4010E94A525C4010E94D51367E8F7
:10E4400087EA99E00E94601460E887EA99E00E94F8
:10E4500060140E94FAABC4010E94A525982ED80131
:10E4600015968D919C910E94742695FC02C0F8012E
:10E47000B082AE014F5F5F4FBE01605E7F4FC8014B
:10E480000E94B526D80111969C9088A1803109F48C
:10E49000B2C2BE01605E7F4FC8010E942427891569
:10E4A00010F5F8018181D80111968C93119714967B
:10E4B0008C9114978F5F14968C9360CFE091A9078D
:10E4C000F091AA071282E091B807F091B907E680AF
:10E4D000F7809FE7D92E8091B8079091B907892BD3
:10E4E00071F481E04BCE88A1803111F48CE0DBCF58
:10E4F000BE01605E7F4FC8010E942427D4CFE11483
:10E50000F10479F3BE01605E7F4FF7018081918154
:10E510000E94DA2E882329F366E973E187EE9AE0F8
:10E520000E94C48CD7016D917C9187EE9AE00E9485
:10E530006D8C87EE9AE00E94F68A0091A9071091EF
:10E54000AA07AE014F5F5F4FBE01605E7F4FC801FB
:10E550000E940A27882309F45EC088A1803109F44B
:10E560005AC0DD82F801858196810E947426BE0121
:10E57000605E7F4FD80115968D919C910E94472631
:10E5800040E06EE4F801858196810E94212640E0FA
:10E590006B81D80115968D919C910E94212640E0B7
:10E5A0006C81F801858196810E94212688A18031A5
:10E5B00041F040E06D81D80115968D919C910E94AB
:10E5C0002126F801858196810E947426BE01605E35
:10E5D0007F4FD80115968D919C910E944726F80196
:10E5E000408168E4858196810E94212664E170E083
:10E5F00080E090E00E94FDABD8018C91882331F03F
:10E600006AE070E080E090E00E94FDABF801858157
:10E6100096810E947426D7011296ED90FC905BCFF4
:10E62000CE0101960E94FBA18C01912C812C97FFB9
:10E6300006C011950195110988248394912CCE016F
:10E6400001960E94C341C82ED12C8B85853091F054
:10E65000863009F00BCEB02E61E0802F0E948CAA8C
:10E6600061E0892809F441C0CA94CD2809F041C06D
:10E6700060E03FC0CD2829F462E0CE0101960E94FF
:10E68000F81B40E050E160E070E0CE0101960E948E
:10E69000AB1B8F819885892B41F040E050E260E010
:10E6A00070E0CE0101960E94AB1B61E0802F0E94BA
:10E6B0008CAA60E0802F0E945EAA63E774E187EE77
:10E6C0009AE00E94C48CB80187EE9AE00E9452A1A1
:10E6D0006EE674E187EE9AE00E94C48C6CE674E109
:10E6E00087EE9AE00E94C48CC1CDCA94CD2809F06F
:10E6F000BFCFC62ED12C8B2D0E945EAA67E674E197
:10E7000087EE9AE00E94C48CB80187EE9AE00E94DE
:10E7100052A165E674E187EE9AE00E94C48CB601CE
:10E7200087EE9AE00E9452A163E674E1D9CFF80126
:10E73000868197819093AE078093AD0787EE9AE02C
:10E740000E94F68A62E873E186E39AE00E94C48C34
:10E7500086E39AE00E94F68AE091B207F091B3074F
:10E76000309709F4A8C08091B0078F5F8093B007FD
:10E77000068117810115110509F498C0D801189672
:10E780008C918F70863009F07EC019A708A770E0C1
:10E7900060E0CE0188960E94F7628DA59EA5892B28
:10E7A00009F471C08091DD069091DE06892B09F491
:10E7B0006AC0E8A4F9A4E114F104B9F1F701808575
:10E7C0008F70863091F5F9A2E8A270E060E0CE018A
:10E7D00080960E94F762EDA1FEA110821182128242
:10E7E000138267E374E0C7010E94CB9CFC01892B74
:10E7F000E1F090859F7095509230B8F4C680D78034
:10E80000C114D10491F0DA82C982B701CE01019618
:10E810000E94F762EE81FF811082118212821382C0
:10E82000D6011296CD90DC90EBCF6DE773E187EEC9
:10E830009AE00E94C48C6BA587EE9AE00E944BA1DF
:10E840006BE773E187EE9AE00E94C48C6AA587EEBD
:10E850009AE00E944BA187EE9AE00E94F68AEDA50D
:10E86000FEA510821182128213828AA5843078F468
:10E87000823098F060E08BA50E948CAAEDA5FEA5E1
:10E880008181807F8183F8010281138173CF80347D
:10E8900059F0823421F08032B1F762E0ECCF60E0D1
:10E8A0008BA50E948CAAEFCF62E0FACF8091B007CF
:10E8B00081508093B0076EE673E186E39AE00E9490
:10E8C000C48C66E673E186E39AE00E94C48C81E022
:10E8D0002091B6073091B707232B09F480E00E94FE
:10E8E000471C6DE573E186E39AE00E94C48C81E0E9
:10E8F0002091B2073091B307232B09F480E00E94E6
:10E90000471C66E573E186E39AE00E94C48C81E0CF
:10E910002091A5073091A607232B09F480E00E94DF
:10E92000471C6DE473E186E39AE00E94C48C81E0A9
:10E930002091B8073091B907232B09F480E00E9499
:10E94000471C64E473E186E39AE00E94C48C8091E2
:10E950003A070E94471C86E39AE00E94F68A6FE31A
:10E9600073E186E39AE00E94C48C0E944B2DAB01B8
:10E97000BC0186E39AE00E9448A186E39AE00E94E7
:10E98000F68A81E08093A80783E09AE00E94F61956
:10E99000882351F083E09AE00E94BB6F84E090E00E
:10E9A0009093B5078093B4078091B4079091B50711
:10E9B000079731F484E090E09093B5078093B40713
:10E9C0008091B00781508093B0078091A807AE96E0
:10E9D0000FB6F894DEBF0FBECDBFDF91CF911F9170
:10E9E0000F91FF90EF90DF90CF90BF909F908F900E
:10E9F000089580E0ECCFFCE0F91508F452CD76CD17
:10EA0000CF92DF92EF92FF921F93CF93DF93EC01AF
:10EA10007B016A018C85883048F40E94CC98882359
:10EA200019F08C850E94B09888E08C87F70182816C
:10EA30009381A481B5810097A105B10551F490E0BF
:10EA400080E0DF91CF911F91FF90EF90DF90CF900A
:10EA500008958F3F9F4FAF4FBF4F89F370E060E045
:10EA600081E20E940799182F8C87883040F780E553
:10EA700091E00E94DEA6A7014E5F5F4F24E030E0E8
:10EA80006CE070E0812F0E94BD22B601812F0E94B0
:10EA9000DB9864E070E0812F0E94E8930E9430AC24
:10EAA0006B017C018C850E94CC98873121F18C31DF
:10EAB00011F1882321F20E9430ACAB01BC014C194A
:10EAC0005D096E097F098D859E85B0E0A0E0841701
:10EAD0009507A607B70748F00E94A96F61E070E0AC
:10EAE00080E090E00E94FDABDDCF8C850E94BE9857
:10EAF00088E08C87A4CF81E090E0A3CFA89582E046
:10EB000090E00C94DB6EAF92BF92DF92EF92FF9297
:10EB10000F931F93CF93DF9300D000D0CDB7DEB714
:10EB20008C017B01D42EFB0184819581892BF9F026
:10EB3000A080B1806FE370E0C5010E9484DC009783
:10EB4000B1F09C012A193B0937FD11C050E040E0AB
:10EB5000B701CE0101960E94A788BE016F5F7F4F6B
:10EB6000C7010E94F586CE0101960E9457886FE981
:10EB700075E0C7010E94E086882321F1F801128A1E
:10EB8000118A80E090E19587848784E890E0948BF7
:10EB9000838B81E0868780E090E2908B8787D58A9F
:10EBA00081E090E026960FB6F894DEBF0FBECDBF91
:10EBB000DF91CF911F910F91FF90EF90DF90BF9069
:10EBC000AF9008956CEA75E0C7010E94E086882343
:10EBD00069F0F801128A118A148A138A84E890E095
:10EBE00095878487168680E090E3D7CF90E080E019
:10EBF000D9CFEF92FF920F931F93CF93DF9300D063
:10EC00001F92CDB7DEB78C017B01FB018485883074
:10EC1000A8F08CE294E0F801918380831282138241
:10EC200014821582C8010F900F900F900F90DF9102
:10EC3000CF911F910F91FF90EF90089580E591E0A3
:10EC40000E94DEA624E030E0AE014F5F5F4F6CE033
:10EC500070E0F70184850E940E23BE016F5F7F4F35
:10EC6000C8010E94048DDECFEF92FF920F931F9395
:10EC7000CF93DF9300D000D0CDB7DEB78091120ADA
:10EC80009091130A892B09F46CC087E70E94179EA4
:10EC90008091120A9091130ADC01ED91FC91008899
:10ECA000F189E02D70E060E0199510E000E08091BE
:10ECB000120A9091130ADC01ED91FC9111971C96B8
:10ECC0002D913C910217130740F40190F081E02D43
:10ECD00060E019950F5F1F4FEACF0088F189E02DA2
:10ECE00070E060E0199505E313E089E3E82E83E026
:10ECF000F82E8091120A9091130AF80161918F0108
:10ED0000DC01ED91FC910190F081E02D1995E01668
:10ED1000F10679F78091120A9091130ADC01ED91C6
:10ED2000FC910488F589E02D199565E076E0CE0127
:10ED300001960E949688CE0101960E94B6B3CE013C
:10ED400001960E94578887E090E00E9433A187E0F7
:10ED500090E00E943DA165EC76E186E39AE00E9496
:10ED6000C48C1092320A1092310A80E090E19093A4
:10ED70002D0A80932C0A84E890E09093340A8093C3
:10ED8000330A81E080932E0A80E090E29093300A6B
:10ED900080932F0A82E78093350A80E29AE00E94EE
:10EDA0004A1780E29AE00E94671C88EC90E0269661
:10EDB0000FB6F894DEBF0FBECDBFDF91CF911F918C
:10EDC0000F91FF90EF900895CF93DF93CDB7DEB70B
:10EDD0002E970FB6F894DEBF0FBECDBF8091B0075F
:10EDE000811121C18091B0078F5F8093B0076AEFD6
:10EDF00074E186E39AE00E94C48C86E39AE00E9464
:10EE0000F68A1092320A1092310A80E090E19093D3
:10EE10002D0A80932C0A84E890E09093340A809322
:10EE2000330A81E080932E0A80E090E29093300ACA
:10EE300080932F0A82E78093350A80E29AE00E944D
:10EE4000AA228B37910509F0C5C06CEE74E187EEFC
:10EE50009AE00E94C48C87EE9AE00E94F68A809124
:10EE6000DD069091DE06892B21F081E090E00E9482
:10EE70005B631C821B8287E892E09A83898380E22D
:10EE80009AE09E838D838FEF9FEF98878F83CE01CB
:10EE900001960E9462A79093DE068093DD0680E2D1
:10EEA0009AE00E94671C8091DD069091DE06892B16
:10EEB00001F560EE74E180E49AE00E94C48C80E485
:10EEC0009AE00E94F68A65E076E0CE0109960E94FB
:10EED0009688CE0109960E94B6B3CE0109960E948B
:10EEE00057888091B00781508093B00790E080E010
:10EEF00019C06DEC74E186E39AE00E94C48C86E34D
:10EF00009AE00E94F68A8091B00781508093B00702
:10EF10000E94F66F8091120A9091130A892B59F47E
:10EF200081E090E02E960FB6F894DEBF0FBECDBF05
:10EF3000DF91CF9108950E942C9E882389F382E768
:10EF40000E94179E8091120A9091130ADC01ED91A4
:10EF5000FC910088F189E02D60E670E019956091E0
:10EF6000120A7091130A40E0CE0109960E94738A3A
:10EF7000BE01675F7F4F84E19AE00E94F586CE0173
:10EF800009960E9457888091120A9091130ADC0119
:10EF9000ED91FC910488F589E02D19956FEA74E1F3
:10EFA00087EE9AE00E94C48C64E17AE0CE01099673
:10EFB0000E948D88BE01675F7F4F87EE9AE00E94B6
:10EFC000B68C87EE9AE00E94F68ACE0109960E94DE
:10EFD0005788A6CF80E29AE00E942017892BA1F0E3
:10EFE00080E29AE00E944A1765E076E0CE01019641
:10EFF0000E949688CE0101960E94B6B3CE0101967A
:10F000000E9457880E9437B480E29AE00E94671CF1
:10F010006CEB74E186E39AE00E94C48C86E39AE08C
:10F020000E94F68A5ECF8FEF9FEF7CCFFF920F9307
:10F030001F93CF93DF9300D000D0CDB7DEB78C0104
:10F04000BC01CE0101960E948D88BE016F5F7F4F8B
:10F0500087EE9AE00E94B68C87EE9AE00E94F68ACC
:10F06000CE0101960E94578860EF76E1CE010196AD
:10F070000E945F88BE016F5F7F4FC8010E94C586F6
:10F08000F82ECE0101960E945788FF2069F0B80142
:10F09000CE0101960E948D88CE0101960E94B6B3E2
:10F0A000CE0101960E94578826960FB6F894DEBFCF
:10F0B0000FBECDBFDF91CF911F910F91FF900895AB
:10F0C0004F925F926F927F928F929F92AF92BF9278
:10F0D000CF92DF92EF92FF920F931F93CF93DF9324
:10F0E000CDB7DEB7C859D1090FB6F894DEBF0FBE51
:10F0F000CDBF8E010F5B1F4FD8011D921C92FE01E8
:10F10000ED5BFF4F8EE1DF011D928A95E9F780915B
:10F11000120A9091130A892B09F4CEC10E942C9EE9
:10F12000882309F4C9C182E70E94179E8091120AC0
:10F130009091130ADC01ED91FC910088F189E02D9A
:10F1400060E270E019954FE150E0B8018091120A39
:10F150009091130A0E94719E7C018091120A9091F5
:10F16000130ADC01ED91FC910488F589E02D1995D5
:10F17000E114F10409F4A0C1F801EE0DFF1D1082A5
:10F1800080911F0A1F928F9380911E0A1F928F9366
:10F1900080911D0A1F928F9380911C0A1F928F935A
:10F1A00080911B0A1F928F9380911A0A1F928F934E
:10F1B00088EB95E09F938F931F9280E48F93FE01DD
:10F1C00031966F01FF93EF930E94D7DC6FED77E1EB
:10F1D00086E39AE00E94C48CB80186E39AE00E941C
:10F1E0006D8CB60186E39AE00E946D8C86E39AE00E
:10F1F0000E94F68A7E01F1E6EF0EF11CD70113960C
:10F200001C921E92129788EE93E0A0E0B0E0F70106
:10F2100084839583A683B78388E0848788EE93E010
:10F22000968785878FE392E091838083108A178683
:10F23000128B018B148A138A80E590E0968B858B64
:10F24000118E67EF76E187EE9AE00E94C48C64E14C
:10F250007AE0CE0185589F4F0E948D88BE01655887
:10F260007F4F87EE9AE00E94B68C87EE9AE00E946C
:10F27000F68ACE0185589F4F0E94578867EE75E049
:10F28000CE0183579F4F0E94968867EE75E0CE01AE
:10F2900085589F4F0E949688BE0165587F4FCE01CA
:10F2A0008B579F4F0E948D8864E17AE0CE018B5787
:10F2B0009F4F0E94F387BE0163577F4F0E94F387E1
:10F2C000BC01CE018D569F4F0E948D88CE018B5779
:10F2D0009F4F0E945788CE0185589F4F0E945788A4
:10F2E000CE0183579F4F0E94578889EE95E0CB57F8
:10F2F000DF4F99838883C558D040C757DF4F1982A5
:10F300001882C958D040C557DF4F19821882CB5890
:10F31000D040CD56DF4F88819981C359D040C9571D
:10F32000DF4F99838883C758D04069ED77E187EE36
:10F330009AE00E94C48C0E944B2DAB01BC0187EE69
:10F340009AE00E9448A187EE9AE00E94F68A64E65D
:10F3500070E080E090E00E94FDAB86E198E7D70185
:10F3600050969C938E931F9767E874E882E393E925
:10F370000E946ED18C010FB6F894DEBF0FBECDBFD8
:10F38000892B09F4F4C083E090E00E942BCED801D1
:10F390001D969C938E931C97FC01F182E082128251
:10F3A000C7010E94F619882319F0C7010E94BB6F9C
:10F3B000D70153966D917C9154975596AD90BC9022
:10F3C0006115710509F48FC0CE0185589F4F0E94C9
:10F3D000048DA501BE0165587F4FC7010E940075CD
:10F3E000181619060CF0C0C0D7015196BC90519761
:10F3F0005296AC90DF92CF9282E597E19F938F93E4
:10F400001F930F930E94F5D1DF92CF928DE497E185
:10F410009F938F931F930F930E94F5D1D8011C9651
:10F42000ED91FC9181E08283DF92CF928AE497E1B3
:10F430009F938F931F930F930E94F5D1D8011C9631
:10F44000ED91FC911282AF92BF9284E197E19F937C
:10F450008F931F930F930E94F5D10FB6F894DEBFE0
:10F460000FBECDBFB12C8BE0C82E87E1D82E8B2DDF
:10F4700094E08902F0011124A5E8B0E0AC0FBD1FB3
:10F48000EA0FFB1F808191810097A9F122813381CE
:10F4900021153105C9F33F932F939F938F93DF92EB
:10F4A000CF921F930F930E94F5D1B3940FB6F894A7
:10F4B000DEBF0FBECDBFDBCF40E250E061E178E1BF
:10F4C000C8010E949BD063EF77E186E39AE00E9437
:10F4D000C48CB80186E39AE00E946D8C86E39AE0C2
:10F4E0000E94F68A4DCEF70161897289A501C70194
:10F4F0000E949D1A75CF8FE497E19F938F931F937E
:10F500000F930E94F5D1D70158961C921E925797DF
:10F51000D8011C96ED91FC91C080D1800F900F9086
:10F520000F900F9043E3A42EB12CD601ED91FC91E6
:10F530000084F185E02DC601199541975CF4B1E096
:10F54000AB1AB10839F064E170E080E090E00E940D
:10F55000FDABEBCFD601ED91FC910084F185E02D60
:10F56000C6011995419734F4C8010E940B9310E02D
:10F5700000E05AC065E076E0CE0183579F4F0E94BD
:10F580009688912CA12CD601ED91FC910688F789E3
:10F59000E02DC60119958823E1F1BDE0AB1201C051
:10F5A000A92CD601ED91FC910688F789E02DC601C2
:10F5B00019958111BBC0D601ED91FC910084F185B4
:10F5C000E02DC6011995892B09F4C2C0D601ED9131
:10F5D000FC910284F385E02DC6011995B82EBAE09E
:10F5E0008B1709F4B7C0EDE08E1709F4B3C0FFEF35
:10F5F0008F1709F4ADC0682FCE0183579F4F0E942B
:10F6000082879A2CAB2CBFCFBAE0BB12FACFAB12D9
:10F61000F8CFCC24C394D12CCE0183579F4F0E94A6
:10F620005788CD2809F4A3CFD7015796ED90FC90C9
:10F630006BEC77E187EE9AE00E94C48CB70187EE0D
:10F640009AE00E9452A187EE9AE00E94F68A64E650
:10F6500070E080E090E00E94FDAB0115110509F417
:10F6600065C1B8ECEB16F10409F03EC16FEB77E130
:10F6700086E39AE00E94C48C64EF71E080E090E041
:10F680000E94FDABEF961FAE1EAEEF97C158DF4F45
:10F6900019821882CF57D0408FEF9FEFCF57DF4F9F
:10F6A00099838883C158D04081E792E0ED969FAF5F
:10F6B0008EAFED97CD57DF4F19830883C358D040E5
:10F6C000F89490E080E00E945B638111CEC063EB10
:10F6D00077E180E49AE00E94C48C80E49AE00E9482
:10F6E000F68AC8010E940B9324EFE22EFF24F394C4
:10F6F000CE018D569F4F0E945788C701C856DF4FD5
:10F700000FB6F894DEBF0FBECDBFDF91CF911F9132
:10F710000F91FF90EF90DF90CF90BF90AF909F90B0
:10F720008F907F906F905F904F900895D601ED91EC
:10F73000FC910084F185E02DC6011995892B09F013
:10F740003ACF64E670E080E090E00E94FDAB29CF04
:10F75000BB24BA9467EF75E08AE49AE00E946D8C4E
:10F76000BE0163577F4F8AE49AE00E94B68C8AE418
:10F770009AE00E94F68A62E077E1CE0185589F4FB9
:10F780000E945F88BE0165587F4FCE0183579F4F0F
:10F790000E94C586982ECE0185589F4F0E9457889B
:10F7A000992099F1CF56DF4F28813981C159D04036
:10F7B00049E050E0BE0163577F4FCE0185589F4F0F
:10F7C0000E94A788ED968EAD9FADED97412C512CF0
:10F7D0003201009719F00E9416D02B014201CE0190
:10F7E00085589F4F0E9457884114510429F0D70132
:10F7F00058965C924E925797B4018AE49AE00E9420
:10F8000052A18AE49AE00E94F68AF70187849088E0
:10F8100081149104D1F0CF56DF4F88819981C1596D
:10F82000D040892B91F0BE0163577F4FCE018558A0
:10F830009F4F0E948D88CE0185589F4FF4011995E6
:10F84000CE0185589F4F0E94578865E076E0CE0133
:10F8500083579F4F0E942788FFEFBF12D5CEC80164
:10F860000E940B93D12CC12CD7CECE0185589F4F2F
:10F870000E9462A79093DE068093DD067894C8010B
:10F880000E940B938091DD069091DE06892BD1F4C6
:10F8900065E076E0CE0183579F4F0E949688CE01A7
:10F8A00083579F4F0E94B6B3CE0183579F4F0E944C
:10F8B00057886CE977E180E49AE00E94C48CF12CCF
:10F8C000E12C16CF0E94F66F8091A807882329F0BB
:10F8D0000E948BA071FF0E94A61D65E977E186E377
:10F8E0009AE00E94C48C04CFE0E3EE16E1E0FE064D
:10F8F00051F461E877E186E39AE00E94C48CC80184
:10F900000E940B93F5CE69E677E180E49AE00E94CD
:10F91000C48CC8010E940B93B70180E49AE00E9456
:10F9200052A180E49AE00E94F68AE2CE66E577E191
:10F9300087EE9AE00E94C48CEE24EA94FE2CD8CE86
:10F940004F925F926F927F928F929F92AF92BF92EF
:10F95000CF92DF92EF92FF920F931F93CF93DF939B
:10F96000CDB7DEB7C157D1090FB6F894DEBF0FBED1
:10F97000CDBF8C014B01F42E642F87EE9AE00E94DC
:10F980004BA160EC7FE087EE9AE00E94C48CB4014A
:10F99000CE0101965C010E948D88B50187EE9AE048
:10F9A0000E94B68C87EE9AE00E94F68AC5010E94FA
:10F9B000578892E0F91280C16EEB7FE0C5010E948A
:10F9C0005F88D40114962D913C9115978D819E816D
:10F9D0002817390711F58D919C9169817A810097DB
:10F9E00059F06115710509F064C1232B09F4A3C115
:10F9F000DC018C9190E00DC06115710509F49BC18B
:10FA0000232B09F498C1FB01808190E091958195A9
:10FA10009109FF24F394892B09F0F12CC5010E9470
:10FA20005788FF2009F4D3C240E06DE271E0C801BD
:10FA30000E94AEB48090A3079090A40767EB7FE08C
:10FA4000CE0184599F4F0E945F8860EB7FE0CE011A
:10FA50008A599F4F0E945F88CE01865A9F4F0E940D
:10FA60005D24A096FFACA0976F96EFAC6F976E9653
:10FA7000DFAC6E976D96CFAC6D9765E076E0CE010A
:10FA800081960E949688BE016F5D7F4FC5010E94DE
:10FA90008D886C2DC5010E94A8876AEF75E00E94D1
:10FAA000D9876D2D0E94A8876AEF75E00E94D987DB
:10FAB0006E2D0E94A8876AEF75E00E94D9876F2D8E
:10FAC0000E94A887BC01CE01805A9F4F0E948D885A
:10FAD000C5010E945788CE0181960E9457886BEA23
:10FAE0007FE0CE018C5A9F4F0E945F886E01EEE44A
:10FAF000CE0ED11C65E076E0C6010E94968892E1A8
:10FB0000E92E9AE0F92E28E1622E2AE0722E2601D3
:10FB1000D70118966C9170E084E0759567958A9589
:10FB2000E1F7C5010E94EB9D4D815E8169817A817B
:10FB3000C2010E945687C5010E945788F70160855F
:10FB40006F7070E0C5010E94EB9D4D815E816981FF
:10FB50007A81C2010E945687C5010E945788FFEF33
:10FB6000EF1AFF0A6E147F0499F665EA7FE0CE0172
:10FB7000885B9F4F0E945F8863E97FE0CE0181969A
:10FB80000E945F88BE016F5D7F4FCE01805C9F4FFA
:10FB90000E948D882696EEACFFAC269788E1E80E91
:10FBA000F11CB701CE01805C9F4F0E942E8781110E
:10FBB000C5C0CE01805C9F4F0E949687BE01685BE6
:10FBC0007F4FCE01805C9F4F0E94F387B6010E9459
:10FBD000F387BE016C5A7F4F0E94F387BE01605AC3
:10FBE0007F4F0E94F387BE016A597F4F0E94F387BF
:10FBF0007C014AE0B50180E590E00E94E0D0F5018B
:10FC000001900020E9F73197AF014A195B09B5016E
:10FC1000C7010E945687811103C0C7010E949687C1
:10FC2000BE0164597F4FC7010E94F387B4010E944F
:10FC3000D987BC01C8010E94B68CC8010E94F68A0F
:10FC4000CE01805C9F4F0E945788CE0181960E9412
:10FC50005788CE01885B9F4F0E945788C2010E943F
:10FC60005788CE018C5A9F4F0E945788CE01805AE8
:10FC70009F4F0E945788CE018A599F4F0E945788F4
:10FC8000CE0184599F4F0E945788C8010E94F68A6E
:10FC900064E670E080E090E00E94FDABD801ED9159
:10FCA000FC910488F589E02DC801199501E010E068
:10FCB000EDC00E948FDCADCEB1E0FB1220C263E745
:10FCC0007FE0C5010E945F88B501C4010E94C5861E
:10FCD000582EC5010E945788552009F4D8C1EE203E
:10FCE00009F473C166E070E0C4010E94A5A84AE06F
:10FCF000B801CE01885B9F4F0E94738A4091B6077E
:10FD00005091B707F40160817181CE0181960E9404
:10FD10002C40CE0181960E949A3E811122C000E9BA
:10FD200011E0CE0181960E948F45CE01885B9F4FE6
:10FD30000E945788ABC0FF24F39470CE22962EAD5C
:10FD40003FAD229726968EAD9FAD26976AE77FE05E
:10FD5000820F931F0E946DD02696FFAEEEAE2697BF
:10FD60002DCF2A966EAD7FAD2A97CE0181960E9447
:10FD700015A4892BA1F224961CAE1DAE1EAE1FAE9B
:10FD8000249728961CAE1DAE1EAE1FAE2897229655
:10FD90008FAD2297807F22968FAF229740E050E36D
:10FDA000BE016F5D7F4FCE01805C9F4F0E94774305
:10FDB00000E020E030E340E250E0B501CE01805C9D
:10FDC0009F4F0E946B20BC01C6010E94318808EC45
:10FDD00010E1A7CFEE2009F4F8C066E070E0C4019E
:10FDE0000E94A5A84091B6075091B707D4016D9124
:10FDF0007C91CE0181960E942C40CE0181960E947A
:10FE00009A3E00E911E08823E9F18BA5873061F47F
:10FE1000CE0181960E942F4861E0892B09F462E0AF
:10FE2000CE0181960E94F81B24961CAE1DAE1EAE1C
:10FE30001FAE249728961CAE1DAE1EAE1FAE28978F
:10FE400022968FAD2297807F22968FAF229740E037
:10FE500050E3BE016F5D7F4FCE01805C9F4F0E94DB
:10FE6000774300E020E030E340E250E0B501CE010E
:10FE7000805C9F4F0E946B20BC01C6010E943188AC
:10FE800008EC10E1CE0181960E948F45C801CF5841
:10FE9000DF4F0FB6F894DEBF0FBECDBFDF91CF911D
:10FEA0001F910F91FF90EF90DF90CF90BF90AF9098
:10FEB0009F908F907F906F905F904F900895F40186
:10FEC000608171810E94CB9C7C01892B09F0C5C0A7
:10FED00004E911E0DBCFEE2009F477C069E070E0BF
:10FEE000C4010E94A5A84AE0B801C5010E94738A16
:10FEF00041E050E067EB74E0C4010E9456874D81F9
:10FF00005E8169817A81C4010E94568766E57FE03F
:10FF100087EE9AE00E94C48CB401CE0181960E94C3
:10FF20008D88BE016F5D7F4F87EE9AE00E94B68C90
:10FF300087EE9AE00E94F68ACE0181960E94578849
:10FF40006EE47FE0CE0181960E945F88F401848197
:10FF500095812DA13EA182179307E1F4892B91F1A0
:10FF6000E080F18069A07AA0D7018D917D0188237E
:10FF700049F1082E000C990B0E9414DC6C01F3016E
:10FF800081913F01082E000C990B0E9414DCC816C9
:10FF9000D90651F3CE0181960E945788552031F041
:10FFA00041E068EC70E0C8010E94AEB4D4018D91CC
:10FFB0009C910E949590009711F484E991E08C0146
:10FFC000C501B6CE55245394E5CF01E982CF6CE646
:10FFD0007FE0C5010E945F88B501C4010E94C5860B
:10FFE000F82EC5010E945788F110F4CE66E67FE036
:10FFF000C5010E945F88B501C4010E94C586F82E24
:020000021000EC
:10000000C5010E945788FF2009F479C0EE20E9F26B
:1000100065E070E0C4010E94A5A86AEF75E0C40124
:100020000E94E086882339F0E090B607F090B70789
:10003000E114F10491F465E076E0C4010E94E086E9
:10004000811107C08091B6079091B707009709F01A
:1000500036CFE090DD06F090DE0640E068EC70E21E
:10006000C8010E94AEB4C8010E94F68A1C821B829D
:1000700087E892E09A8389831E830D838FEF9FEF39
:1000800098878F83B701C5010E94CCA201CE6CE591
:100090007FE0C5010E945F88B501C4010E94C5864A
:1000A000F82EC5010E945788F11015CF61E47FE05A
:1000B000C5010E945F88B501C4010E94C586182F42
:1000C000C5010E94578800E0112309F4DFCE80E0CB
:1000D0000E9429A169E17FE086E39AE00E94C48C36
:1000E00086E39AE00E94F68A65E076E0C5010E9408
:1000F0009688C5010E94B6B3C5010E94578800E0EA
:10010000D6CD0895FC01248135816217730748F428
:1001100080819181009729F0860F971FFC018081D3
:10012000089580E0089508950895AF92BF92CF9208
:10013000DF92EF92FF920F931F93CF93DF936C01A7
:100140007B018B01040F151FEB015E01AE18BF0888
:10015000C017D10759F06991D601ED91FC9101903A
:10016000F081E02DC6011995892B79F7C501DF9142
:10017000CF911F910F91FF90EF90DF90CF90BF90A4
:10018000AF900895FC01538D448D252F30E0842FCE
:1001900090E0821B930B541710F0CF9608950197AF
:1001A0000895FC01918D828D981761F0A28DAE0F9C
:1001B000BF2FB11D5D968C91928D9F5F9F73928F23
:1001C00090E008958FEF9FEF0895FC01918D828D4F
:1001D000981731F0828DE80FF11D858D90E008951C
:1001E0008FEF9FEF0895FC01918D228D892F90E074
:1001F000805C9F4F821B91098F73992708958AE431
:100200009AE00E94F38021E0892B09F420E0822FFC
:100210000895FC01A48DA80FB92FB11DA35ABF4F9B
:100220002C91848D90E001968F739927848FA689F5
:10023000B7892C93A089B1898C91837080648C9349
:10024000938D848D981306C00288F389E02D8081F8
:100250008F7D80830895EF92FF920F931F93CF932A
:10026000DF93EC0181E0888F9B8D8C8D98131AC0F1
:10027000E889F989808185FF15C09FB7F894EE89D8
:10028000FF896083E889F989808183708064808335
:100290009FBF81E090E0DF91CF911F910F91FF9080
:1002A000EF900895F62E0B8D10E00F5F1F4F0F7328
:1002B0001127E02E8C8D8E110CC00FB607FCFACFE3
:1002C000E889F989808185FFF5CFCE010E940981F7
:1002D000F1CFEB8DEC0FFD2FF11DE35AFF4FF082B4
:1002E0009FB7F8940B8FEA89FB8980818062CFCF1A
:1002F000CF93DF93EC01888D8823B9F0AA89BB895D
:10030000E889F9898C9185FD03C0808186FD0DC047
:100310000FB607FCF7CF8C9185FFF2CF808185FF68
:10032000EDCFCE010E940981E9CFDF91CF910895F1
:1003300080E090E0892B29F00E94FF8081110E94CB
:10034000000080E090E0892B49F080E090E0892B6C
:1003500029F00E94000081110E94000080E090E0DE
:10036000892B49F080E090E0892B29F00E94000061
:1003700081110E94000080E090E0892B49F080E02C
:1003800090E0892B29F00E94000081110C9400005C
:100390000895DC01ED91FC910190F081E02D19941C
:1003A0008FEF9FEF0895FC01628973898489958995
:1003B0000895EF920F931F93CF93DF93FC01248D49
:1003C000222341F0213051F1DF91CF911F910F9104
:1003D000EF900895228933894489558986899789C0
:1003E000A08DB18D821B930BA40BB50B892F9A2F77
:1003F000AB2FBB278C010F5F1F4F628173818481FC
:100400009581CFB7F894DCB7E1E0ECBFEE24E3943C
:10041000E2E0FEEF1995DCBFCFBFD6CFF0E0E0E021
:10042000DF91CF911F910F91EF901994FC01138EE2
:10043000128E41110CC082899389A489B589868B5B
:10044000978BA08FB18F148E81E090E0089590E09B
:1004500080E00895CF92DF92EF92FF92CF93DF93E7
:10046000DC01CB01642FCFB7F8946D01EE24FF249B
:10047000CBBEDCB741E04CBFA901E1E0FEEF19952E
:10048000DCBFCFBFDF91CF91FF90EF90DF90CF9097
:100490000895CF93DF93FC01248D211110C0EC014E
:1004A000828D938D892B49F066897789808D918D16
:1004B00030E020E045E00E942A821B8E1A8EDF91F8
:1004C000CF9108951F93CF93DF93FC01248D2111C9
:1004D00045C0162FEC01828D938D892B49F46689D6
:1004E0007789808D918D30E020E043E00E942A8260
:1004F0004A8D5B8DCA0181709927FE01E80FF91FB3
:10050000158F892B69F02D8D3E8D6E897F89888DA1
:10051000998D640F751F811D911D41E00E942A82F3
:100520008A8D9B8D01969B8F8A8F81159140B1F4A6
:100530006E897F89888D998D30E020E045E00E94AA
:100540002A821B8E1A8E8E899F89A88DB98D9F5FF6
:10055000AF4FBF4F8E8B9F8BA88FB98F81E090E0FC
:10056000DF91CF911F910895DC01ED91FC91028004
:10057000F381E02D40E01994FB01448155812281F3
:100580003381215031094217530750F4A081B181C2
:10059000A40FB51F8C9384819581019695838483E4
:1005A00080E00895CF93DF93EC01E881F981028424
:1005B000F385E02DCE0119950196B9F7DF91CF9122
:1005C0000895FC01A285B3851097A9F086859785CB
:1005D000029788F0CD010196938782876C93868578
:1005E00097850197978786870284F385E02D10828F
:1005F00081E090E0089590E080E00895FC0186811C
:1006000097818F3F980729F02FEF3FEF378326839D
:100610000895A085B185109789F024853585211529
:10062000310561F0CD010196918780878C91215031
:10063000310935872487082E000C990B0895FC0199
:1006400086819781019639F481E024853585232BB5
:1006500019F480E0089581E00895CF92DF92EF923F
:10066000FF920F931F93CF93DF937C016A018B015D
:10067000D0E0C0E0CC15DD0581F0D701ED91FC9113
:100680000284F385E02DC70119958F3F980729F063
:10069000F80181938F012196EDCFCE01DF91CF91AB
:1006A0001F910F91FF90EF90DF90CF900895CF931F
:1006B000C62FDC01ED91FC910088F189E02D1995A0
:1006C000DC01ED91FC910190F081E02D6C2FCF9138
:1006D0001994062E000C770BFC017783668308952E
:1006E000CF93DF93EC018E819F81019611F5E88114
:1006F000F9810088F189E02DCE011995DC01ED9199
:10070000FC910084F185E02D1995892BB1F0E881E9
:10071000F9810284F385E02DCE011995813291058E
:1007200034F3E881F9810684F785E02D682FCE0146
:10073000199581E0DF91CF91089580E0FBCFFC0116
:1007400020812EBD9B012150310941F051810DB412
:1007500007FEFDCF4EB55EBD4193F5CF61507109E7
:10076000860F971F0DB407FEFDCF2EB5FC01208329
:100770000895E091BC07F091BD0780819091BB077F
:10078000892B80830895E091BC07F091BD0790818B
:100790008091BB0780958923808308958EBD0000DA
:1007A0000DB407FEFDCF8EB5089590E0209113099A
:1007B000233339F40C96982F990F990F990F80E0F5
:1007C00008954896F8CFEF92FF920F931F93CF931F
:1007D000DF93EC018B017A010E9430AC688B798B3E
:1007E0008A8B9B8B8C819D81DC01ED91FC91028039
:1007F000F381E02DA701B801DF91CF911F910F91F7
:10080000FF90EF9019941F93CF93DF93EC01162F75
:100810000E9430AC688B798B8A8B9B8B8C819D81FD
:10082000DC01ED91FC910190F081E02D612FDF91D1
:10083000CF911F911994CF92DF92EF92FF92CF93B5
:10084000DF93EC018E819F818F3F980759F02FEF46
:100850003FEF3F832E83DF91CF91FF90EF90DF90AA
:10086000CF9008950E9430AC6B017C01A4EFCA0EBA
:10087000A1E0DA1EE11CF11CE881F9810088F18910
:10088000E02DCE011995DC01ED91FC910084F185FC
:10089000E02D1995892B39F40E9430AC6C157D053B
:1008A0008E059F0548F3E881F9810088F189E02DE4
:1008B000CE011995DC01ED91FC910284F385E02DC8
:1008C000DF91CF91FF90EF90DF90CF9019940E942D
:1008D0000FDC0F931F93CF93DF938C01C0E0D8E020
:1008E000688179816115710529F0C8010E948FDC4A
:1008F000892B29F00B80DC81C02D209789F7CE0150
:10090000DF91CF911F910F9108950C94C7CEEF9274
:10091000FF920F931F93CF93DF93009751F4CFEF84
:10092000DFEFCE01DF91CF911F910F91FF90EF90FC
:100930000895DC011C96ED90FC90F7010081118177
:10094000D801ED91FC910688F789E02DC801199531
:10095000882329F3D801ED91FC910084F185E02DE5
:10096000C8011995D801ED91FC91892B61F302849E
:10097000F385E02DC8011995EC01019681F2F8018B
:10098000818D882329F06C2F8AE49AE00E944BA184
:10099000D70112968C91882321F2C532D10509F630
:1009A000D801ED91FC910084F185E02DC8011995E5
:1009B00002975CF0D801ED91FC910688F789E02D53
:1009C000C80119958111ECCFAACFD1E0C0E0D801C0
:1009D000ED91FC910284F385E02DC80119958F3FBC
:1009E000980709F49CCF9C01215431092A31310523
:1009F00070F48D2F8295807F829FC00D1124D111BC
:100A000004C00C2E000CDD0B8CCFD0E0E0CF9C019D
:100A1000215631092A31310560F3C0978A3091059A
:100A200070F79D2F9295907F989FC00D1124E7CF6E
:100A3000CF92DF92EF92FF920F931F93CF93DF93AA
:100A40006C018B0186E090E00E942BCEEC0190932C
:100A5000060880930508F60101900020E9F7CF0110
:100A60008C199D090E942BCE7C01B6010E9498DC56
:100A7000F60101900020E9F73197EC19FD09EE0D20
:100A8000FF1D1082F982E8821B830A83809143084C
:100A9000909144089D838C83D0934408C09343086D
:100AA000DF91CF911F910F91FF90EF90DF90CF904A
:100AB0000895FC01868197818F3F980729F02FEFD9
:100AC0003FEF378326830895808591850C94B9D1B3
:100AD0007F928F929F92AF92BF92CF92DF92EF92CE
:100AE000FF920F931F93CF93DF93CDB7DEB7A697F7
:100AF0000FB6F894DEBF0FBECDBF8C01762E942EBC
:100B0000852E20E2A22ECE0101967C01DC01EA2D89
:100B10001D92EA95E9F76801F3E4CF0ED11C8CE24F
:100B200094E09AA389A38FEF8BA38CA38DA38EA3AC
:100B300043E450E0BE016F5D7F4FC6010E94A023D9
:100B4000019609F4BFC081E089838A8386E0B82ECC
:100B5000BB821C82D80114966D917D918D919C91E0
:100B600017970E9436D86D837E838F8398878986F6
:100B70009A8680E890E09C878B874CE150E0B70133
:100B8000C6010E943523FE0137968AE1DF011D92DE
:100B90008A95E9F74801B8E08B0E911CF401D70162
:100BA00001900D92BA94E1F740E150E0B701C6011F
:100BB0000E943523F7011192AA94E9F796E0A92E35
:100BC000B12C40E250E0B701C6010E943523F1E0AC
:100BD000AF1AB108B1F783E6898392E89A8393E567
:100BE0009B838C8385E38D8381E08E837F829DE36D
:100BF000988797E099878A8786E0F401DE011B9643
:100C000001900D928A95E1F78CE0898B8A8B6CEFCD
:100C100075E0CE0143960E9498DCD8011B966C913A
:100C2000CE0149960E9480A7F8016485CE014B96BB
:100C30000E9480A7D8011D966C91CE014D960E940E
:100C400080A74EE150E0B701C6010E943523B3E012
:100C50007B121EC082E3898384E08A83F801968533
:100C60009B8397859C8390899D8391899E8396E33E
:100C70009F838887828D8987838D8A87848D8B87E0
:100C8000858D8C874CE050E0B701C6010E9435236A
:100C900087E3898386E08A8391E09B8393E09C834A
:100CA0008D838FE08E838AE38F838BE388878FEF3A
:100CB000898749E050E0B701C6010E943523C6018B
:100CC0000E946F23A6960FB6F894DEBF0FBECDBF6D
:100CD000DF91CF911F910F91FF90EF90DF90CF9018
:100CE000BF90AF909F908F907F90089590E080E0AC
:100CF0000C94EB22CF93DF93C4E1D0E00E94768680
:100D0000882361F061E070E080E090E00E94FDAB3C
:100D10002197A1F780E0DF91CF91089581E0FBCF8B
:100D2000FF920F931F93CF93DF931F921F92CDB724
:100D3000DEB7F82E22E030E0AE014F5F5F4F66E293
:100D400070E00E940E2309811A81102701271027C5
:100D500022E030E0AE014F5F5F4F66E270E08F2D22
:100D60000E940E2389819A8198278927982708173E
:100D7000190749F4C8010F900F90DF91CF911F918F
:100D80000F91FF9008958C01E3CFFB0144815581C1
:100D9000FC01248135812417350778F08081918109
:100DA000009759F0FB01608171816115710529F08F
:100DB0000E94AFDC21E0892B09F020E0822F08950A
:100DC000FC0124813581232B39F421E0FB01808152
:100DD000882349F020E007C0808191810E948FDC48
:100DE00021E0892BB9F7822F08950F931F93CF939A
:100DF000DF938C01EB01FC01808191810097E1F090
:100E00006881798161157105A9F0428153812C8136
:100E10003D814217530770F00E9498DC8C819D81C0
:100E2000F801958384831D821C82DF91CF911F91ED
:100E30000F9108950E94C7CE88819981F80191830E
:100E400080838A819B81938382838C819D8195831A
:100E50008483198218821B821A82E5CF0F931F9315
:100E6000CF93DF93EC0188819981009759F02A8113
:100E70003B812617370730F081E0DF91CF911F913A
:100E80000F9108958B016F5F7F4F0E942EDB0097BB
:100E900059F0998388831B830A832C813D81232BFE
:100EA00059F7FC011082E8CF80E0E7CFEF92FF9284
:100EB0000F931F93CF93DF936115710541F480E089
:100EC000DF91CF911F910F91FF90EF900895411501
:100ED0005105B1F07B01EC010C811D81040F151F40
:100EE000B8010E942E87882351F3288139818C8193
:100EF0009D81B701820F931F0E9498DC1D830C8394
:100F000081E0DECFCF93DF931F921F92CDB7DEB784
:100F100069831A8241E050E0BE016F5F7F4F0E94FB
:100F200056870F900F90DF91CF910895CF93DF9365
:100F3000EC0188819981009711F00E94C7CE198237
:100F400018821D821C821B821A82DF91CF91089524
:100F5000EF92FF920F931F93CF93DF9300D01F92D6
:100F6000CDB7DEB77C01862F4AE08E010F5F1F4FA1
:100F7000B80190E00E94E0D0F80101900020E9F76C
:100F80003197AF01401B510BB801C7010E94568732
:100F9000811103C0C7010E949687C7010F900F906F
:100FA0000F900F90DF91CF911F910F91FF90EF90D5
:100FB0000895CF93DF93EC016115710539F4CE01EB
:100FC0000E949687CE01DF91CF910895FB01019099
:100FD0000020E9F73197AF01461B570B0E94568757
:100FE000882369F3EFCFCF93DF93EC01FB014481BA
:100FF0005581608171810E945687811103C0CE01A5
:101000000E949687CE01DF91CF910895EF92FF92D3
:101010000F931F93CF93DF93EC017B018A01BA01F9
:101020000E942E8781110BC0CE010E949687CE01AF
:10103000DF91CF911F910F91FF90EF9008951D8345
:101040000C83B701888199810E9498DCF0CFFB0165
:1010500001900020E9F73197AF01461B570B0C9424
:101060000688CF93DF93EC016115710531F00E9482
:101070002788CE01DF91CF9108950E949687F9CFFE
:10108000CF93DF93EC01FB018617970749F060814E
:1010900071816115710541F0448155810E94068876
:1010A000CE01DF91CF9108950E949687F9CFFC0180
:1010B00080819181009711F00C94C7CE0895EF9232
:1010C000FF920F931F93CF93DF93EC018B01198253
:1010D00018821B821A821D821C82CB010E9474D04E
:1010E0007C01BC01CE010E942E87811109C0CE0176
:1010F000DF91CF911F910F91FF90EF900C94968705
:10110000FD82EC82B80188819981DF91CF911F9196
:101110000F91FF90EF900C946DD0FC011182108222
:1011200013821282158214820C944088FC01118271
:1011300010821382128215821482FB01019000201A
:10114000E9F73197AF01461B570B0C940688AF9215
:10115000BF92CF92DF92EF92FF920F931F93CF93A4
:10116000DF935C016B017A0189012417350720F4B4
:101170008F2D7901042F182F65E076E0C5010E94BC
:101180009688D6011496CD91DC91EC16FD06C8F434
:101190000C171D0708F4E801D601ED91FC91119799
:1011A000EC0FFD1F108110826D917C916E0D7F1DE3
:1011B000C5010E943188F60180819181C80FD91F35
:1011C0001883C501DF91CF911F910F91FF90EF9090
:1011D000DF90CF90BF90AF9008951F920F920FB6FF
:1011E0000F9211240BB60F922F933F934F935F935F
:1011F0006F937F938F939F93AF93BF93EF93FF93DF
:10120000E0911202F09113021995FF91EF91BF91B5
:10121000AF919F918F917F916F915F914F913F918E
:101220002F910F900BBE0F900FBE0F901F9018952F
:101230001F920F920FB60F9211240BB60F922F939D
:101240003F934F935F936F937F938F939F93AF934E
:10125000BF93EF93FF93E0911002F0911102199563
:10126000FF91EF91BF91AF919F918F917F916F917E
:101270005F914F913F912F910F900BBE0F900FBE3A
:101280000F901F9018951F920F920FB60F92112476
:101290000BB60F922F933F934F935F936F937F9370
:1012A0008F939F93AF93BF93EF93FF93E0910602C9
:1012B000F09107021995FF91EF91BF91AF919F9126
:1012C0008F917F916F915F914F913F912F910F90EF
:1012D0000BBE0F900FBE0F901F9018951F920F928C
:1012E0000FB60F9211240BB60F922F933F934F938B
:1012F0005F936F937F938F939F93AF93BF93EF937E
:10130000FF93E0910402F09105021995FF91EF918E
:10131000BF91AF919F918F917F916F915F914F910D
:101320003F912F910F900BBE0F900FBE0F901F900B
:1013300018951F920F920FB60F9211240BB60F92B1
:101340002F933F934F935F936F937F938F939F93CD
:10135000AF93BF93EF93FF93E0910E02F0910F02D2
:101360001995FF91EF91BF91AF919F918F917F91CF
:101370006F915F914F913F912F910F900BBE0F9006
:101380000FBE0F901F9018951F920F920FB60F92DD
:1013900011240BB60F922F933F934F935F936F934C
:1013A0007F938F939F93AF93BF93EF93FF93E091BE
:1013B0000C02F0910D021995FF91EF91BF91AF9141
:1013C0009F918F917F916F915F914F913F912F915D
:1013D0000F900BBE0F900FBE0F901F9018951F928D
:1013E0000F920FB60F9211240BB60F922F933F93CB
:1013F0004F935F936F937F938F939F93AF93BF931D
:10140000EF93FF93E0910A02F0910B021995FF917F
:10141000EF91BF91AF919F918F917F916F915F916C
:101420004F913F912F910F900BBE0F900FBE0F90D9
:101430001F9018951F920F920FB60F9211240BB6A2
:101440000F922F933F934F935F936F937F938F935D
:101450009F93AF93BF93EF93FF93E0910802F091B6
:1014600009021995FF91EF91BF91AF919F918F91D3
:101470007F916F915F914F913F912F910F900BBE94
:101480000F900FBE0F901F9018950F931F93CF933F
:10149000DF93EC010E9430AC688779878A879B874D
:1014A000E881F9810284F385E02DCE01199597FF3B
:1014B00015C00E9430AC088519852A853B85601BC4
:1014C000710B820B930B0C811D812E813F81601764
:1014D00071078207930720F38FEF9FEFDF91CF9182
:1014E0001F910F910895EF92FF920F931F93CF9347
:1014F000DF93EC017B01042F65E076E00E94968883
:10150000C7010E94458A002E000C110B97FD0BC0ED
:101510000817190741F0682FCE010E948287C70182
:101520000E94458AF3CFCE01DF91CF911F910F9199
:10153000FF90EF900895FB0101900020E9F73197AB
:10154000AF01461B570BDC01ED91FC910280F3814A
:10155000E02D19948F929F92AF92BF92EF92FF92DB
:101560000F931F93CF93DF93CDB7DEB7A1970FB63D
:10157000F894DEBF0FBECDBF7C01FA01CB0119A2EA
:10158000223008F42AE08E010F5D1F4F822E912C2D
:10159000B12CA12CBF01A50194010E94A3D7F90190
:1015A000CA016A300CF5605DD8016E938D01232B62
:1015B000242B252B79F790E080E0109721F0BD01D6
:1015C000C7010E949B8AA1960FB6F894DEBF0FBE9A
:1015D000CDBFDF91CF911F910F91FF90EF90BF9002
:1015E000AF909F908F900895695CDECF63E076E0C6
:1015F0000C949B8ADC01ED91FC910190F081E02D2F
:1016000019942F923F924F925F926F927F928F9296
:101610009F92AF92BF92CF92DF92EF92FF921F9371
:10162000CF93DF93EC016A017B01722EAB0196012F
:10163000CB01B6010E94C1D966E076E0811126C0D7
:1016400046015701E894B7F82FEF3FEF4FE75FE708
:10165000C501B4010E94C1D981110CC02FEF3FEF29
:101660004FE75FE7C501B4010E9459D66AE076E012
:10167000181664F02FEF3FEF4FE75FE4C701B601A4
:101680000E9461D91816B4F46EE076E0CE01DF91C5
:10169000CF911F91FF90EF90DF90CF90BF90AF90D0
:1016A0009F908F907F906F905F904F903F902F9082
:1016B0000C949B8A2FEF3FEF4FE75FECC701B60119
:1016C0000E9459D687FDE0CF20E030E0A901C70194
:1016D000B6010E9459D6312C212C87FF09C06DE23A
:1016E000CE010E94FA8A1C01F7FAF094F7F8F09400
:1016F00010E060E070E080E09FE3711641F020E0D0
:1017000030E040E251E40E94B9D81F5FF6CFA70154
:1017100096010E944DD82B013C010E9432D94B0109
:101720005C012AE0BC01A401CE010E94AA8A7C01CE
:10173000E20CF31C1123C1F1C501B4010E945ED675
:101740009B01AC01C301B2010E944CD84B015C016A
:101750006EE2CE010E94FA8AE80EF91E115020F1C5
:1017600020E030E040E251E4C501B4010E94BFD660
:101770002B013C010E9432D94B01B12CA12C2AE053
:10178000B501A401CE010E94AA8AE80EF91EC50186
:10179000B4010E945ED69B01AC01C301B2010E945C
:1017A0004CD84B015C01DACFC701DF91CF911F917B
:1017B000FF90EF90DF90CF90BF90AF909F908F9071
:1017C0007F906F905F904F903F902F900895CF92B1
:1017D000DF92EF92FF920F931F93CF93DF93211528
:1017E000310581F4DC01ED91FC910190F081E02D57
:1017F000642FDF91CF911F910F91FF90EF90DF90B9
:10180000CF9019942A30310501F52AE077FF1DC0E9
:101810006A017B01EC016DE20E94FA8A8C01442787
:101820005527BA014C195D096E097F092AE0CE01DE
:101830000E94AA8A800F911FDF91CF911F910F9173
:10184000FF90EF90DF90CF900895DF91CF911F919F
:101850000F91FF90EF90DF90CF900C94AA8A8F9217
:101860009F92AF92BF92CF92DF92EF92FF920F932F
:101870001F93CF93DF937C018B014C0182E0880E94
:10188000911C5701E5E0AE0EB11CD0E0C0E0F401C0
:1018900061914F01C8010E944BA16C016EE2C80129
:1018A0000E94FA8A8C0D9D1DC80FD91F8A149B04B3
:1018B00071F7F7016581C8010E944BA18C0F9D1F34
:1018C000DF91CF911F910F91FF90EF90DF90CF901C
:1018D000BF90AF909F908F9008956115710511F0A2
:1018E0000C949B8A90E080E008950F931F93CF9310
:1018F000DF93EC0162E176E08AE49AE00E946D8C6D
:101900004A855B856C857D858A819B81AC81BD81A3
:10191000481B590B6A0B7B0B8E859F85A889B9895B
:10192000481B590B6A0B7B0B2AE08AE49AE00E9461
:10193000AA8A8AE49AE00E94F68A6A857B858C8569
:101940009D850A811B812C813D81601B710B820B5F
:10195000930B0E851F8528893989601B710B820BBB
:10196000930BDF91CF911F910F910895DB01149696
:101970004D915C9115976D917C91DC01ED91FC91FD
:101980000280F381E02D1994EF92FF920F931F9341
:10199000CF93DF938C017B01D0E0C0E0F701EC0F27
:1019A000FD1F6491662361F0D801ED91FC910190D7
:1019B000F081E02DC8011995892B11F02196EECF09
:1019C000CE01DF91CF911F910F91FF90EF9008957D
:1019D0000F931F93CF93DF93EC010E94C48C8C0173
:1019E000CE010E94F68A800F911FDF91CF911F9147
:1019F0000F9108958AE49AE00E94F68A6FE77DE1EC
:101A00008AE49AE00C94C48CDC018CE294E08D931F
:101A10009D9384E0FB0101900D928A95E1F7089572
:101A20003F924F925F926F927F928F929F92AF926E
:101A3000BF92CF92DF92EF92FF920F931F93CF93BB
:101A4000DF93CDB7DEB7EA970FB6F894DEBF0FBECF
:101A5000CDBF7C012A013B0169010E9430AC4B01E2
:101A60005C0187010D5B1F4FC8010E94C218181648
:101A70001906ACF00E9430AC681979098A099B09F3
:101A8000461657066806790608F468C10E94A96FD1
:101A900061E070E080E090E00E94FDABE5CF42E2C3
:101AA00050E0BE016F5F7F4FC8010E944D188981D1
:101AB0008230D1F0312C832DEA960FB6F894DEBF38
:101AC0000FBECDBFDF91CF911F910F91FF90EF908F
:101AD000DF90CF90BF90AF909F908F907F906F904E
:101AE0005F904F903F900895F801848995898334E1
:101AF000910501F76D817E818F8198850E9436D88E
:101B00004B015C01F60180829182A282B38246E0A1
:101B100050E0B701685F7F4FCE014D960E943EDCDA
:101B2000892B41F6F70180819181A281B3818816CA
:101B30009906AA06BB0608F4BDCF84819581A681CB
:101B4000B78188159905AA05BB0508F4B3CF898923
:101B50009A89AB89BC8986879787A08BB18B4EEC1D
:101B600050E070E060E0C8010E944D18312CC701C0
:101B7000829698AB8FA7F701B696FAABE9AB0896B9
:101B80009CAB8BAB67019AE1C90ED11CBD96FEAB35
:101B9000EDABC701429698AF8FABFD97FAAFE9AFB7
:101BA0004701FEE18F0E911CF801818D928D181670
:101BB00019060CF080CFC8010E946C188333910580
:101BC00009F4B2C014F58130910509F464C044F4FD
:101BD000892B51F3C8010E946C18AC01552775C0C0
:101BE0008330910509F462C00697A1F7C8010E94ED
:101BF0006C18B82E44E050E0B401C8010E944D18A2
:101C0000EB2DE450FF0BAF0160C08A33910509F45E
